:020000040800F2
:1000000000000220CD9F0008B59F0008B59F0008A2
:10001000B59F0008B59F0008B59F000800000000CC
:10002000000000000000000000000000B59F000874
:10003000B59F000800000000B59F0008BD9F0008A4
:10004000B59F0008B59F0008B59F0008B59F000840
:10005000B59F0008B59F0008B59F0008B59F000830
:10006000B59F0008B59F0008B59F00081519000846
:10007000B59F0008B59F0008B59F0008B59F000810
:10008000B59F0008B59F0008F1070008B59F00085C
:10009000B59F0008B59F0008B59F00089D0900089E
:1000A000B59F0008B59F0008B59F0008B59F0008E0
:1000B000610A0008810A0008B59F0008AD0E00081B
:1000C000C5160008B59F0008B59F0008B59F000839
:1000D000B1090008850D0008B59F0008B59F00080C
:1000E000B59F0008B59F0008B59F0008B59F0008A0
:1000F000B59F0008B59F0008B59F000825190008A6
:10010000B59F0008B59F0008B59F0008B59F00087F
:10011000B59F0008B59F0008B59F0008B59F00086F
:10012000B59F0008B59F0008B59F0008B59F00085F
:10013000B59F00080000000000000000B59F000807
:10014000B59F0008B59F0008B59F0008B59F00083F
:10015000B59F0008B59F0008B59F0008B59F00082F
:10016000B59F0008B59F0008B59F0008B59F00081F
:10017000B59F0008B59F0008B59F0008000000006B
:1001800000000000B59F0008000000000000000013
:10019000B59F00080000000000000000B59F0008A7
:1001A000000000000000000000000000B59F0008F3
:1001B000B59F0008B59F0008B59F0008B59F0008CF
:0401C000B59F0008DF
:10020000BFF34F8F0549064BCA6802F4E060034311
:10021000CB60BFF34F8F00BFFDE700BF00ED00E0F4
:100220000400FA0500B51A4BDB68C3F30223C3F1DF
:10023000070EBEF1040F03F1040C28BF4FF0040EAB
:10024000BCF1060F1CD9A3F1030C4FF0FF3303FAE6
:100250000CF322EA03024FF0FF3303FA0EF321EA14
:10026000030101FA0CF313431A01D1B2421C0AD064
:1002700000F1604000F5614C8CF800135DF804FB60
:1002800000229446E7E7024B83F823105DF804FB55
:1002900000ED00E0F0B583B06F4A876D166800236B
:1002A0000193C36D3D68082202FA03F12942044616
:1002B00004D001680868400700F1A18067489840B1
:1002C000284204D021684A69110600F19180644AED
:1002D0009A402A4204D021680868800700F1818092
:1002E00010209840284203D021680A68110766D47C
:1002F0004FF0200C0CFA03F0284215D025682A682C
:10030000D50611D5B86094F83510052935D0276881
:100310003B68580340F187803B68190340F19280A5
:10032000E56B0DB12046A847606D002845D0626D91
:10033000D2071BD527684B4D052184F835103B6843
:10034000A5FB061623F00100B20A386003E021681D
:100350000B68DB0704D5019F013797420197F6D957
:100360000025012084F8345084F83500E36C23B371
:10037000204603B0BDE8F04018472668326822F0F6
:10038000160131602568686920F080036B61266C76
:10039000002E5CD021680D6825F008000860E66D2D
:1003A0003F23B340BB60236D00274FF0010C84F85E
:1003B000347084F835C0002BDAD103B0F0BDB860DA
:1003C00023681868400327D41968CA0503D41A683B
:1003D00022F008001860216C09B120468847E36DBF
:1003E00086E7BA60636D43F004026265E36D77E708
:1003F000B860636D43F002006065E36D67E70B680A
:1004000023F004000860E16D8A40BA60626D42F03A
:1004100001036365E36D51E71B681903DBD5A16C2C
:100420000029DAD1DBE7386810F480757FF478AF03
:100430003A6822F010013960012784F8345084F8BA
:1004400035706DE7656C002D7FF46CAF6CE7A26CC6
:10045000002A9FD1A3E700BF000000200100800018
:1004600004008000B5814E1B2DE9F04F0023734D31
:10047000734C83B04FF0010E4FF0030903E00133DA
:10048000102B00F0BF800F680EFA03F202EA070A91
:1004900032EA0707F3D14F6827F01006022E14D175
:1004A000DF0800EB870803F007064FEA860CD8F850
:1004B00020B00F690F2606FA0CF607FA0CF72BEAA4
:1004C00006063743C8F820704F68D0F800B007F030
:1004D00003064FEA430806FA08F709FA08F62BEA7A
:1004E000060C47EA0C0707604F6827F0100B0BF16A
:1004F000FF37012F6FEA060612D8876806EA070C55
:10050000CF6807FA08FB4BEA0C0787604F68D0F802
:1005100004C0C7F300179F402CEA0202174347604C
:10052000C7688A683E4002FA08F73E43C6604A68D8
:10053000D600A4D5002701976E6C46F480426A6409
:100540006F6C23F0030807F48046019608F1804B96
:10055000019A0BF59C3203F003074FEA870C0F2634
:10056000976806FA0CF627EA0607364EB0421DD009
:1005700006F58068404548D0334EB0424AD0DFF897
:10058000CCB058454BD0DFF8C88040454CD0DFF8A0
:10059000C4B058454DD0DFF8C08040450CBF4FF087
:1005A00006084FF0080808FA0CF6374397604A68C7
:1005B00026686FEA0A0CD20354BF0CEA06064AEA20
:1005C000060626604A686768960354BF0CEA070768
:1005D0004AEA070767604E68A768F20254BF0CEA50
:1005E00007074AEA0707A7604E68E268B60203F108
:1005F000010354BF0CEA02024AEA0202102BE26035
:100600007FF441AF03B0BDE8F08F012606FA0CF687
:100610003743CBE7022606FA0CF63743C6E7032634
:1006200006FA0CF63743C1E7042606FA0CF6374300
:10063000BCE7052606FA0CF63743B7E70038024058
:10064000003C01400000024000080240000C024053
:10065000001002400014024000180240836B93F81F
:100660003D1093F83E202129C8B2D2B228D02228CA
:1006700024D01968086820F480620A601968086844
:1006800040F400720A601968486820F480524A6099
:10069000196848684FF0000C20F400624A60A3F823
:1006A0002AC0186C48B94FF0200C83F83DC093F86D
:1006B0003E1083F83E0040290FD07047202AD8D141
:1006C00019684A6822F400624A6019680020588557
:1006D0004B6843F44070486070477047836B1868FC
:1006E000026800214FF0200C22F4806202605985DC
:1006F00083F83DC083F83E10196C41F01000186477
:10070000704700BF836B1868016821F48061016045
:10071000586B00225A850265996B4FF0200C0A65D0
:1007200093F83D0083F83DC083F83E20704700BF3A
:100730002D4A0368904210B43CD0B0F1804F27D0CE
:10074000A2F57C44A04223D004F5806C60451FD004
:100750000CF58062904241D002F57844A04229D045
:10076000224A904218D002F5806C604514D00CF5F6
:100770008064A04210D0A4F5983290420CD002F5CB
:10078000806C604508D00CF58064A04208D103E07D
:100790004A6823F070031343CA6823F44073134379
:1007A00003608C68C4620968816201235DF8044BB0
:1007B000436170474C68CA6823F07003234323F4F5
:1007C0004073134303608A68C2620C6884620969DB
:1007D000016301235DF8044B436170474C68CA68AC
:1007E00023F070032343D8E700000140004001409C
:1007F000694A536819685868890701D580064DD43D
:1008000019685868490701D5000618D4196858684E
:10081000C90701D5410606D419685868890601D56B
:1008200041017FD470471968C807F5D5516C6FF046
:10083000010041F48031516418605368ECE7516C59
:10084000C90603D4506C40F400515164986810F408
:10085000401F1ED1996B11F4401F02D098684005CB
:1008600017D45968490514D49968D06901F04051EA
:1008700001430ED1586820F080015960506C20F47B
:1008800080515164506CC00503D4516C41F001009B
:1008900050646FF00C0119605368B7E7516CC906DA
:1008A00003D4506C40F4007151649968D06901F030
:1008B0004051014340D0D96C44F27C7089B200FBB6
:1008C00001F1C1F30F3C42F61F308445A2F84CC041
:1008D00059D942F62D418C4558D942F6E550844508
:1008E00057D943F2C7218C458CBF4FF0040C4FF011
:1008F000030C92F8400082F84EC001280DD001216F
:1009000082F84010986820F0010199609868C0074B
:1009100026D54FF0000C82F840C06FF0120119602C
:1009200053686DE7916C6FF0200041F00201916413
:100930001860526810607047D86A10F4700F1ED1AA
:10094000586820F020015960506C20F48071516487
:10095000506CC104AFD4516C41F001005064AAE75F
:10096000596821F0806020F020015960506C20F41B
:10097000885C2CF0010141F001005064C9E79968DE
:10098000480598D4DCE74FF0000CB2E74FF0010CBB
:10099000AFE74FF0020CACE740000120034B5A696F
:1009A000D00544BF4FF4807058617047003C01404F
:1009B00010B40A4B0A4A186DD3F88810C4680C802A
:1009C000196D4B684FF400744FF4806023F04003BE
:1009D0004B60946190615DF8044B704740000120CA
:1009E0000004024010B41B4A02F1A8031168116D03
:1009F000146883B0C2F88000C2F8883003E013683E
:100A00001B1B642B17D88B689B07F8D50288CA601C
:100A100000200190CC6801948B680193019B4A6887
:100A200042F0400048600C6844F040030B6003B0A3
:100A30005DF8044B7047084B08249C614FF400623A
:100A4000402080214FF480549A61986199619C61A3
:100A5000FEE700BF4000012000000240704700BFD9
:100A600010B54FF080442369DB0706D50348416881
:100A70008847226922F00103236110BD0000002095
:100A80004A4B1869C10700D47047494B93F8AA2014
:100A90004AB193F8AB2062B946494FF4805088615F
:100AA000013283F8AB20414A136923F0010111613F
:100AB000704793F84E10481CB2EB400F6DDB0429D1
:100AC0006BD0122AECD910B493F8404083B00022C6
:100AD000012C019255D05968012083F840008C68A0
:100AE000E20714D4344A354C12688868A4FB0242E9
:100AF000940C04EB440240F0010088600192019CD8
:100B00002CB10198421E0192019C002CF9D18868F9
:100B1000C40736D55A6C22F4E06424F0010040F496
:100B200080725A644C68600505D5586C20F4405CAE
:100B30004CF480525A645C6C14F4805018BF986C6A
:100B40004FF0000418BF20F006006FF022029864F6
:100B500083F840400A60596819484C6844F0806C3A
:100B60004CF020024A604068C20602D0154CA142F7
:100B700007D18A6812F0405F03D1886840F0804452
:100B80008C600A4A002183F8AB10136923F001003E
:100B9000106103B05DF8044B70470648416981F469
:100BA000805C4CF0805181618BE700BF0004004005
:100BB00040000120000002400000002083DE1B43B3
:100BC00000230140002001406B4B93F8E520202AD0
:100BD00001D00020704710B5684A212483F8E54011
:100BE00005294FF04004946140F29180002800F004
:100BF0008E804FF4047CA3F8ECC000EB010C0139AB
:100C000011F003014FF0020236D010F8014B102C06
:100C100004D183F8EE4010F8014C032203EB020EDE
:100C200001298EF8EC4002F1010225D0022911D0F1
:100C300010F8011B102906D19C18013284F8EC1021
:100C400010F8011C92B2541C1A4482F8EC10A2B2A3
:100C5000FC2A5CD810F8011B102906D19C1801321F
:100C600084F8EC1010F8011C92B2541C1A4482F85B
:100C7000EC10A2B2FC2A4AD810F8011B102906D1A8
:100C80009C18013284F8EC1010F8011C92B203EBAE
:100C9000020E541C84458EF8EC10A1B247D0FC29FA
:100CA00035D8024612F801EBBEF1100F06D15C18E0
:100CB000013184F8ECE012F801EC89B24A1C92B2DE
:100CC0001944FC2A81F8ECE021D890F801E0BEF14B
:100CD000100F06D19C18013284F8ECE090F801E086
:100CE00092B2511C8CB21A44FC2C82F8ECE00ED863
:100CF00090F802E0BEF1100F00F1030033D021465E
:100D00004C1CA2B21944FC2A81F8ECE0B4D91B4A6D
:100D10001B48C3F8CC004FF0000C20214FF4800496
:100D200083F8E510A3F8D2C09461002010BD901C98
:100D300013FA80FC19441248C3F8CC000332A3F81C
:100D4000D220D3F8AC400D4A1020032381F8EC00E8
:100D50008CF8EC30E3684FF4800143F08003E360EB
:100D60009161012010BD1A19013482F8ECE010F8ED
:100D700001ECA1B2C4E700BF40000120000802401E
:100D80002C01012070B5474CD4F8AC301A68D968F2
:100D9000950601D5880629D4160601D50D0604D47A
:100DA000500601D54A0619D470BDD4F8CC20511C88
:100DB000C4F8CC1010785860B4F8D2C00CF1FF35EC
:100DC000AEB2A4F8D260002EEED1DC6824F080022E
:100DD000DA60D96841F04000D86070BDD86820253D
:100DE00020F04006DE6084F8E55070BD2E4DD4F84A
:100DF000F021A8685B68111ADBB2882984F8EC310D
:100E00000DD90021102BC4F8F00184F8F41184F8F6
:100E1000F511C9D14FF0010C84F8F5C170BD94F8FB
:100E2000F5619EB3022B94F8F4610ED0032B1FD012
:100E3000102B13D1002EB7D04FF0000C501C84F8AB
:100E4000F5C1C4F8F001137070BD4EB9012284F8E9
:100E5000F56184F8F421C4F8F00170BD002EA3D030
:100E60000025C4F8F00184F8F45184F8F55170BD00
:100E7000002E99D00529F3D942798B1F9A42EFD1E0
:100E8000D4F8F81101B18847A860E9E7102BC1D068
:100E900094F8F461002E87D0501CC4F8F001137050
:100EA00070BD00BF4000012000000020F0B5B04B35
:100EB000D3F8FC2195695169546893F83A021028D7
:100EC0008BB04BD0C6B2402E48D0AA48084000286C
:100ED00000F0C880A00500F15B81A74F2F40A74D0F
:100EE0000D40002F00F0F280A54F0F40002F00F0C2
:100EF0006D81660540F16A81002D40F06A8193F8AA
:100F00003952B3F826C21FFA8CF1EEB221B3D3F8EE
:100F10002002441CC3F8204207781761B3F8265218
:100F200005F1FF3C1FFA8CF1A3F82612B3F8260254
:100F300084B28CB9292E0FD1566826F480672820F8
:100F4000576093F8395293F83A2205F003010A43A7
:100F5000C3F82C2283F839020BB0F0BD11F0011F49
:100F600030D0A00500F1EA80834A84482A40084036
:100F7000002A4AD0824A0A40002A42D0670540D55A
:100F8000002800F08081A605E6D5D3F8285293F812
:100F900039022128E0D1B3F82642D3F8FC61A7B288
:100FA000002F00F05282D3F820727A1CC3F820225E
:100FB00039783161B3F826C20CF1FF36B5B2A3F827
:100FC0002652C9E76F480840002840F0AF80694EBC
:100FD0000E40002EC8D0A605C6D593F83A72FEB2D0
:100FE000D3F82872D3F82CE293F839C2BCF1220F5F
:100FF00000F0888101905069019092690192019AF4
:10100000B2E70028BFD10BB0F0BD5F4D0D402DB34E
:10101000650523D5002800F0F480A4059CD5D3F8FD
:101020002842B3F82662D3F8FC11B7B2032F00F0C0
:10103000B581B3F8260282B2022A00F0C681D3F845
:1010400020520C696E1CC3F820622C70B3F826C2C3
:101050000CF1FF37B9B2A3F826127DE70028DCD1E6
:101060000BB0F0BD494F0F40002F3FF436AFA7053E
:101070007FF533AF93F839C2546824F4E0665660C4
:10108000099057690997146844F001061660D3F86F
:10109000FC71099A3A68ACF1280122F480640229B3
:1010A0005FFA8CF53C6040F25081D3F82C02222884
:1010B00002D0222D7FF450AF00254FF0200CC3F852
:1010C0002C5283F839C283F83A5245E72E4808403B
:1010D000002860D060055ED5002D5FD193F83942BD
:1010E000B3F826128FB2E6B2002F3FF435AFD3F833
:1010F00020521269681CC3F820022A70B3F826C275
:101100000CF1FF34A1B2A3F82612B3F82672BDB2D7
:10111000002D7FF421AF2A2E7FF41EAFD3F8FC619F
:10112000726822F48064282074600AE7A7057FF5BE
:101130001BAFD3F84072F8B2106115E793F83A622A
:10114000402E00F00D81D3F80C72B7F5804F00F0FF
:10115000CC80D3F84C02002840F00B81D3F8400239
:10116000C61106F0060747F0F0001061FCE600BF6C
:1011700040000120020001000400100004000100F2
:101180008000010008000100400001001000010083
:1011900093699369E0E6002D3FF4DEAEA1057FF58B
:1011A000DBAEB3F82642A1B200293FF4D5AED3F8A6
:1011B00020621269771CC3F820723270B3F826C21D
:1011C0000CF1FF35A8B2A3F82602C5E6002D3FF4C6
:1011D000C3AEA4057FF5C0AEB3F826C21FFA8CF1EA
:1011E00000293FF4B9AED3F820526E1CC3F8206238
:1011F00028781061B3F82622541EA7B2A3F82672ED
:10120000AAE693F8390222287FF4A6AEB3F826C2E4
:10121000D3F8FC111FFA8CF2032A3FF610AF951E8B
:10122000012DD3F8284240F260810E68022C14BFD1
:1012300026F4806646F480660E60D3F8FC71796807
:1012400021F4E0607860D3F820523A696C1CC3F84E
:1012500020422A70B3F826C20CF1FF36B7B2A3F8C9
:10126000267293F8391293F83A0201F00302104300
:101270002025C3F82C0283F83952002593F83A222E
:1012800083F83A5268E693F83942B3F8240293F8A7
:101290003A72D3F82862E2B2F9B2002840F08C80AA
:1012A000212A00F0368140297FF456AE222A7FF4AD
:1012B00053AEB3F82652ACB2002C00F0238193F861
:1012C0003A02402800F0B481D3F82042D3F8FC71F0
:1012D000601CC3F8200222783A61B3F826C20CF1F0
:1012E000FF36B1B2A3F8261236E693F83962D3F886
:1012F0004072212E16BF47F0010707F0FE07FFB22C
:10130000176131E6D3F84C0210B9402E00F01E816F
:10131000D3F84C622EB9D3F80C02B0F5404F00F070
:101320002F81B3F82662B0B2002840F0A880069062
:1013300056690696976906970698106840F40076F5
:1013400016600022C3F84C220EE6AC49C3F82812FE
:101350002026C3F82C0283F8396283F83A02FBE5B1
:10136000D3F84C0298B9D3F8406206F0FE07176133
:10137000FAE5D3F84C62012E7FF4F6ADD3F8407253
:10138000F81100F0060646F0F1071761ECE5D3F816
:10139000406246F00107F8B21061E5E5042C0FD079
:1013A000082C0DD014F5803F0AD0D3F82052D3F882
:1013B000FC116E1C0C6946E6212A7FF474AF78E7B5
:1013C0000E6826F480670F60EFE7042C71D0082CBC
:1013D0006FD014F5803F6CD00F68022C14BF27F437
:1013E000806747F480670F6093F839C293F83A0238
:1013F0000CF003010843C3F82C02D3F82022D3F8E1
:10140000FC51541C2E69C3F820421670B3F82672A2
:10141000D3F82012D3F8FC0107F1FF3C1FFA8CF23D
:10142000A3F8262205694C1CC3F820420D70B3F8BE
:101430002662D3F8FC71711E88B2A3F826027A687E
:1014400022F4407420257C6015E7042D39D0082D46
:1014500037D015F5803F34D0726822F4E0617160B6
:1014600093F8396293F83A5206F0030005432024BA
:10147000C3F82C5283F83A7283F839426CE5B3F81A
:101480002662B0B2012800F08B80B3F82672BEB29B
:10149000022E00F0B580106840F480671760D3F822
:1014A000FC610022029270690290B7690297029A69
:1014B00047E71225C3F82C520C6844F400760E60FE
:1014C0009BE7726822F4E0657560306800214FF098
:1014D000200C40F400743460C3F82C1283F839C235
:1014E00093F83A2283F83A1236E5022C0C6800F0A1
:1014F000B38024F480670F60D3F8FC11086840F4CF
:1015000000620A60D3F8FC516B6823F48061696063
:1015100022E5042ED3F8FC711FD0082E1DD016F53D
:10152000803F1AD07C6824F4E0627A6093F83972C4
:1015300093F83A6207F003052E434FF0200CC3F8EE
:101540002C6283F83A0283F839C205E508905069A5
:10155000089096690896089A06E57C6824F4E0628B
:101560007A603E680020202546F400713960C3F897
:101570002C0283F8395293F83A2283F83A02EBE4CA
:10158000079657690797906907900798166846F479
:1015900080771760D3F84C220132C3F84C22E3E481
:1015A000042F18D0082F16D0BEF1120F13D0D3F885
:1015B00028721068022F14BF20F4806040F480600D
:1015C0001060D3F8FC610022059277690597B06935
:1015D0000590059AB5E6166826F480601060D3F889
:1015E000FC71002204927E690496B8690490049804
:1015F0003A6842F400763E60A3E600BF0000FFFFB9
:10160000D3F828621068022E2AD020F48066166073
:10161000D3F8FC01026842F400670760D3F8FC21AC
:10162000002603965069039097690397039A88E60A
:10163000D3F84C72C7B9D3F84852D3F8FC11D3F899
:101640004442012D23D0C4F307270F61D3F84C0285
:101650000130C3F84C027FE444F480660E6051E729
:1016600040F480671760D9E7D3F84C22012A16D0DE
:10167000D3F84C62022E7FF46FAC93F83912222912
:1016800019D093F83952212D7FF466AC1CE6E2B2F2
:101690000A61D3F84C620236C3F84C625CE4D3F8BA
:1016A0004472D3F8FC01FAB20261D3F84C620136FD
:1016B000C3F84C6250E4D3F8FC512B6843F48074B7
:1016C0002C6049E470B58F4C8F48D4F8FC315A69CE
:1016D000596802423ED0CE0502F481354ED5D4F889
:1016E0003C6246F001006FF48076C4F83C025E6113
:1016F000002D00F09A80D4F83C526FF4007645F04B
:10170000020012F4823FC4F83C025E6128D094F8D3
:101710003A52B4F826C294F83902D4F82C62202D3B
:101720001FFA8CF1C0B200F08580D4F83C1241F071
:101730000406C4F83C621D6845F400711960D4F8D1
:10174000FC316FF48060586112F4843F16D0D4F8F5
:10175000FC310AE012F4813F58D112F4823F59D192
:1017600012F4843F0AD0C90508D5D4F83C226FF49E
:10177000006642F00805C4F83C525E61D4F83C02B1
:1017800000B970BD94F839C2ACF12901012945D9DD
:1017900094F83932602B4FF000021CBF202384F8EC
:1017A0003932C4F82C2284F83A22D4F8FC010168BA
:1017B00021F400630360D4F8FC613268120555D54A
:1017C000706820F400617160D4F83002002855D0B0
:1017D00090F835304D4E0665022B54D0802343657A
:1017E000FEF790FF94F83962282ECAD1D4F83C2233
:1017F0005307C6D500254648C4F828022021C4F85E
:101800002C5284F8391284F83A5270BDCD053FF558
:1018100072AFB3E7C8053FF57AAFAFE700262825DA
:10182000C4F82C6284F83952BFE712F4823F7FF487
:101830006EAF95E700297FF478AF00F0F705212D12
:1018400005D028287FF471AF212E7FF46EAF94F875
:101850003962D4F828020428F5B21DD008281BD01C
:10186000212D32D06FF4806159616DE794F83952BF
:10187000602D04BF202584F83952B3E7D4F8340230
:101880000028A5D1AEE70268052580F8355010681C
:1018900020F001011160A5E7282DE1D11C4DC4F80D
:1018A000285259686FF4806021F4E0665E605861E8
:1018B0001D6825F48061196000202023C4F82C02E3
:1018C00084F8393284F83A023EE7114EC4F82862AF
:1018D00094F839C294F83A520CF0030005432021E1
:1018E0000026C4F82C5284F8391284F83A625D68F4
:1018F0006FF4806025F4E061596058611E6806400D
:101900001E6021E7400001200001010005070008DA
:101910000000FFFF024BD3F83402FEF7BBBC00BF50
:1019200040000120024BD3F83002FEF7B3BC00BFE9
:1019300040000120034AD2F850320133C2F850323D
:10194000704700BF4000012038B5104A92F8543269
:10195000112B00D938BD0E480E4D41690133DCB260
:1019600081F4807C4CF08073836115F8141082F848
:101970005442002002F03AF805EB4402012051786D
:1019800002F034F80448047338BD00BF4000012061
:1019900000080240C0A300080000002038B5104A2B
:1019A00092F8543203B938BD0E4841695C1EE4B266
:1019B00081F4007545F00073122C82F85442836163
:1019C000F1D8094D002015F8141002F00FF805EBBE
:1019D00044020120517802F009F80448047338BD2C
:1019E0004000012000080240C0A3000800000020C1
:1019F00008B5234B2349D3F850224FF080600132C1
:101A0000C3F850228861D3F85812D3F85C2291426F
:101A100024D0D3F85802D3F85C1288421BD0D3F8F4
:101A20005C22D0B2043003EB400EBEF858C2D3F8AB
:101A30005C1201311FFA8CFCC3F85C121248A3F847
:101A400060C4FEF7CFFF114A536983F0200040F4D1
:101A50000011916108BD4FF6FF7CEFE793F8623407
:101A600053B90B48FEF7BEFF0848416981F04002B8
:101A700042F48003836108BD0648FEF7B3FFF3E735
:101A80004000012000040240A004012000080240A0
:101A9000E8A30008E6A3000838B5234C94F86324B3
:101AA000D4F85032054652B1D4F8640438B1D4F8B1
:101AB00068145A1A142A2FD90023C4F86434D4F8AD
:101AC0006C04D4F87014D4F8742401309142C4F832
:101AD0006C0423D0D4F87434D9B2043104EB41023D
:101AE000B2F87004D4F8743401331FFA80FCC4F8DF
:101AF000743400B2D4F878260C49288001320C4D99
:101B00000869C4F87826C2F30E0405EB4403A0F874
:101B100000C00B61012038BD8047CDE74FF0FF309A
:101B20004FF6FF7CE6E700BF4000012000000020E8
:101B3000400000200120704701207047024B93F8BD
:101B40007F160170012070474000012000EB010C5E
:101B500002464BF6AD21002012F8013B80EA032338
:101B600018B20028ABBF5B0081EA40009BB283B291
:101B700018B20028ABBF5B0081EA40009BB283B281
:101B800018B20028ABBF5B0081EA40009BB283B271
:101B900018B20028ABBF5B0081EA40009BB283B261
:101BA00018B20028ABBF5B0081EA40009BB283B251
:101BB00018B20028ABBF5B0081EA40009BB283B241
:101BC00018B20028ABBF5B0081EA40009BB283B231
:101BD00018B20028ABBF5B0081EA400098B280B227
:101BE0009445B9D1704700BF70B4194D040C012C55
:101BF000D5F8FC6104D113E02C68E41AA2421BD38F
:101C0000B46920EA0404A4B2B4FA84F464098C42EE
:101C1000F2D0002070BC70472C68E41AA2420BD3AB
:101C2000746920EA040C1FFA8CF4B4FA84F4640991
:101C30008C42F1D00020EDE700232022C5F82C32A1
:101C400085F8383285F83922032070BC704700BF10
:101C50004000012010B41849D1F8FC41636913F029
:101C6000800326D1626912F4806211D10B681B1ABD
:101C7000012BF3D9D1F83C0281F8382220242043EB
:101C8000C1F83C02C1F82C22032081F839420DE052
:101C90006FF48062626104202024C1F83C0281F864
:101CA0003832C1F82C32012081F839425DF8044BFA
:101CB00070470020FAE700BF40000120024BB3F854
:101CC0004C10018002207047400001200120704725
:101CD0000020704708B5024B024A1A60FEF790FADE
:101CE00000C00120AD700DB00020704708B5FEF7B0
:101CF00087FA00BF024B012083F88006704700BFBF
:101D00004000012000207047024B93F881160170BB
:101D100001207047400001204379012B01D00120B0
:101D2000704780790228FAD8084A012882F881068B
:101D3000F5D192F8821621B105494FF400628A610B
:101D4000EDE7034B4FF000609861E8E740000120A9
:101D500000080240084B5969642202FB01F111F5A9
:101D6000001304D503F57F1C0CF57F533F339A1500
:101D700002700120704700BF000000204379012B52
:101D800001D0012070478079421E632AF9D8054AA4
:101D9000054983053233A2FB032042094A61012031
:101DA000704700BF1F85EB5100000020024B197ED9
:101DB00001700120704700BF000000204379012B13
:101DC00001D0012070478079421E072A9CBF024A39
:101DD00010760120704700BF00000020064B4FF036
:101DE000000C197F5B7F80F800C001224170827077
:101DF000C3700420704700BF00000020084B997F8B
:101E0000DB7F002261F3070263F30F2289080133AD
:101E100061F317429B1063F31F6202600420704756
:101E2000000000204379022B01D00120704710B43C
:101E300083799A08911E06290BD80F4CE17F013156
:101E400003F0FC03B2EB910FA377BCBF03F1FF33A8
:101E5000E377C07901308408A21E062A07D8064815
:101E6000837FB4EB930F02D8A1004C1EC4770120EE
:101E70005DF8044B704700BF00000020024B93F850
:101E800063140170012070474000012000B50B4B26
:101E900093F8201093F821C093F82820417093F80C
:101EA000293080F802C04FF0000E012180F800E0D8
:101EB000C1700271437106205DF804FB0000002030
:101EC000034B0B2193F88326027041700220704768
:101ED000400001204379012B01D001207047807917
:101EE0000A289CBF024A82F883060120704700BF7F
:101EF0004000012010B5134BB3F830C004464FEA40
:101F00004C10B0EB0C0162EB02025302480210EBE2
:101F10000C0043EAD15141F100029301810143EAEF
:101F2000906E081A6EEB020E10EB0C00064A4FF092
:101F300000034EF1000104F093FF024622800220CC
:101F400010BD00BF00000020400D03004379022BAC
:101F500001D001207047C0880649074A01FB00F004
:101F60009042F6D8054B0649A3FB0020820C0A8656
:101F700001207047400D03003F62B00783DE1B4322
:101F8000000000204379012B01D0012070478079A7
:101F900005289CBF024A82F884060120704700BFD2
:101FA00040000120054B06495B6B064A591A8B100D
:101FB00002FB03F303700120704700BF0000002004
:101FC000ECA30008ABAAAAAA01207047034B132177
:101FD0001A7B027041700220704700BF0000002091
:101FE0001B4B93F88526032A30D810B519491A4C93
:101FF0000A69B0F807E090F806C083F885C6141B9C
:102000006210002183F88616C3F88816C3F8782674
:10201000B0F80910A3F88C161EF4004F1FFA8EF0CA
:102020001CBF4FF4004E70468CB208BF86468442F7
:1020300088BFA3F88C06BCF1010FA3F88EE604BF9D
:1020400083F886C6C3F88826012010BD002070479B
:1020500040000120000000204000002000207047C8
:102060004379012B01D001207047827922B10549C3
:10207000012081F890367047024880F890260120B0
:10208000704700BF40000120044B93F890160246B1
:102090000B1E18BF01230120137070474000012060
:1020A000074B084AD3F894364FF47A7101FB03F3D7
:1020B0009909A2FB01239A0902600420704700BF1E
:1020C00040000120632D3E054379042B01D00120FF
:1020D0007047D0F806000649064A01FB00F0A2FB53
:1020E000002305499809C1F894060120704700BFF4
:1020F000400D0300D34D62104000012000207047C6
:102100000020704700207047002070470120704772
:1021100001207047114BB3F898260280B3F89A1645
:102120004180B3F89C268280B3F89E16C180B3F834
:10213000A0260281B3F8A2164181B3F8A4268281B9
:10214000B3F8A616C181B3F8A8260282B3F8AA167E
:102150004182B3F8AC3683821620704740000120DC
:1021600001207047002070470120704730B5334B85
:10217000DC7F002C59D014F00701314A4FF00003E6
:102180002BD0012922D002291BD0032914D00429E5
:102190000DD0052906D006294BD132F802CB20F804
:1021A00013C0013332F8021B20F81310013332F848
:1021B000025B20F81350013332F802CB20F813C031
:1021C000013332F8021B20F81310013332F8025B9E
:1021D00020F813500133A34227D0114603F1010C1C
:1021E00031F802EB20F813E0558820F81C5003F179
:1021F000020E498820F81E10DD1CD18820F8151029
:102200001D1D118920F815105D1D518920F815102C
:102210009D1D918920F81510DD1D0833D18920F806
:102220001510A34202F11002D7D1600000F0FE00A9
:1022300030BD32F8025B05800123AEE700000020CC
:10224000F00601200020704701207047184BDA7F0C
:10225000997F01328B1A48BF03339A10013212F072
:10226000FF0321D0134A012BB2F8F01601801BD0D6
:10227000B2F8F2164180022B16D0B2F8F416818023
:10228000032B11D0B2F8F616C180042B0CD0B2F893
:10229000F8160181052B07D0B2F8FA164181062BFA
:1022A0001CBFB2F8FC268281580000F0FE00704787
:1022B0000000002040000120002070472DE9F84375
:1022C00081FB0141A50B5B0045EA8146B6FBF2F7B5
:1022D000C11B4FEAE07060F10008A1FB030403FB9F
:1022E0000841002304F06CFD002976DBB0F1004FBB
:1022F00071F1000474DB0B4606460121B50845EA7E
:102300008376B6F1004F4FEAA3034FEA410773F11A
:102310000000F9B2F2DA9803002440EA9645B203CD
:1023200000234FF0804E9E0846EA8E739A424FEA91
:10233000AE0E75EB0E00F6DB53EA0E004DD04FF0FB
:102340000008464613EB080046EB0E0C824275EB84
:102350000C094FEA93070BDBB2EB000965EB0C05A8
:10236000DB184EEB0E0213EB080846EB02064A465A
:102370004FEA580047EA8E734FEAAE0E40EAC6783D
:1023800053EA0E004FEA6606DCD14FEAE87708FB15
:1023900004F4A8FB012C01FB07469518664446EBA4
:1023A0000601AB1846EB010778015D0140EAD364F2
:1023B0005B1947EB04019A1846EB0106002E0CDB73
:1023C00012F5005746F10009B80B40EA8944FF2C8A
:1023D00028BFFF24E0B2BDE8F8830020BDE8F88301
:1023E0008A0342EA904501218203002498E700BF56
:1023F0002DE9F0410026154C82B080464FF400755F
:102400003746D4F87024D4F874349A420DF106009B
:10241000F7D0FFF741FB0028F3D0BDF90600013DDE
:1024200000FB00F1ADB207EBA1370644002DE8D167
:10243000314601234FF400723846FFF73FFF06464E
:10244000012088F8006002B0BDE8F0814000012062
:1024500030B5374D034605F110020020698803EAC4
:10246000010414F00F0E05F1020C0CD05FEA5E05BA
:1024700055D05FEA9E048EEA050102D0614081EAF0
:10248000DE0101F0010EBCF80250400081B21D4097
:1024900041EA0E0015F00F010AD04C0841D08D081A
:1024A00081EA040402D06C4084EAD10404F0010102
:1024B000BCF8045044001D40A0B215F00F0E40EAD5
:1024C00001000CD05FEA5E012DD05FEA9E048EEA27
:1024D000010502D0654085EADE0505F0010EBCF875
:1024E000061044001940A5B211F00F0145EA0E0094
:1024F0000CF106050CD04C0817D05FEA910C81EA6C
:10250000040E03D08CEA0E0484EAD10E0EF0010111
:102510004400A0B2954240EA01009FD130BD0121A4
:10252000AFE70124C2E70125D7E74FF0010EEDE741
:1025300002A40008224910B5864601F120040020BB
:1025400031F8023F0EEA0302C2F30A037BB35A08D2
:1025500034D05FEA930C82EA030226D08CEA0202AE
:102560005FEAD30C21D082EA0C025FEA131C1CD074
:1025700082EA0C025FEA531C17D082EA0C025FEA7F
:10258000931C12D082EA0C025FEAD31C0DD082EABF
:102590000C025FEA132C08D082EA0C025FEA532C8B
:1025A00003D082EA932383EA0C0202F00103400085
:1025B00082B2A14242EA0300C2D110BD0122F4E777
:1025C00012A4000870B5334C0D4604F1080E1146F4
:1025D00000223EF8023D0340520013F0FF0392B286
:1025E0001CD05E0824D083EA060C9E0813D08CEA27
:1025F000060CDE080FD08CEA060C1E090BD08CEA04
:10260000060C5E0907D08CEA060C9E0903D08CEA02
:10261000D31383EA060C0CF001063243A645D8D149
:102620000AB3072A07D84FF6FF700880002070BD54
:102630004FF0010CEFE7A2F1080414F0FF0221D1E2
:10264000C0F34014C0F3C00242EA4406C0F3800362
:1026500043EA4604C0F3400040EA440601220A80EF
:102660002E80012070BDC0F3401CC0F3C003C0F336
:10267000800443EA4C0644EA4606C0F3400040EAC0
:102680004606ECE7C2F108060123B340434098B286
:10269000D6E700BF34A400082DE9F041DFF898C167
:1026A00005460F4616469CE8070084B001AB9846E5
:1026B00003C30DF10E0E00241A803EF8020D6400D3
:1026C00015EA0001A4B240D04A084BD0880881EA3C
:1026D000020337D05FEAD10C83EA000332D00A0943
:1026E00083EA0C032ED0480983EA02032AD05FEA6A
:1026F000911C83EA000325D0CA0983EA0C0321D088
:10270000080A83EA02031DD05FEA512C83EA000322
:1027100018D08A0A83EA0C0314D0C80A83EA020399
:1027200010D05FEA113C83EA00030BD04A0B83EA26
:102730000C0307D0880B83EA020303D083EAD1316C
:1027400081EA000303F001031C43F045B5D1002CDE
:1027500040D00F2C08D84FF6FF750020358004B00C
:10276000BDE8F0810123EDE7A4F1100818F0FF04A3
:102770005BD1C5F34031C5F3C02343EA4104C5F33F
:10278000802242EA4400C5F3402141EA4004C5F3F7
:10279000C01C4CEA4408C5F3801343EA4802C5F361
:1027A000401040EA4201C5F3001444EA410CC5F36D
:1027B000C008C5F3800248EA4C0342EA4300C5F36F
:1027C000400545EA4001012401203480398004B0ED
:1027D000BDE8F081C5F3403CC5F3C02343EA4C0893
:1027E000C5F3802242EA4800C5F3402141EA400C8B
:1027F000C5F3C01343EA4C00C5F3801848EA400211
:10280000C5F3401141EA420CC5F3001343EA4C0002
:10281000C5F3C00242EA4001C5F3800343EA410028
:10282000C5F3400545EA4001CEE7C4F1100201209E
:102830009040684085B29CE73CA400081C491D4AB2
:102840004B6992F805C783F0400343F480038B6122
:1028500092F804178C4502D092F8303703B97047CC
:1028600092F806C7D2F8001741F82C0092F8061724
:1028700092F8040701315FFA81FC92F8051782F89B
:1028800006C760458CBF0131013103F1FF3398BFAA
:1028900000205FFA81FCD9B298BF82F8060702EBEC
:1028A000810082F805C7D0F8080782F83017704712
:1028B000000002404000012010B4194CD4F8FC1173
:1028C00007E04A6912F0100C0BD123681A1A012A8A
:1028D00018D84B6913F04003F3D000205DF8044B87
:1028E00070476FF010004FF0200C4861C4F83C3284
:1028F00084F83832C4F82C3284F839C201205DF8EB
:10290000044B7047D4F83C0284F838C220210843B5
:10291000C4F83C0284F8391203205DF8044B704778
:102920004000012070B41B4ED6F8FC5107E06C69E2
:1029300014F4806316D13468A41AA14208D36B69D9
:1029400020EA0304A3B2002BF1D1184670BC7047F3
:102950002022C6F82C3286F8383286F83922032035
:1029600070BC7047286840F400712960D6F8FC51AB
:1029700000246FF48063042220216B61C6F83C229E
:1029800086F83842C6F82C4286F83912012070BC0D
:10299000704700BF40000120F8B5254CD4F828321C
:1029A000042B16460746D4F8FC210D4608D0012B0F
:1029B00006D013F5803F03D0D4F82C02122803D19F
:1029C000116841F480731360D4F8FC2103E020689F
:1029D000811B8D4214D35069C307F8D5D4F80C126B
:1029E000B1F5804F17D11761124832462946FFF7DB
:1029F00099FF20B1D4F83C42042C0AD10120F8BD43
:102A000000234FF0200CC4F82C3284F8383284F8BC
:102A100039C20320F8BDF023136107483246294626
:102A2000FFF780FF0028E5D1D4F8FC211761DBE730
:102A300040000120020001000800010010B51E4CFA
:102A4000D4F83407C36823F00101C160036A41F27E
:102A5000111213420AD1026A40F244410A4205D1DE
:102A6000036823F001020260D4F8340713491123EC
:102A7000C4F84037FDF75CFED4F83427D4F83C079F
:102A8000136823F070030343D4F8440723F440731E
:102A900003431360D4F83437D4F84007D4F83847E8
:102AA000D86201219C625961DA680A43DA601868C9
:102AB0000843186010BD00BF4000012078070120C6
:102AC00030B4464902680C680025022380F835308E
:102AD00080F83450156825F001031360026803E0A4
:102AE0000B681D1B052D4FD81568ED07F8D4D0E9EC
:102AF0000134C1682343D0E904540B432B432343DF
:102B0000D0E906412343046A15680B432343344943
:102B1000446A2940042C43EA010303D1D0E90B5451
:102B200025432B4313600168426A4B69042A23F052
:102B3000070545EA020508D1826A8469154354BB3A
:102B4000012A45D0022A2DD062B34D610368254C7D
:102B500025495FFA83FCACF11002A4FB025401EB9F
:102B600014156FF3090395F88810C1655F2A88BFB3
:102B700004333F228A400024012583659A6044651E
:102B800080F8355030BC704720210322416580F821
:102B9000352030BC7047B4F5005F0CD0022A04D950
:102BA000032AD2D1C26AD201CFD540210125416585
:102BB00080F83550EDE7032AC7D801A454F822F075
:102BC000AB2B0008A52B0008AB2B0008D12B00086D
:102BD000C36AB3F1C07FB8D1E7E700BF400001206E
:102BE0003F8010F0ABAAAAAAC0A3000830B4174BCC
:102BF000D3F85822D3F85C12501AB0F5807F10D168
:102C0000134D14498024AC610A6922F00400086164
:102C100030BFD3F85822D3F85C02121AB2F5807F85
:102C2000F1D0D3F85852E9B2043103EB410C4FF420
:102C30000044ACF85842D3F85822054D4FF4000038
:102C40000132C3F85822A86130BC7047400001200F
:102C50000008024000ED00E0B0F5804F70B438DAB3
:102C600010F5804F32DB00F5804290B241001FFA30
:102C700081FC194AD2F85832D2F85C421D1BB5F5D6
:102C8000807F10D1154E16488021B161036923F071
:102C90000404046130BFD2F85852D2F85C32EC1A06
:102CA000B4F5807FF1D0D2F858620C48F1B204310B
:102CB00002EB41054FF40004A5F858C2D2F858328F
:102CC0000133C2F85832846170BC70474FF0000C79
:102CD000CFE74FF6FF7CCCE7400001200008024020
:102CE00000ED00E0094B4FF4E052986892FAA2F32D
:102CF0000749B3FA83F200F4E053D3400B4405488C
:102D000093F890100068C840704700BF0038024038
:102D1000C0A3000800000020094B4FF460429868EF
:102D200092FAA2F30749B3FA83F200F46043D34066
:102D30000B44054893F890100068C840704700BFE6
:102D400000380240C0A3000800000020884A136831
:102D500003F00F0C8C4507D2CBB21370126802F04F
:102D60000F0C614500D0704730B40468A50707D543
:102D7000804D8468AB6823F0F0022243AA600468A7
:102D8000E40727D54468012C00F0EB80794BA51EA1
:102D9000012D1A6840F2E180950728D5754A95689B
:102DA00025F00303234393604368734C012B25688C
:102DB00041F2883C00F0B380022B00F0BB80032B73
:102DC00004D1C2E023685B1B634510D8936813F0FD
:102DD0000C0FF7D1664A146804F00F05A94208D217
:102DE000CBB21370126802F00F04A14201D030BCC4
:102DF00070470468620707D55E4DC168AB6823F46D
:102E0000E0520A43AA600468230753D4594A9468DD
:102E100004F00C05082D5BD00C2D40F09C8055680B
:102E20005368536805F03F0447F6C07090FAA0FC61
:102E30005249B1FBF4F5BCFA8CF24E4C0340D3403E
:102E400005FB03F34FF0E040626890FAA0FCBCFA87
:102E50008CF102F0E045CD40B3FBF5F34548F0249A
:102E6000826894FAA4F54649B5FA85F02240C2403A
:102E70001144444A91F890504349EB40A2FB0302AD
:102E80009009451EB5F1807F0B600CD24FF0E02C0D
:102E90003E4BCCF81450002183F823400724CCF893
:102EA0001810CCF8104030BC00220F214FF0FF303A
:102EB000FDF7B8B92F4D0069A9682E4A21F4604C7E
:102EC0004CEAC003AB60946804F00C05082DA3D154
:102ED00050685368536800F03F0147F6C07494FA95
:102EE000A4FCBCFA8CF22340224C244DB5FBF1F03B
:102EF000D34000FB03F362684FF4403191FAA1F52F
:102F0000B5FA85F002F44034C44001346100B3FBEB
:102F1000F1F3A3E723685B1B63453FF668AF936853
:102F200003F00C03042BF5D154E723685B1B6345C6
:102F30003FF65DAF936803F00C03082BF5D149E72A
:102F400023685B1B63453FF652AF936803F00C03A5
:102F50000C2BF5D13EE7094B80E793013FF51EAFFF
:102F600045E7044D2B689A033FF518AF3FE700BFD4
:102F7000003C024000380240400001200024F400E0
:102F8000C0A30008D34D62100000002000ED00E057
:102F900070B58A4A936803F00C01042982B000F0EE
:102FA000A980946804F00C05082D00F09F80834AE6
:102FB000936803F00C010C2900F0AE807F4A804931
:102FC0000125957046680C68002E72D013689E0328
:102FD00006D40D682E1B642E65D813689E03F8D5A1
:102FE0000268910730D5754CA26812F00C0F67D0BB
:102FF000A36803F00C05082D5FD070498C6804F0BD
:103000000C020C2A00F0D180C568002D00F0BE80B3
:103010006C4B6B4901221A600C68684A03E00E6829
:10302000331B022B3FD81568AD07F8D514684FF055
:10303000F80C9CFAACF10669B1FA81F39E4024F0D9
:10304000F8052E4316600268160712D54469002C55
:1030500053D05C4B5A4A0121C3F8801E146857496B
:1030600003E013681D1B022D1DD84E6FB507F8D560
:103070000268560755D48569ADB1504A916801F090
:103080000C04082C0FD0022D4E4B4D4900F09280BD
:10309000002018660D6803E00C68631B022B02D841
:1030A0001668B301F8D402B070BD0D682E1B642EF3
:1030B000F9D813689D03F8D492E7666872029CD42D
:1030C0003E4D29688E0702D5C268012AEBD13B4CE0
:1030D000F826256896FAA6F10369B1FA81F29340C1
:1030E00025F0F806334323600268ADE756687202A4
:1030F0007FF55DAF31490B6872E7324D304AC5F854
:10310000804E16682D4903E01468A51B022DCAD80D
:103110004B6F9B07F8D4ABE7546863027FF54EAF63
:10312000E8E7264C284900250195236C43F080569A
:103130002664226C02F080540194019B0D68204AA1
:1031400045F480730B60146803E015682E1B022E93
:10315000A9D80E68F505F8D51849047A81F87040A9
:103160008368156841F2883C3BB10E6FB30782D487
:103170001668731B6345F8D995E70E6FB6077FF5A0
:103180007AAF1468631B6345F7D98CE70D4E0C4A80
:1031900035601468094903E015682E1B022E82D899
:1031A0000B689B07F8D402684EE74B685B023FF55B
:1031B0002BAF85E700261E660E680CE00038024043
:1031C0004000012000004742007000400B689C1B3B
:1031D000022C3FF668AF1568AD01F7D447F6C0740E
:1031E00094FAA4F34FF4403CB3FA83FE9CFAACF695
:1031F0004FF07065B6FA86F695FAA5F44FF0E04305
:10320000B4FA84FC93FAA3F5846A63085C1EB440A4
:10321000D0E907363343466A06FA0EF633432343B2
:10322000C46A006BB5FA85F504FA0CF6A84033437E
:103230000343084D536001222A660E68064804E0E5
:103240000C68A51B022D3FF62EAF03689C01F7D535
:1032500029E700BF00004742003802402DE9F0474F
:10326000A14CA24B94F83912A14E00224FF4804099
:10327000FE255E278AB0C4E98425C4E98622C4F805
:10328000FC31C4F80402C4F80C02C4F80062C4F8AB
:103290000872002974D0242184F839121F68954ED1
:1032A00027F001001860B5684FF4E05C9CFAACFAB6
:1032B0009149924FBAFA8AF205F4E053D3400B4495
:1032C000386893F890608E4DD4F8FC11F040A5FB5F
:1032D00000239F0C4F60D4F800228A4EB2422AD8B5
:1032E00040F6FC7901375500B0FBF5F616EA090FF8
:1032F0000F6208BF0426CE61D4E9867007430F60D1
:10330000D4E98212D4F8FC310A439A60D4E9846586
:103310002E43DE601868002740F00101202219606A
:10332000C4F83C7284F83922C4F82C7284F83A72DA
:103330000AB0BDE8F087744D4FF4967303FB07F7AE
:10334000A5FB0757BE09D4F8045201360E6255B9E1
:1033500002EB420AB0FBFAF2C2F30B03002B40F07F
:10336000BF800126C7E702EB820909EB8908B0FBA1
:10337000F8FCCCF30B000028F3D04CF44046BAE73D
:1033800001F0FF0503F5F23303951A6B84F8385208
:1033900042F002011963186B00F002060396039ACB
:1033A00002951F6B47F002021A63196B01F00200CD
:1033B0000290029A01951E6C46F400171F641A6C65
:1033C00002F400110191019A0095186B40F4001667
:1033D0001E631B6B40201221CDE90401002003F481
:1033E0000017012100F18048CDE90601009708F59A
:1033F000013004A90426009A0896FDF735F88022CA
:103400000492FDF731F84FF4000704F5EE60402315
:103410003E4983604FF400164FF0007A4FF4806904
:103420004FF00308C0E90555C0E90755C0E90A8710
:103430000663C5604562C0F81090C0F804A0C4F8E7
:103440007017FFF73DFBC4F8300204F5FA6030490D
:10345000C4F8FC774FF4003204F5FE77C4F8EC575B
:10346000C4F8F457C4F8D8570262C4F8DC57C4F85B
:10347000E457C4F8E857C4F80068C4F8D017254EDC
:10348000C4F8D4A7C4F8E097C4F8F887C4F8A877BC
:10349000FFF716FB0122C4F8340202212F20C4F8E2
:1034A0000878FCF7BFFE4FF400402A467060022106
:1034B0000B204FF40065FCF7B5FE0122022120200D
:1034C0003560FCF7AFFE01230222736011461F2016
:1034D000FCF7A8FE4FF00042D4F8FC313260DAE687
:1034E00042F4004607E700BF4000012000540040BE
:1034F000801A060000380240C0A300080000002027
:1035000083DE1B43A0860100D34D6210B8600240E9
:103510001060024000E100E010B46449644A4B6965
:1035200083F0800040F4000483B08C61D2F8501224
:103530000131C2F85012B2F8A83098B2C4001FFA94
:1035400084FCACF580410BB2002B88B292F83018A5
:10355000D2F85042BCBFCCF5804C0FFA8CF302EB92
:10356000410C013101F03F0182F83018BCF93418E8
:10357000ACF834385B1AD2F8B4180B44D2F8B81847
:10358000C2F8B4388B4254DAB2F8BE3803F1FF3CCB
:1035900021211FFA8CF3A2F8BC18A2F8BE38002B28
:1035A0006BD0D2F87044D2F87434E11AB1F5807F50
:1035B00031D13E48446984F4806C4CF0806383616F
:1035C0003C4B3D4C4FF0007199613C4B1168C2F887
:1035D0008040116D1068C2F8883003E013681C1A2F
:1035E000642C54D88C68A307F8D54AF6AA22002088
:1035F000CA600190CB6801938C680194019B4A6872
:1036000042F0400048600B6843F040040C6003B097
:103610005DF8044B7047D2F87014CCB2043402EB5E
:10362000440CACF87004D2F870040130C2F8700495
:10363000C6E7D2F8C0188B4217DDB2F8BC3803F1E8
:10364000FF3C40F201211FFA8CF3A2F8BE18A2F849
:10365000BC38002BA5D11A49C2F868444FF0210CA0
:10366000C2F86414A2F8BCC89BE7212440F2012CE4
:10367000A2F8BC48A2F8BEC893E71249C2F8684451
:1036800040F2012CC2F86414A2F8BEC889E70E4BC0
:1036900008249C614FF40062402080214FF4805444
:1036A0009A61986199619C61FEE700BF0008024041
:1036B000400001200004024060A40008E80001204E
:1036C0009D19000849190008000002402DE9F04347
:1036D000654C94F83932202B83B003D0002003B01E
:1036E000BDE8F08300220092226894F839620D78D8
:1036F000497884F8C4580227202E84F8C51884F825
:10370000C479EBD1594B5A4E1D68E908A6FB011745
:103710003B0A03EB830808EB8806D4F8FC510096BB
:1037200003E0AB6913F002030CD0009F791E0091F7
:10373000002FF6D12026C4F82C7284F8387284F851
:103740003962CBE794F83862012EC7D04FF0010CF4
:1037500084F838C22F68474E27F400612960D4F8F6
:103760003012454FD4F8FC810B654FF021094FF022
:10377000100E84F8399284F83AE2C4F83C320225FB
:1037800091F834E0A4F82652C4F828723B4FCF6376
:10379000E6453B4FD1F858900B64C1E91133A4F8CA
:1037A0002452C4F82062CF6407D091F835E081F844
:1037B00034C0E64522D081F83430400080B2232165
:1037C000FFF7EAF8064628B10020D4F83C2284F836
:1037D000380283E7D4F8FC21019053690193916981
:1037E00001910199556845F480775760536843F417
:1037F00000615160012084F8386270E7D1F800C0A0
:1038000081F835504B65DCF8007027F48027CCF840
:1038100000700F687D608D680F68402D08F11003FF
:103820001ED0BE600E68F360CD6D3F27AF40C9F873
:1038300008700E68336843F0160535600F687E69BE
:1038400046F080037B610D6C25B10F683E6846F041
:1038500008033B6009680D6845F001070F60ACE79D
:10386000BB600B68DE60DFE7400001200000002045
:1038700089B5F814040901200000FFFF5D06000867
:10388000DD06000870B53B4B3B4C082282B09A61C4
:10389000D4F85052FFF7D2F872B6384E38487060FC
:1038A00062B672B60021C4F85812C4F85C1262B64F
:1038B000344B4FF4803202209A619861D4F8501250
:1038C000D4F850325A1AB2F5487F0BD22E48036909
:1038D00023F00402026130BFD4F850325A1AB2F514
:1038E000487FF4D394F883C628496144002091F8B6
:1038F000A4E08DF8040001A92D208DF805E0FFF764
:10390000E5FE226D116841F002001060226D012376
:1039100084F86234136843F001011160FFF78EF8F8
:1039200072B61B48706062B6D4F85062721BB2F572
:10393000166F15D205F51665AE1B11D0D4F85002DE
:10394000D4F85032191A8E420AD90F4A156925F057
:103950000403136130BFD4F850120D1AAE42F5D8EB
:10396000084C044E04204FF40022A061B26102B062
:1039700070BD00BF00080240400001200000002090
:10398000351900080000024000ED00E0C0A3000867
:10399000F1190008012804D80B4620B9012911D9D2
:1039A00070470020704710B50E4C82B0002201A96C
:1039B0002C2063778DF804208DF80530FFF786FE04
:1039C00002B010BD0748017741B901F1804C0CF5F8
:1039D00002304FF480328261012070470249012396
:1039E0008B61F9E70000002000080240012800D99F
:1039F000704738B5094D05EBC0050C4695F8211008
:103A0000A14200D838BD6A6A12F83410FFF7C2FF2D
:103A10000028F7D085F8204038BD00BF0000002006
:103A2000134B144901229A61D1F85002D1F8503257
:103A30001A1AB2F5C87F0BD20F4A136923F0040398
:103A4000136130BFD1F850321B1AB3F5C87FF4D3DD
:103A500091F8630458B910B5084C94F82010FFF79A
:103A6000C5FF94F828100120BDE81040BEE770475C
:103A7000000002404000012000ED00E000000020B6
:103A800070B54479012C01D0012070BD8579122DCB
:103A9000FAD8084E002016F81510FFF7A7FF06EB1E
:103AA000450120464978FFF7A1FF034B1D73012014
:103AB00070BD00BFC0A3000800000020F8B51C4C7A
:103AC00094F86334A3B194F8545215BB0122194EF3
:103AD00084F854221146174615460020FFF786FF4A
:103AE00006EB470101204978FFF780FF124B1D7359
:103AF000124D134EC4F8C05840F201274020002256
:103B0000A4F8BE78A4F8BC08C4F86424C4F8B86863
:103B1000F8BD112D07D91120064E84F8540207462E
:103B200001210546D9E7034E2F4616F81510D4E7B4
:103B300040000120C0A3000800000020DB1B04009F
:103B4000B9A201004F4B082270B59A6172B64E4C73
:103B50000020C4F87004C4F8740462B694F86214C7
:103B6000002968D0D4F85052D4F85002D4F850321A
:103B70001A1A632A0AD845490E6926F004030B6114
:103B800030BFD4F85022161A632EF5D93D48404B69
:103B90004FF400214FF4802281619A61D4F8506281
:103BA000D4F85002831B632B0AD838490A6922F0E3
:103BB0000400086130BFD4F850329A1B632AF5D94B
:103BC000FFF72EFF2F48324E082181614FF400335A
:103BD0004FF480220020B36184F86204B261FEF7E2
:103BE0002DFF72B62B4E2C49716062B62B4B2C48C0
:103BF0004FF080629A61FCF7F5FED4F85002411B49
:103C0000B1F5166F25D394F86354FDB9206D0368A0
:103C100043F002020260246D216821F00105256055
:103C2000FEF70CFF72B61F48706062B6154E4FF477
:103C30000023B36170BD164D4FF48026AE61FFF7CF
:103C4000EFFE94F86354134E002DDFD0FFF736FFDC
:103C5000DCE705F5166CBCEB000ED4D0D4F850525E
:103C6000D4F850325A1B9645CDD90848016921F045
:103C70000403036130BFD4F85022511B8E45F5D8A0
:103C8000C1E700BF000802404000012000ED00E055
:103C90000000024000000020351900080004024026
:103CA000E8A30008193500084379022B72D12DE9E9
:103CB000F0418479302C6FD8C579002D77D0642DF0
:103CC0006DD9424F424E4FF4804507EB8404FFF715
:103CD000D9FDD4F8FC72BC1E07F2FE37B4F90220FD
:103CE00005FB02F242F38F30FEF7B6FFB4F9040091
:103CF00005FB00F040F38F30FEF7AEFFB4F906107D
:103D000005FB01F141F38F30FEF7A6FFB4F908304F
:103D100005FB03F343F38F30FEF79EFFB4F90A204F
:103D200005FB02F242F38F30FEF796FFB4F90C0068
:103D300005FB00F040F38F30FEF78EFFB4F90E1054
:103D400005FB01F141F38F30FEF786FF34F9103F98
:103D500005FB03F343F38F30FEF77EFFA742BDD18F
:103D6000FEF744FFD6F85852D6F85C42A54208D078
:103D7000184F1020B861D6F85822D6F85C128A4243
:103D8000F8D1144E4FF48013B361FFF7DBFE01202E
:103D9000BDE8F081002070470020BDE8F0810E4AA8
:103DA0000A4F0B4EA803A2FB00214D098DE7084ED8
:103DB000064F96F88486C8EBC80CCCEBCC0EA64414
:103DC00007EB4E03B3F9B0507FE700BFC0A3000874
:103DD00040000120000802401F85EB512DE9F84FFB
:103DE0004379022B02D00020BDE8F88F0546714EC2
:103DF000DFF8CC81FFF746FDA979D6F800B000279F
:103E00003846A6F53F7900296BD1FEF725FF04243B
:103E1000BBF9020033E0FEF71FFFB4F5806F47D017
:103E2000A9793BF90400D6F800B00234002940F02B
:103E30009880FEF711FFA9793BF90400D6F800A09D
:103E400004F1020B00297CD1FEF706FFAA793AF9AA
:103E50000B00D6F800A004F1040B002A61D1FEF794
:103E6000FBFEAB793AF90B00D6F800A004F1060B83
:103E7000002B46D1FEF7F0FE3AF90B000834AB797F
:103E8000D6F800B0002BC6D098F88416C1EBC1025A
:103E9000C2EBC20ABA4409EB4A0CBCF8B0E01EFB04
:103EA00000F040F38F30FEF7D7FEB4F5806FB7D146
:103EB000EB7900243BB1FEF799FE0134E979A4B215
:103EC000B4EB412FF7DB3C4A964207F1010758D08B
:103ED00056F8043FA979B3F90000D6F800B00029DC
:103EE00093D098F88426C2EBC204C4EBC40ABA4447
:103EF00009EB4A0CBCF8B0E01EFB00F040F38F3039
:103F000083E798F88416C1EBC102C2EBC20CBC4433
:103F100009EB4C0EBEF8B03013FB00F040F38F30CD
:103F2000A8E798F884C6CCEBCC0ECEEBCE033B448E
:103F300009EB4301B1F8B02012FB00F040F38F30E1
:103F40008DE798F88426C2EBC20CCCEBCC0EBE44B5
:103F500009EB4E03B3F8B01011FB00F040F38F30C3
:103F600072E798F88426C2EBC20ACAEBCA0CBC44BA
:103F700009EB4C0EBEF8B03013FB00F040F38F306D
:103F800057E7D8F85852D8F85C62AE4208D00B4FC9
:103F90001023BB61D8F85802D8F85C128842F8D1D7
:103FA000064C4FF48012A261FFF7CCFD0120BDE862
:103FB000F88F00BFBCA600087CA7000800080240DC
:103FC000400001204379012B57D12DE9F0413249BE
:103FD0008079324A01FB00F0A2FB0024A50905F517
:103FE0008076B6F5006F4FEA562748D2FFF74AFCB5
:103FF0004FF004082A4E00272A4CB4F90200FEF7BD
:104000002BFEB4F90400FEF727FEB4F90600FEF714
:1040100023FEB4F90800FEF71FFEB4F90A00FEF70C
:104020001BFEB4F90C00FEF717FEB4F90E00FEF704
:1040300013FE34F9100FFEF70FFEB442DDD1013745
:104040004745D9D1FEF7D2FD174BD3F85802D3F824
:104050005C12814208D0154D1024AC61D3F858622F
:10406000D3F85C229642F8D1104F4FF48013BB6115
:10407000FFF768FD0120BDE8F0810020704740F2A5
:10408000D138474502D9FFF7FDFBB3E71FFA87F8A0
:10409000FFF7F8FBAEE700BF80841E00D34D62102F
:1040A0007EAB00087EA70008400001200008024007
:1040B0002DE9F04FC279ADF20C4D0346002A00F015
:1040C000DC801446197A09B9012018729D79002DF7
:1040D00000F0CB806B4A6C4E92F8841600924FF041
:1040E000000BC1EBC100C0EBC0055A46AF1806EB90
:1040F00047092244B9F9B0A092B2302AD344F5D985
:10410000624F019302A94FEAEB7A07F2FE390DF1F3
:1041100006060020C1F10208A7F5F865302C08EB6F
:10412000060C98BF23460AD805EB830E2344DEF81D
:10413000FC229BB232F90C10302B0844F4D9C3177F
:104140009A0342EA9041534680035A4602F038FEF1
:10415000B94526F8020F02D037F9020FDEE7FFF764
:1041600091FB0198047A002C61D000270DF20646DD
:1041700080460DF10605711B8B1E5A08013212F0A4
:1041800007000DF106042AD0012822D002281CD0F5
:10419000032816D0042810D005280AD0062804D0F9
:1041A000BDF9080002ACFEF757FD34F9020FFEF727
:1041B00053FD34F9020FFEF74FFD34F9020FFEF7FD
:1041C0004BFD34F9020FFEF747FD34F9020FFEF7FD
:1041D00043FD34F9020FFEF73FFDB44221D0B4F99C
:1041E0000200FEF739FDB4F90400FEF735FDB4F91D
:1041F0000600FEF731FDB4F90800FEF72DFDB4F915
:104200000A00FEF729FDB4F90C00FEF725FDB4F90C
:104210000E00FEF721FD34F9100FFEF71DFDB4422C
:10422000DDD198F808500137B9B28D42A1D8FEF718
:10423000DDFC009FD7F85862D7F85C329E4209D067
:1042400013481025BC468561DCF85842DCF85C2236
:104250009442F8D10E494FF480178F61FFF772FC3A
:1042600001200DF20C4DBDE8F08F064E009631276F
:10427000B7FBF2F84FEA883B42E701221446C271CD
:1042800020E700BF40000120C0A3000880AB000869
:10429000000802404379032B00D109E70020704752
:1042A00008B54379012B01D0012008BD82794AB1BC
:1042B00009490A4A8020886182F86334FFF7FEFBCF
:1042C000012008BD0548044B80F863244FF4000129
:1042D0009961012008BD00BF00000240400001209C
:1042E00038B54379022B01D0012038BD8179C579D9
:1042F0000129F9D8084C04EBC10494F82120AA4202
:10430000F2D9636A084613F83510FFF743FB00281B
:10431000EAD084F82050E7E7000000204379022B20
:1043200001D00120704781790129FAD8C27949B9B1
:10433000012AF6D80D480E4B0277A2B94FF480320D
:104340009A61EEE710B5094C82B04FF0000C01A95C
:104350002C2062778DF804C08DF80520FFF7B6F9A0
:10436000012002B010BD01219961DAE700000020B0
:104370000008024010B4094C84460FCCCCF8000071
:1043800020788CF81000CCF80410CCF80820CCF879
:104390000C3011205DF8044B704700BF60F9020833
:1043A0004379012B01D0012070472DE9F04180793C
:1043B0008B4C020211B2002986B084F87F06BABF86
:1043C0004BF6AD2080EA4100400285B22EB2002EAD
:1043D000BABF4BF6AD2585EA46056D00AFB23BB2DC
:1043E000002BBABF4BF6AD2787EA43077F00B8B270
:1043F00002B2002ABABF4BF6AD2080EA420040006C
:1044000081B20DB2002DBABF4BF6AD2181EA450154
:1044100049008EB237B2002FB6BF4BF6AD267600FC
:1044200086EA4706B3B218B20028B6BF4BF6AD23F2
:104430005B0083EA400399B20AB2002ABABF4BF686
:10444000AD2181EA42014900B4F87D668DB2AE42E9
:1044500010D094F83932A4F87D56FF2784F87C7682
:10446000D4F87C06CDF805004FF00008202B8DF81D
:10447000048003D0012006B0BDE8F0810DF1040CEA
:10448000DCE90001D4F8008094F83922C4F8C408AB
:104490000525202A84F8C45984F8C818EAD1D4F82C
:1044A000FC6104E02768A7EB0800192825D8B1694A
:1044B000CF4317F00203F5D094F838020128D9D081
:1044C000012184F83812326822F400653560212712
:1044D000444E84F83972102300254246A02084F807
:1044E0003A32C4F83C52C4F82862FEF755FA60B17B
:1044F000D4F83C3284F83852BCE72021C4F82C327E
:1045000084F8383284F83912B4E7D4F8FC310090DA
:1045100059690091986900900099334F05265A69AE
:1045200012F080052BD1596911F480601AD12568E9
:10453000A5EB0802012AF2D9D4F83C6220273E43B9
:10454000C4F83C62C4F82C0284F83972D4F83C52A6
:104550000022042D84F838228CD11C6844F40076A3
:104560001E6087E76FF4806004214FF0200C5861D3
:10457000C4F83C12C4F82C5284F839C2E6E7BE46AF
:10458000751E1EF8010B18615A695207A9B224D58D
:1045900019B37D781D61023EB6B20237596911F038
:1045A000040509D1596911F48060DBD12568A5EBB8
:1045B0000802012AF2D9BFE7002EB0D11F682020DF
:1045C00047F400721A6084F83902012084F83862D6
:1045D00084F83A6206B0BDE8F0810E467746DDE722
:1045E000400001200000FFFF040901202D4A2E4950
:1045F000034670B42D4D10680C68186003CD2C4E26
:10460000C3F80340C3F80A10C3F8060003CE294AD2
:104610001861596103CA2E88D961274D2749284C52
:10462000986128680D68C3F82B50264D2268C3F89E
:1046300022004FF03A0CA08883F820C03124DE819C
:1046400083F82140C3F82520A3F8290007CD1E4E8A
:104650001E4CC3F832103168C3F82E00C3F83B106B
:1046600003CCC3F836201A4A1A4DC3F83F00C3F8EA
:10467000431003CA2E88C3F84D10A3F8506093F876
:1046800050102478C3F849004FF02C0C614583F892
:104690003AC083F848C083F8474014BF51205020E7
:1046A00070BC704774F9020878F902087CF90208B6
:1046B00088F9020894F90208A0F90208ACF9020886
:1046C000A4F90208B0F90208C0F90208C8F9020802
:1046D000D4F90208DCF9020808B5094B094993F836
:1046E000842600F8012B01EB820C7E22DCF8C01B33
:1046F00005F02CFC02F084FC0130C0B208BD00BF04
:1047000040000120C0A300082DE9F04FAB4AAC499E
:10471000AC4BAD4CAD4DB1B0824602F50060CDE979
:104720000D130C92099001F5006603F500678022D5
:10473000002110A808940F950A960B9705F0B4FB7A
:10474000A34C4FF40075D4F87024D4F874148A4242
:10475000F9D00DF11E00FDF79FF90028F3D0DDE937
:1047600008C06646BDF91EB0BCF8021036F8043B1E
:104770000896DDE90A72119EB0F8029011FB0BF168
:1047800041F38F38464430F8041B11967E88099017
:1047900011FB0BF037F8041B0A9719FB0BFC159F54
:1047A00016FB0BF949F38F3640F38F3811FB0BF0F2
:1047B000518813FB0BF3374443F38F3E15974CF3AB
:1047C0008F3311FB0BF740F38F3C109932F8040B39
:1047D0000B92714410FB0BF2DDE913E042F38F39C9
:1047E0009E44DDE9163247F38F36129F1091B8448C
:1047F00084444B443244CDE9128ECDF850C0CDE90B
:104800001632DDE90C86B8F8027038F8043BCDF8B2
:10481000308013FB0BF917FB0BF7209BDDE90E0132
:1048200049F38F3247F38F3C219FB0F802901A442E
:1048300073882092BC4436F8047B0D9613FB0BF36F
:1048400043F38F3E17FB0BF34E88CDF884C019FB62
:104850000BF243F38F3830F8043B0E9042F38F395C
:1048600031F8042B0F9113FB0BF016FB0BF7279B72
:1048700047F38F3612FB0BFB40F38F3C4BF38F312A
:104880003344DDE9242BDDE92260269F2793013D97
:104890000F44464470446244CB44ADB2CDE922603B
:1048A000CDE9242B2697002D7FF44DAF5646CAF84C
:1048B00000500DF1400C46F8045FDFF818A12F46B8
:1048C0004FF06409E046331F4146CDF814801D4681
:1048D000CDE90361A8468E46AC1CAB463E46DEE9F8
:1048E000007080FB002C87FB0771930BB80B43EA29
:1048F0008C4540EA8142AB185ED49D1498034FF07A
:10490000804100239F0847EA817398424FEAA10142
:1049100075EB0102F6DB53EA01024FF000022ED0E4
:10492000CDE9008B1746CDF808E013EB020C41EB04
:10493000070E604575EB0E0B4FEA930809DBB0EBF1
:104940000C0065EB0E05DB1841EB010B9A1847EBE9
:104950000B0748EA81738910520853EA010C42EAB6
:10496000C7724FEA6707E0D109FB02F00028DDE9D2
:10497000008BB8BF5044DDF808E0C0F3875208F858
:10498000012B44450EF1080EA9D13746039E049928
:10499000A64201F1100101D0254699E7DDF814C0C7
:1049A00002375D46042F05F106060CF140088AD156
:1049B000082031B0BDE8F08F0022E0E798B700088A
:1049C00098C7000898D7000898AF000898E7000833
:1049D00040000120FFFF3F0007490023C1F898363F
:1049E000C1F89C36C1F8A036C1F8A436C1F8A83683
:1049F000A1F8AC36012070474000012008B54022E4
:104A00000021024805F050FA012008BDF0060120FF
:104A100005490023C1F8F036C1F8F436C1F8F8367C
:104A2000A1F8FC36012070474000012070B5A6B007
:104A300006469822144C0021684605F035FAFE22FD
:104A4000012325688DF802208DF805308DF8066069
:104A500003E02068411B642907D807216846FCF75A
:104A6000B3F80028F5D026B070BD084E08234FF4E7
:104A70000062402480254FF48050B361B261B4617C
:104A8000B561B061FEE700BF4000012000000240B8
:104A90002DE9F04F724D95F8CC6995F8CD39B342B8
:104AA00085B004463BD095F83007C0B3E17801F0FB
:104AB0000303012B00F08780022B00F09F80A17878
:104AC0007F2930D095F8CE29D5F8C81995F8817688
:104AD00041F8224095F8CE4995F8CD0995F8CC6972
:104AE00001345FFA84FB5E4598BF4FF0000B013044
:104AF00085F8CEB985F8CD09012F05D1594B85F838
:104B000082764FF400629A6195F830473CB1611E9D
:104B1000CFB205EB870885F83077D8F808472046EC
:104B200005B0BDE8F08F6379002BCBD0677895F89E
:104B30007F96B94501D0FF2FC4D1D4F890B0D5F8F5
:104B40006CAA494AD4F80690ABEB0A00A0FB02011C
:104B50000023464A02F084F9A0EB090808EBD8715B
:104B60004B10A3F1220727EAE77095F88176022F10
:104B70006BD0D5F850823D4A0090A8EB0A0CDFF8C4
:104B8000E8A00023ACFB0A0102F06AF9A8EB0B01D4
:104B9000364A01900023A1FB0A0102F061F9CDE938
:104BA00002091020E9466071B9E80F0095F8CDE9D7
:104BB000C4F80600B645C4F80A10C4F80E20C4F8BC
:104BC000123099D07EE795F87F0694F801808045F1
:104BD0007FF475AF9822002105F6D41085F8D039FE
:104BE00005F062F985F8D4892778237985F8D57995
:104BF0007F2685F8D66985F8D83963E795F87F76FA
:104C00006278BA4202D0FF2A7FF459AF95F8901625
:104C100000297FF454AF98221548012685F8D06901
:104C200005F042F985F8D4792378277985F8D539C4
:104C30007F20042185F8D60985F8D87985F8D91917
:104C4000D4F89420C5F8DA293CE706494A6982F489
:104C5000006343F000628A61D4F890B089E700BF36
:104C6000400001200008024040420F00400D0300B8
:104C7000140A01202DE9F04FDFF8E082B349D8F89B
:104C800038902022ADF2DC4D8A6199F805B0BBF175
:104C9000000F07D14FF40010886101200DF2DC4DA8
:104CA000BDE8F08F99F80300A94F10F0040F14BF6E
:104CB0000C260026C0F38003B91903EB4304A7F1C7
:104CC0002C0606EB840ABBF10C0F9AF82CC09AF85C
:104CD0002D7000918CBF022501255D440CEBC505AC
:104CE000B4AC6A1EC8F83410B2FBFCF500216A00AF
:104CF00020461FFA85FA05F0D7F8002F00F09C80B7
:104D00000AF1FF301FFA80FE0DF2D223914ACDF84E
:104D1000049003EB4E0C00208023002D00F08680D1
:104D2000ACEB0409A9F102014E08013616F00306A6
:104D3000214633D0012E20D0022E0FD0218892F8A8
:104D400000E04E0013EA0E0F214618BF46F00106A0
:104D500021F8026B5B0804BF013280230E8892F8B1
:104D60000090760013EA090F18BF46F0010621F8FB
:104D7000026B5B0804BF013280230E8892F800E0CA
:104D8000760013EA0E0F18BF46F001065B0821F803
:104D9000026B01D101328023614547D0B1F800E0B8
:104DA00092F800900E4613EA090F4FEA4E0118BF21
:104DB00041F0010126F8021B5B08B64608BF01322C
:104DC0003EF8021B92F8009008BF802313EA090FF7
:104DD0004FEA410118BF41F001015B082EF8021CA7
:104DE00001D180230132718892F800904FEA410E80
:104DF00013EA090F18BF4EF0010E5B0808BF01321D
:104E000006F10601A6F802E092F80090B68808BF05
:104E1000802313EA090F4FEA460618BF46F0010641
:104E20005B0821F8026CB5D06145B7D10130B842BA
:104E30007FF473AFDDF80490002D00F071820AF169
:104E4000FF318EB20DF2D22B0BEB460A32AF1AF0C5
:104E5000020F414DDFF8F4904FEA4606BB4616D0EC
:104E60002088009C0DF14202A36839460DF2D2243D
:104E70009847002858D0BDF84200002840F03A82F8
:104E8000D8F834200092A24507F1020B69D0009BAC
:104E900041E0BDF842300BF1020B0DF142025946E0
:104EA000A3B1B5F8A8C6D8F838E05CFA83F09EF84C
:104EB00088C0A5F8A80663448EF88830D9F8143065
:104EC00083F0400040F48003C9F81830D8F834006B
:104ED000836834F8020B984730B3BDF842000BF1F9
:104EE000020BA0B1D8F83810B5F8A82691F888E0E0
:104EF00052FA80F3704481F88800A5F8A836D9F8F2
:104F0000140080F0400141F48002C9F81820A24545
:104F1000D8F8343024D09B6834F8020B0DF14202EB
:104F2000594698470028B4D1084D0B4E6B69B6F826
:104F3000AA7683F0800242F400010137A961A6F845
:104F4000AA7600200DF2DC4DBDE8F08F000802408B
:104F5000ECA30008BE0A0120400001200000002050
:104F600000930DF1440A82220021504604F09CFF78
:104F7000009DCDF83CA095F80090012009F1FF3488
:104F8000A04081B2B1FA81F2C0F30B14C0F34A1110
:104F9000C2F11F03BD1CC0F3891203940491C0F336
:104FA000C814C0F30721AE1905920694C0F3462237
:104FB000C0F385240791C0F3C42102930096002317
:104FC00086B2C0F34E0CC0F38D0EC0F3CC0B08922A
:104FD0000994C0F30332C0F342340A91C0F3813123
:104FE000C0F3C0300B920C940D910E901A465446AB
:104FF000019600E00235019E002E00F0688139889C
:105000005F000E4218BF47F001073BB202F00707EE
:10501000072F02F1010008BF04F8013B80B20CBF6A
:1050200000239BB2BCF1000F00F04E8111EA0C0F7F
:105030004FEA430318BF43F0010300F0070A1BB215
:10504000BAF1070F02F1020608BF04F8013BB6B23D
:105050000CBF00239BB2BEF1000F00F0358111EAB6
:105060000E0F4FEA430318BF43F0010306F0070693
:105070001BB2072E02F1030908BF04F8013B1FFA17
:1050800089FA0CBF00239BB2BBF1000F00F01C811A
:105090000AF0070611EA0B0F4FEA430318BF43F06B
:1050A0000103072E039E1BB202F1040908BF04F896
:1050B000013B1FFA89FA0CBF00239BB2002E00F0BF
:1050C000038131424FEA43030AF0070618BF43F059
:1050D0000103072E049E1BB202F1050908BF04F864
:1050E000013B1FFA89FA0CBF00239BB2002E00F08F
:1050F000EB8031424FEA43030AF0070618BF43F042
:105100000103072E059E1BB202F1060908BF04F831
:10511000013B1FFA89FA0CBF00239BB2002E00F05E
:10512000D38031424FEA43030AF0070618BF43F029
:105130000103072E069E1BB202F1070908BF04F8FF
:10514000013B1FFA89FA0CBF00239BB2002E00F02E
:10515000BB8031424FEA43030AF0070618BF43F011
:105160000103072E079E1BB20ABF04F8013B9BB246
:105170000023002E00F0A88031424FEA430318BFFD
:1051800043F00103072F089F1BB202F1090608BF75
:1051900004F8013B1FFA86F90CBF00239BB2002FD5
:1051A00000F0928039424FEA430318BF43F00103F5
:1051B00009F00706099F1BB2072E02F10A0A08BF71
:1051C00004F8013B1FFA8AF90CBF00239BB2002FA1
:1051D0007AD0394209F007064FEA430318BF43F07B
:1051E0000103072E0A9E1BB202F10B0708BF04F849
:1051F000013BBFB20CBF00239BB2002E64D03142F2
:105200004FEA430318BF43F0010307F007060B9F63
:105210001BB2072E02F10C0A08BF04F8013B1FFA6B
:105220008AF90CBF00239BB2002F4DD0394209F000
:1052300007064FEA430318BF43F00103072E0C9EF5
:105240001BB202F10D0708BF04F8013BBFB20CBF4F
:1052500000239BB2002E37D031424FEA430318BFE0
:1052600043F0010307F007060D9F1BB2072E02F162
:105270000E0A08BF04F8013B1FFA8AF90CBF00238D
:105280009BB20FB339424FEA430318BF43F0010307
:1052900009F007060E9F1BB2072E02F10F0208BF8E
:1052A00004F8013B92B20CBF00239BB267B101F03E
:1052B000010141EA430602F00702072A37B20ABF9A
:1052C00004F8017BBBB200230299084482B2009823
:1052D00085422F467FF48EAED8F83890DDF83CA09A
:1052E00099F805B0BBF10C0F24D8BBF1000F79D1B0
:1052F0006949CFE4D8F83810B5F8A8E691F888C025
:105300005EFA80F2604481F88800A5F8A826D9F8F2
:10531000143083F0400040F48001C9F81810AFE564
:105320000DF1440A82222946504604F0BDFDBBF12E
:105330000C0F57D90DF14605D04605EB0B0C002399
:105340004BF6AD2418F8016B83EA06273BB2002B1D
:10535000B9B2B3BF84EA430349008BB29BB21AB21D
:10536000002AABBF5B0084EA42029BB293B218B240
:105370000028ABBF5B0084EA40009BB283B21DB241
:10538000002DABBF5B0084EA45059BB2ABB21EB2F9
:10539000002EABBF5B0084EA46069BB2B3B21FB2DD
:1053A000002FABBF5B0084EA47079BB2BBB219B2C8
:1053B0000029ABBF5B0084EA41019BB28BB21AB2F9
:1053C000002AABBF5B0084EA42029BB293B2C445A1
:1053D000B8D1002B59D03148B0F8A6460134A0F816
:1053E000A646AEE50BF1010400235FFA84F8D4462B
:1053F0001A463FE04500EEB274B2002CBABF660018
:1054000086F097067600F0B243B2002BBABF580080
:1054100080F097004000C5B26EB2002EBABF750092
:1054200085F097056D00EFB279B20029BABF4F0041
:1054300087F097077F00F8B244B2002CBABF600033
:1054400080F097004000C3B25DB2002DBABF6B0080
:1054500083F097035B00DEB277B2002F02F1010206
:10546000B8BF7E00D2B2ACBF760086F09706424548
:10547000F3B2AED21CF8010B584043B2002BB9DA9C
:105480005F0087F09701CEB2B6E75A46514609F160
:10549000060001F0FFFC2BE700080240400001205D
:1054A0002DE9F04FC178DFF83491447911F0040F01
:1054B00014BF0C230023ADF2A44D09F12C051D44AB
:1054C00003AF454B0646C1F380082246811D38468E
:1054D0005D6301F0DFFC0C2C00F28280002C00F0F8
:1054E0005E82BE463A19002026E04800C1B24BB2A7
:1054F000002B2EDB4900CBB258B2002830DB5B001A
:10550000D9B248B2002832DB4900CBB258B20028E9
:1055100034DB5B00D9B248B2002836DB4900CBB29D
:1055200058B2002838DB5B00D9B248B200283ADB19
:1055300049009645C8B23DD01EF8011B41404BB210
:10554000002BD2DA5B0083F09700C1B24BB2002B84
:10555000D0DA580080F09701CBB258B20028CEDAEA
:10556000400080F09703D9B248B20028CCDA40005E
:1055700080F09701CBB258B20028CADA400080F020
:105580009703D9B248B20028C8DA400080F09701EA
:10559000CBB258B20028C6DA400080F09703D9B2E7
:1055A00048B20028C4DA430083F0970A96455FFAB0
:1055B0008AF0C1D10DF1900B38554FF402720021E1
:1055C000584604F071FC08EB480209EB82094FF0E1
:1055D000010899F82CC066E000000020C0A3000874
:1055E000601E0DF10D0212FA80FABB4600234BF645
:1055F000AD211BF8010B83EA00231AB2002AABBFCE
:105600005B0081EA42029BB293B218B20028ABBFA2
:105610005B0081EA40009BB283B21AB2002AABBFA2
:105620005B0081EA42029BB293B218B20028ABBF82
:105630005B0081EA40009BB283B21AB2002AABBF82
:105640005B0081EA42029BB293B218B20028ABBF62
:105650005B0081EA40009BB283B21AB2002AABBF62
:105660005B0081EA42029BB293B218B20028ABBF42
:105670005B0081EA40009BB283B2DA45B9D13A19A6
:10568000190A0DF1900B39555846537000214FF40B
:10569000027204F009FC08EB480309EB83094FF0A0
:1056A000020899F82CC03878A0444FEAC801614438
:1056B00001F1FF3E9EFBFCF3002B40F3B380002280
:1056C0004FF0800A009401956446D9469646D44628
:1056D0001D464FF0000129F8021B002C00F09980B4
:1056E000002314F0030A194640D0BAF1010F27D065
:1056F000BAF1020F10D01CEA000F14BF01230023DF
:105700005FEA5C0C07D10132D2B290458CBFB85C25
:1057100060464FF0800C01211CEA000F4FEA430362
:1057200018BF43F001035FEA5C0C9BB207D1013262
:10573000D2B290458CBFB85C60464FF0800C01310E
:105740001CEA000F4FEA430318BF43F001035FEA6E
:105750005C0C9BB207D10132D2B290458CBFB85CD1
:1057600060464FF0800C0131A14250D01CEA000F7E
:105770004FEA430318BF43F001035FEA5C0C9BB29E
:1057800007D10132D2B290458CBFB85C60464FF071
:10579000800C1CEA000F4FEA430318BF43F00103DB
:1057A0005FEA5C0A01F101019BB207D10132D2B27A
:1057B00090458CBFB85C50464FF0800A1AEA000F43
:1057C0004FEA430318BF43F001035FEA5A0C9BB250
:1057D00007D10132D2B290458CBFB85C60464FF021
:1057E000800C1CEA000F4FEA430318BF43F001038B
:1057F0005FEA5C0C9BB207D10132D2B290458CBFFC
:10580000B85C60464FF0800C0331A142AED129F85C
:10581000023C0EF101011FFA81FE75453FF759AFB9
:10582000DDE90045A6AF4FF402720021384604F0CE
:105830003BFBB9464FF000082CB10C2C8CBF022367
:1058400001231C44E4002A781319581E90FBF2F13E
:1058500041450BDD6A683BF8020B9047594B29F82C
:10586000020B74795D6B08F10108E5E76E7801259C
:10587000741EA540ACB288B2002C00F08C80421E91
:105880001FFA82FBBB1C504A03EB4B050023002888
:105890007ED0E91B8E1E7108013111F003013E46D6
:1058A00038D0012923D0022910D0117836F802AB64
:1058B000013314EA0A0FDBB24FEA410118BF41F08D
:1058C0000101082B117004BF00230132117836F852
:1058D00002CB013314EA0C0FDBB24FEA410118BFCF
:1058E00041F00101082B117004BF0023013211782F
:1058F00036F8028B490014EA080F03F10103DBB20A
:1059000018BF41F00101082B117004BF00230132C0
:10591000B5423DD03146167831F8029B0133DBB2F7
:1059200014EA090F4FEA460618BF46F00106082B95
:10593000167004BF013200231678B1F800E001337D
:1059400014EA0E0F4FEA4606DBB218BF46F0010616
:10595000082B167001D1002301321678B1F802B07D
:10596000B1F804A0013314EA0B0FDBB24FEA46068C
:1059700018BF46F00106082B167008BF013201F16E
:105980000606117808BF0023490014EA0A0FB4E79D
:1059900064087FF47CAF0DF2A44DBDE8F08F0DF1EB
:1059A000900B21464FF4027258463C7004F07CFA8A
:1059B00008EB480009EB8008214698F82CC02046E7
:1059C000A04674E600000020D20B01202DE9F84328
:1059D000374A384D5369384F064683F0020040F489
:1059E0000031916105F6984000214FF42A7204F0CD
:1059F0005BFA0024B000314B314E324985F8404FFC
:105A0000A5F8444F05F6487C05F6587EA7F5FF68D3
:105A1000DCF80420DCF80090034401449342CCF805
:105A2000001041D0CCF804300021CEE90011CEE9BD
:105A30000211A6F50053C3E90011C3E90411C3E93B
:105A40000811C3E90C11C3E91011C3E91411C3E92A
:105A50001811C3E91C118033B342ECD19CB957F83B
:105A6000044FA17894F8009008EB810308EB8902B9
:105A7000D3F80038D2F800180CF1080C08360EF1F3
:105A8000100E0124C4E70A4C0F4810490422A261F9
:105A90006669C5F8C00886F0020747F40033C5F808
:105AA000B818A361BDE8F8834945D7D0BCE700BF6B
:105AB000000802404000012098EF000898CF00083D
:105AC0005444012098AF0008DB1B0400B9A2010078
:105AD0002DE9F04F114D124AB5F8983604464FF4AF
:105AE0000061A3B00133916105F684304FF48972EF
:105AF0000021A5F89836002604F0D6F9FDF7C2FE7D
:105B0000A7882068ADF84C70A5F8786F12900DF159
:105B100048090DF14E0A374608E000BF4000012059
:105B2000000002405300CA45DFB243D019F8012BF0
:105B30007A4055B2002DBABF6A0082F09702520037
:105B4000D3B259B20029BABF4B0083F097035B0070
:105B5000DEB270B20028BABF460086F09706760023
:105B6000F7B27AB2002ABABF570087F097077F00D2
:105B7000FDB26BB2002BBABF5D0085F097056D00DA
:105B8000E9B24EB2002EBABF710081F09701490010
:105B9000CFB278B20028BABF470087F097077F00DE
:105BA000FAB255B2002DBDDA690081F09706CA45F8
:105BB000F7B2BBD10023CDE91B33CDE91D33CDE9CD
:105BC0001F338DF84E700DF16A0B9DF848702193CC
:105BD0000DF18600D9464FF0800C07EA0C02D5B2D1
:105BE000291ECCF3470E18BF0121BEF1000F40F073
:105BF0005D810133DBB2062B4FEA410109D803F185
:105C000088080DEB080717F9406C17F840EC41EADB
:105C1000D671CEF3801545EA41084FF0200C1EEAFC
:105C20000C0F4FEA480218BF42F001025FEA5C071E
:105C300092B240F094850133DBB2062B4FF0800C1A
:105C400005D803F188070DEB070616F8407C29F804
:105C5000022F4845C1D10023CDE91433CDE91633D5
:105C6000CDE91833C24D1A933BF8022FDFF80893A1
:105C7000002139F8027F02EA070616F00F030CD064
:105C80005F0887EA030700F06E819E0887EA060630
:105C900001D086EAD30707F00103490089B2A9457C
:105CA00041EA0301E5D183452AF8021FDCD1BDF8A2
:105CB0005000BDF85250BDF85A70BDF85E60BDF896
:105CC0006230BDF85620BDF8661005900495029725
:105CD000069607930820BDF85480BDF858E0BDF83B
:105CE0005CC0BDF86070BDF86460BDF86850BDF878
:105CF0006AB0A04B03920891002280210190059880
:105D0000084218784FEA400018BF40F001005FFADF
:105D100080FA049808424FEA4A0018BF40F0010098
:105D20001870901CC0B2082840F02881587818EAF2
:105D3000010F14BF0122002242EA40025A700133CF
:105D400001220398084218784FEA400018BF40F03B
:105D500001001870501C5FFA80F9B9F1080F40F08B
:105D60004E815A781EEA010F4FEA420018BF40F0F8
:105D7000010058700122013302980842187814BFBC
:105D80004FF001094FF0000949EA40001870501C1B
:105D9000C0B2082840F0258193F8019011EA0C0F59
:105DA00014BF0122002242EA49025A700133012243
:105DB00006980142187814BF4FF001094FF000090E
:105DC00049EA40001870501CC0B2082840F0FC801E
:105DD00093F801900F4214BF0122002242EA4902C7
:105DE0005A700133012207980142187814BF4FF00E
:105DF00001094FF0000949EA40001870501CC0B278
:105E0000082840F0D48093F80190314214BF012259
:105E1000002242EA490058700122013308980142E9
:105E2000187814BF4FF001094FF0000949EA40000B
:105E30001870501CC0B2082840F0AD805A78294232
:105E40004FEA420018BF40F00100587001220133B0
:105E500018781BEA010F4FEA400018BF40F001001C
:105E60000132D2B218700198082A04BF013300220F
:105E700001384FEA510101907FF441AFA77866796C
:105E80007F2F00F0CA80002E00F0CA802046FFF766
:105E900007FB6479002C00F0C3800C2C8CBF4FF002
:105EA00002084FF001084444E500BAE007EA0E0694
:105EB000F2B24D00002A18BF45F001051CF47F7FA7
:105EC000CCF3870E1DD10133DBB2062B16D803F1BC
:105ED00088020DEB020E1EF9401C1EF8407CCE0F0E
:105EE00046EA4506C7F3801545EA460229F8022F1F
:105EF00048454FF0200C7FF470AEACE66E0077465C
:105F0000F0E717EA0E0F4FEA4501CCF3C70C0CBFC0
:105F1000884641F00108BCF1000F40F01D840133B8
:105F2000DBB2062B13D84FF0400C03EB0C064836BF
:105F30000DEB060212F9405C12F8407CE90F41EAD1
:105F4000480229F8022F48457FF447AE83E64FEA1E
:105F50004807BAB229F8022F484567464FF0400C6F
:105F60007FF43BAE77E6012707F0010395E600BF1B
:105F700012A40008C40B012002A40008187818EA33
:105F8000010F4FEA400002F1030218BF40F0010088
:105F9000D2B21870D5E693F800A0294214BF0120B0
:105FA0000020023240EA4A00D2B2187050E793F85B
:105FB00000A0314214BF01200020023240EA4A0909
:105FC000D2B283F8009029E718780F424FEA4009CF
:105FD00002F1020218BF49F00109D2B283F8009021
:105FE00001E7187811EA0C0F4FEA400902F10202AA
:105FF00018BF49F00109D2B283F80090D8E61878AA
:106000001EEA010F4FEA400902F1020218BF49F0EF
:106010000109D2B283F80090AEE6002E40F07C83F6
:106020000025D748436B847F93F800E05978D54822
:10603000019475446A1E92FBFEF711FB07F6703659
:10604000B6B290F88456A0F8786F002C00F07F83E9
:10605000C5EBC501CC4CCD4F0297CDE904654FF09F
:10606000000AC1EBC1024FEAC50C0392202104F5DE
:10607000806B0123D046D146CDF818C0039DEE18A1
:10608000029B03EB460E6818BEF9B02003EB4001FB
:10609000D717B1F9B050BE0346EA92415619F3172B
:1060A00090033246079300F08BFE0746E817810302
:1060B000079B324641EA9541A80300F081FE0BF2AE
:1060C000FE33ABF102050646C346023C9846B4F9DE
:1060D0000200B5F902C006FB00F007FB0C02A91C88
:1060E000A31C42F38F3008910793FCF7B5FD079886
:1060F000089AB0F90210B2F9023006FB01F107FB71
:10610000031040F38F30FCF7A7FDB4F90610B5F982
:10611000062006FB01F107FB021343F38F30FCF767
:106120009BFDB4F90800B5F9081006FB00F007FB69
:10613000010242F38F30FCF78FFDB4F90A30B5F954
:106140000A0006FB03F307FB003141F38F30FCF735
:1061500083FDB4F90C30B5F90C2006FB03F307FB03
:10616000023040F38F30FCF777FDB4F90E10B5F92B
:106170000E3006FB01F107FB031242F38F30FCF7F0
:106180006BFD34F9100F35F9101F06FB00F007FB0B
:10619000010343F38F30FCF75FFD454597D1D846A7
:1061A000B9F1000F1BD14FF00109019E0AF1010A5C
:1061B000B24523D0764F029D07EB8902D2F8F8074B
:1061C00010F8083000EB080605EB830CB178DCF81A
:1061D000FC4205EB810EA346DEF8FC424EE70BF1D4
:1061E00001075FFA87F8B8F1010F4FF00009DCD919
:1061F000019E0AF1010AB245C846DBD1DDE904651A
:10620000DDF818E0DFF890910496AEEB0504C4EBDE
:10621000C402002701970392A9F5006AA9F58064DA
:106220000E214FF0130C0595F0460398461802997D
:10623000844401EB460B01EB4C0CBBF9B030BCF9CC
:10624000B050DA175E19900340EA93413246980342
:10625000F317069300F0B4FDE9178346880340EA7C
:1062600095413246A803069B00F0AAFDAAF102055B
:106270000646023C0AF2FE3AB4F90220B5F902E001
:1062800006FB02F20BFB0E23A91CA21C43F38F306A
:1062900007910692FCF7E0FC0698079BB0F9021004
:1062A000B3F9022006FB01F10BFB021040F38F3023
:1062B000FCF7D2FCB4F90610B5F9063006FB01F183
:1062C0000BFB031242F38F30FCF7C6FCB4F9080055
:1062D000B5F9081006FB00F00BFB010343F38F3008
:1062E000FCF7BAFCB4F90A20B5F90A0006FB02F281
:1062F0000BFB002141F38F30FCF7AEFCB4F90C200E
:10630000B5F90C3006FB02F20BFB032040F38F3093
:10631000FCF7A2FCB4F90E10B5F90E2006FB01F152
:106320000BFB021343F38F30FCF796FC34F9100F8C
:1063300035F9101F06FB00F00BFB010242F38F3012
:10634000FCF78AFC554597D1019E3EBB0124019480
:10635000104B99452CD019F8010F0D4B029C03EB03
:10636000800ADAF8F867F519F15D95F802C004EBD8
:10637000810B04EB8C0EDBF8FCA2DEF8FC4254E748
:10638000000000204000012064F00008C0A30008C5
:10639000A0E7000867000108640001080137FFB2A8
:1063A000012F40F2B681CB4B002799450197D2D1FE
:1063B000C94ADDE90461147E0794002E00F04E8185
:1063C000A8EB0105C5EBC5070D97C44C0027019745
:1063D0004FF0800B94F800C01BEA0C0F14BF012093
:1063E00000205FEA5B0340F0648162784FF020098F
:1063F000D1090134C2F38012237819EA030F14BFC4
:10640000012300235FEA590B02D101344FF0800BC6
:10641000079D0437BFB2002D00F01D81B04D05EB84
:10642000800A05EB810E05EB820805EB830CCDE9B4
:106430000E67CDE9104BDAF8D007DEF8D017D8F8A0
:10644000D027DCF8D037029C099000250A910B92E6
:106450000C930495019EA24B099F0A980B990C9DE1
:10646000334493F8D89793F8DBA793F8DE8793F833
:10647000E12793F8E46709EB490B0AEB4A0E08EBB6
:10648000480C02EB420986448C4493F8E70793F8E2
:10649000EA1793F8ED37A944BB441CF801501BF8E8
:1064A000067019F803201EF800600D990392C819B0
:1064B0008B19039A089504EB430E04EB400B4D191E
:1064C00004EB450804EB870A1144BEF9B090BBF910
:1064D000B000DAF8FC72B8F9B0B0059704EB410CE3
:1064E00009EB0003BCF9B0705B44FD18C2174FEA1A
:1064F000E578910343462A4641EA9041800300F043
:106500005FFC82464FEAE970830343EA99412A46D9
:1065100043464FEA893000F053FC4FEAEB72910397
:1065200043462A4641EA9B4181464FEA8B3000F0C0
:1065300047FC2A46FD170690A803434640EA9741C8
:10654000B80300F03DFC089F039B04EB870804EBB5
:10655000860604EB8302D6F8FC128346D8F8FC02C8
:10656000D2F8FC52059B0394069C8F1E861E023DAA
:10657000A3F1020803F2FE31B7F90220B8F90200D4
:10658000B6F902E0089109FB02F1B5F902C00AFB75
:10659000001204FB0E210BFB0C1308F10202B11CCC
:1065A00043F38F3006920591FCF756FB069BB7F933
:1065B00004000599B3F90220B1F9023009FB00F09B
:1065C0000AFB020204FB0321B5F904300BFB0310A4
:1065D00040F38F30FCF740FBB7F90620B8F90630DE
:1065E00009FB02F1B6F906200AFB0310B5F90630E3
:1065F00004FB02010BFB031040F38F30FCF72CFB74
:1066000037F9082F38F9083F09FB02F136F9082F4E
:106610000AFB031035F9083F04FB02010BFB0310D2
:1066200040F38F30FCF718FB08994145A4D1019F36
:10663000049D079A039C0137FEB2032E05F1010564
:1066400008BF00269542049501967FF403AFDDE96B
:106650000E67DDE9104BBE423FF6BCAEFCF7C6FA52
:106660002049D1F85802D1F85C3298420FD01E4F21
:106670001E4E1025BD61346924F00402326130BF22
:106680001849D1F85802D1F85C329842F2D1164F2D
:10669000144A174E4FF48015BD61D2F850124FF0D6
:1066A0000064B461C2F86C1A23B0BDE8F04FFDF786
:1066B00049BA13EA0C0F14BF012100215FEA9B02C3
:1066C00018D163784FF0200BDA090134C3F380133B
:1066D0009EE600BF6700010800000020C40B0120F7
:1066E00098F80008400001200008024000ED00E09A
:1066F0000000024012EA0C0F14BF012200225FEAE0
:10670000DB097FF479AE65784FF0400BEB0901347B
:106710007EE6002501951BE6134E2046D6F8505222
:10672000FEF7BEFED6F85032D4F806200F49C5EB6E
:106730004300871AA7FB01010D4A002300F090FBDC
:106740006679C4F80600002E7FF4A0AB68E4094B1C
:1067500002934FEAC50E55E5BE46FFF760BABC4648
:106760007746FFF774BA00BF4000012040420F0097
:10677000400D0300C0A300082DE9F04F4B4C94F8E6
:106780007B3F0022A3B084F87A2F002B00F009830E
:10679000474800F57F68CDF81C80464994F8807F13
:1067A0000D7B94F8819FD4F87C6FAF4228BF2F46B1
:1067B000A94538BFA94640222E44002112A8C4F89A
:1067C0007C6F84F8807F84F8819F03F06DFB94F8E0
:1067D000822F94F8830F0132D3B2984284F8823F1B
:1067E00000F0C8823249344E344ACD1895F8D8A703
:1067F00095F8E4B70AEB4A0CB444DC449CF8F8760C
:106800009CF804E702EB870802EB8E09D8F8001821
:10681000D9F80008264D284E2B44CDE90A1093F8EC
:10682000DBA793F8DEC793F8E72793F8E1E793F83F
:10683000EA9793F8ED370AEB4A0BB34493440CEB19
:106840004C07F0190EEB4E089BF804179BF8F876EE
:106850004844B044194E984406EB810A06EB870B76
:1068600090F8041790F8F876DAF80028DBF800388A
:106870000D9206EB870006EB810C98F8F87698F8F5
:106880000417DCF800280C9306EB870806EB810E52
:10689000D0F80038DEF80068D8F800080F924FF4FE
:1068A00000750E931196109010E000BF400001207B
:1068B00098F800080000002090090108A0E70008EF
:1068C000C4490A6922F004060E6130BFD4F870246E
:1068D000D4F874349A42F3D00DF12600FBF7DCF8BB
:1068E0000028EDD0DDE90A6CBDF926307188BCF8CE
:1068F0000200DDE90C2B11FB03F747F38F395788B2
:1069000010FB03F117FB03F041F38F3E40F38F318F
:1069100036F8040B0A9610FB03F63CF8040BCDF88E
:106920002CC05F4646F38F3A10FB03F646F38F38D0
:1069300032F8040B37F8046B0C9210FB03F216FBD1
:1069400003F0D4F8886F42F38F3C40F38F321298F3
:106950001E44C4F8886F0AEB000613980596129639
:1069600009EB000614980696139608EB0006159896
:10697000049614960EEB00061698039615960CEBEB
:1069800000060296169617980D970144BBF8027000
:1069900001911791189917FB03F01144DDE9107C60
:1069A000D4F8842FB7F802A0189103FB03F902EB87
:1069B000A93640F38F3BDDE90E201AFB03F851881E
:1069C00032F804ABC4F8846F0E9211FB03F61AFB85
:1069D00003F2418842F38F3A30F8042B0F9046F3CC
:1069E0008F3911FB03F612FB03F046F38F3E37F8A5
:1069F000042B1097664612FB03F736F8042B48F376
:106A00008F3140F38F3847F38F3012FB03F747F392
:106A10008F32199F5F4419971A9F57441A971B9FEB
:106A20004F441B971C9F47441C971D9F77441D97FD
:106A30001E9F119607441F98BCF802601E970844D9
:106A400020991F90114416FB03F3219A2091013DD8
:106A500043F38F3B5A44ADB22192002D7FF436AF01
:106A60005D4F94F88CBF0825BD6194F87A6FBBF137
:106A7000000F00F083800598069D80FB001C85FBBD
:106A800005798B0BB80B049940EA894A039843EACD
:106A90008C4281FB01359F0B80FB003847EA854122
:106AA0009D0B04EB461945EA884C52446144BBF106
:106AB000010FC9F8902FC9F8941F5FD0019981FB8D
:106AC00001050299830B43EA854081FB0153A90B21
:106AD000DDE9182741EA834A5044C9F8980F87FB3B
:106AE0000770BD0B82FB0227910B45EA804341EA08
:106AF00087484344BBF1020FC9F89C3F3ED0DDE913
:106B00001A02DDE91CA582FB0237990B80FB00030A
:106B100041EA8742870B47EA834C85FB05588AFB8D
:106B20000A036244A90B870BC9F8A02F47EA834ADE
:106B300041EA88425244BBF1030FC9F8A42F1DD08B
:106B4000DDE91E2C8CFB0C138F0BDDE9200547EAD9
:106B5000834182FB0223970B47EA8348414480FB31
:106B6000000A85FB053CC9F8A81F9D0B810B41EA73
:106B70008A4245EA8C473A44C9F8AC2F94F87B8F97
:106B8000154801365FFA86F94FF40021C84584F8AC
:106B90007A9F81613FF601AE0F4B10229A61BBF1E3
:106BA000000F00F0E0800D48DFF834E030F8605C62
:106BB0009EF81810DFF82C8003910135049550E9F8
:106BC0001A5600270196DEF83C60029708EB411C3C
:106BD0000AE000BF00ED00E000080240381101208B
:106BE00000000020D00F0120039B9946002B00F0ED
:106BF000978008EBC701ACEB010AAAF12002520909
:106C000001324FF0000912F003024FEAC70A4B4667
:106C100038D0012A23D0022A10D058F80AA04A6896
:106C20005245ABBFA2EB0A02AAEB02024FF0010AE7
:106C3000CA46002AC4BFD14613462031D1E900A27A
:106C40005245ABBFA2EB0A02AAEB02024FF0010AC7
:106C50004FF0000A9A42C4BFD14613462031D1E911
:106C600000A25245ABBFA2EB0A02AAEB02024FF010
:106C7000010A4FF0000A20319A42C4BFD1461346A0
:106C8000614548D00A462BE0A3EB09034FF0000909
:106C90005345D6BF5346CA468A46D2E908198945A4
:106CA000ABBFA9EB0101A1EB09014FF001094FF0C6
:106CB00000099942DCBF1946D146D2E9103A9A45FB
:106CC000ABBFAAEB0303A3EB0A034FF0010A4FF09B
:106CD000000A60328B42CCBFD1460B4662451AD0C7
:106CE000D2E9001A8A45B5BFA1EB0A0AAAEB010A4C
:106CF000002101219A45D8BF9A4602F1200213686B
:106D0000D8BF4946D2F804909945BDDBA9EB0303EF
:106D10004FF00109BCE7019A5D1942EBE371019163
:106D20003378049949EA43023270CA191FFA82F98A
:106D3000520707D11C4B0136F11AB1F5897F1FD2DA
:106D4000012202920137BB450CF1080C7FF44CAFD5
:106D5000029C20F8609C0CB1CEF83C60019E40F88B
:106D6000685C40F8646C11484FF48017876123B069
:106D7000BDE8F08F00230E48079984F8823F49E56B
:106D8000B4F8AC3640F8685C019DCEF83C60013345
:106D900020F8609C40F8645CA4F8AC3623B0BDE8F1
:106DA000F08F94F88CBFF7E6B00A0120000802408B
:106DB00088000108014BC3F8F8017047400001202A
:106DC0007BB972B90029BEBF00204FF0004106E038
:106DD00008BF00281CBF6FF000414FF0FF3000F0EB
:106DE00057B8ADF1080C6DE904CE002909DB002B82
:106DF0001ADB02F0FBFEDDF804E0DDE9022304B05B
:106E00007047404261EB4101002B1BDB02F0EEFEBC
:106E1000DDF804E0DDE9022304B0404261EB41010A
:106E2000524263EB43037047524263EB430302F069
:106E3000DDFEDDF804E0DDE9022304B0404261EB51
:106E400041017047524263EB430302F0CFFEDDF88D
:106E500004E0DDE9022304B0524263EB43037047D0
:106E600053B94AB9002908BF00281CBF4FF0FF31B1
:106E70004FF0FF3000F00CB8ADF1080C6DE904CE16
:106E800002F0B4FEDDF804E0DDE9022304B070474F
:106E9000704700BF844641EA000313F003036DD13D
:106EA000403A41D351F8043B40F8043B51F8043BCD
:106EB00040F8043B51F8043B40F8043B51F8043BD4
:106EC00040F8043B51F8043B40F8043B51F8043BC4
:106ED00040F8043B51F8043B40F8043B51F8043BB4
:106EE00040F8043B51F8043B40F8043B51F8043BA4
:106EF00040F8043B51F8043B40F8043B51F8043B94
:106F000040F8043B51F8043B40F8043B51F8043B83
:106F100040F8043B51F8043B40F8043B51F8043B73
:106F200040F8043B403ABDD2303211D351F8043B13
:106F300040F8043B51F8043B40F8043B51F8043B53
:106F400040F8043B51F8043B40F8043B103AEDD2C2
:106F50000C3205D351F8043B40F8043B043AF9D213
:106F6000043208D0D2071CBF11F8013B00F8013BE6
:106F700001D30B8803806046704700BF082A13D3F3
:106F80008B078DD010F003038AD0C3F10403D21A0B
:106F9000DB071CBF11F8013B00F8013B80D331F83F
:106FA000023B20F8023B7BE7043AD9D3013A11F8BF
:106FB000013B00F8013BF9D20B7803704B7843702A
:106FC0008B7883706046704700000000000000006E
:106FD00000000000000000000000000000000000B1
:106FE00000000000000000000000000000000000A1
:106FF0000000000000000000000000000000000091
:1070000030B490F800F020F007016FF0000C10F0A1
:10701000070491F820F040F048804FF000046FF032
:107020000700D1E9002391F840F000F1080082FA4E
:107030004CF2A4FA8CF283FA4CF3A2FA8CF34BBB19
:10704000D1E9022382FA4CF200F10800A4FA8CF292
:1070500083FA4CF3A2FA8CF3E3B9D1E9042382FA60
:107060004CF200F10800A4FA8CF283FA4CF3A2FA75
:107070008CF37BB9D1E9062301F1200182FA4CF2AD
:1070800000F10800A4FA8CF283FA4CF3A2FA8CF314
:10709000002BC6D0002A04BF04301A4612BAB2FA36
:1070A00082F200EBD20030BC7047D1E9002304F03B
:1070B0000305C4F100004FEAC50514F0040F91F870
:1070C00040F00CFA05F562EA05021CBF63EA05030D
:1070D00062464FF00004AAE72DE98048D3B072B6AB
:1070E0000025BC4C0E95236BDFF8008343F00100B4
:1070F0002063216B01F001020E920E9B0D95266B11
:1071000046F002072763236B03F002000D900D9BEE
:107110000C95216B41F004022263266B2E9506F03C
:1071200004070C97AC4F0C9B2F952CA938460126D1
:107130002D962C96F9F798F94FF48033BB614FF0F8
:10714000020ACDF8B0A0F9F78FF94FF40032BA6116
:107150004FF00409CDF8B090F9F786F94FF480208C
:10716000B8614FF4006340464FF0006B2C93F9F781
:107170007BF93846C8F818B008222C92F9F774F950
:107180004FF40023BB614FF400622C92F9F76CF9C5
:10719000C7F818B04FF0400BCDF8B0B0F9F764F96C
:1071A0004FF48003BB6180222C92F9F75DF94FF414
:1071B0000003BB614FF480522C92F9F755F94FF060
:1071C0008053BB6110272C97F9F74EF9834A8761EA
:1071D0004FF48073CDE92C32F9F746F92A46294657
:1071E0001720F9F71FF80B95206B40EA090323637A
:1071F000226B4FF480612C9102EA090140460B9109
:107200002CA90B9ADFF8E881CDE92D65CDE92F6532
:10721000F9F72AF9CDF8B0A0F9F726F9CDF8B09032
:10722000F9F722F908232C93F9F71EF92C97202758
:10723000F9F71AF92C97F9F717F9CDF8B0B0F9F773
:1072400013F980222C924FF40077F9F70DF94FF4DF
:1072500080732C93F9F708F92C97F9F705F94FF497
:107260008017C8F84457C8F83C574FF400314FF026
:1072700080654FF480224FF40023856181614FF4D3
:10728000001582614FF4800183614FF40002876131
:107290004FF080734FF00077856181618261836177
:1072A000876198F86D574FF0804011211822C8F877
:1072B0003407C8F84017C8F83827002D00F0CF84ED
:1072C0004749022588F86D57F9F732FA454BC8F857
:1072D000605001274AF6C8764FF4FA7188F86D7746
:1072E0009E62D962DF601F600024082698F8A10022
:1072F000C8F85840C8E91C4403F55053C8F8644026
:10730000C8F878404FF482724FF40064C8F86C609B
:1073100007214FF40076C8F85C40C8F85030C8F830
:107320005420C8F87C10C8F8686000F0FF040028FA
:1073300000F026854FF0020A88F8A1A0196821F014
:1073400040061E60D8E91557D8F85C00D8F86040B0
:10735000D8F86430D8F86C10D8F87060D8F850209D
:107360003D43054325431D43D8F87870D8F868009D
:107370000D43354300F400743D4325431560B8F8D0
:107380006A50D8F87410D8F85020174C05F0040350
:107390000B435360D669002126F400670120D761B2
:1073A000C8F8A41088F8A10098F8E520C8F8BC1027
:1073B0004FF4E1350C23C8E92D11C8E93111C8E9B2
:1073C0002B45C8F8C03002F0FF06002A00F08A847E
:1073D0000F460FE00038024000000240000011108C
:1073E000780701200004004000100140000802401E
:1073F00040000120242188F8E510E06820F40056C0
:10740000E6602369D8F8B81023F440520A43226199
:10741000D8E92F60E3680643D8F8C80023F4164281
:10742000064322F00C013E430E43E6606769D8F83C
:10743000C43027F440761E436661D8F8C820B2F500
:10744000004F00F01085CD498C424FEA850500F0D1
:10745000318401F58060844200F02C84FBF742FC0B
:107460008346FBF73FFC4FF0190909FB00F7FBF7D8
:1074700039FCB7FBF5F68246FBF734FC09FB00F359
:10748000B3FBF5F7FBF72EFC642109FB0AFC09FBB3
:107490000BFE09FB00F0BCFBF5FBB0FBF5F9BBFBF9
:1074A000F1FAB9FBF1F301FB1A6601FB1377300126
:1074B0003A0132303232B0FBF1F6B2FBF1F7BEFBEB
:1074C000F5F507F00F03B5FBF1F506F0F0011943F0
:1074D00001EB0510A060206920F4904222616569EB
:1074E00025F02A076761E66846F40051E1604FF035
:1074F000200E0024C8F8E84088F8E5E088F8E6E0C7
:10750000FBF7ACFE9E4B9F4AD8F84470C8F80C407D
:107510004FF480300125C8E90130C8E90B24C8F8D0
:107520001440C8F81C40C8F82440C8F81040C8F8F7
:107530003440C8F81850002F01F06C82D8F844701D
:10754000FA0641F1DB8000264FF0010B199688F80E
:1075500040B018698C4C20F0E0621A611D6945F05A
:1075600000711961586B20F01F025A635D6B082788
:107570003D435D63854B88F8406044E9177B4026B6
:107580009F6180214FF400674FF480509F619E619E
:107590009961986198F839520222202D44F8542CB0
:1075A00000F087847A4C00222046FF27012188F8CA
:1075B0007F2688F87C76FAF7C9FAA8F87D06734C1E
:1075C0004FF480014FF00060A161A061FBF736FA33
:1075D00072B6704B704D5D6062B64FF48036002716
:1075E0004FF400314FF48022A66188F8837688F842
:1075F0006274A161A261A661A161A26172B6C8F8BC
:107600005872C8F85C7262B672B6C8F87074C8F87E
:10761000747462B6FCF796FA5B4B4FF40020A061DD
:1076200013F84C5C4FF400064FF08057A661A76139
:107630003DBB5549594CC8F800474FF0010A052297
:1076400001F84CACC8F804272B46D8F8000740F8DE
:107650002530013598F80467EFB2BE42F5D8504D99
:10766000C8F8C85905240023C8F8CC491A46D8F8E8
:10767000C81941F82320013398F8CCB9D8B2834512
:10768000F5D8484EC8F8086706F1980706F53E7227
:10769000C8F80C7706F59867C8F81C2706F59875A2
:1076A000A7F58F6206F5E47406F5187306F56471A4
:1076B00006F5856006F5AB66C8F82877C8F82C672C
:1076C000394F3A4EC8F81057C8F81447C8F8183759
:1076D000C8F82017C8F82407C2F8C475C2F8C865EE
:1076E000334D344C344B35493548364F364EC2F85D
:1076F000A855C2F8B445C2F8B835C2F8BC15C2F8EE
:10770000C005C2F80876C2F80C66304D304C314BDB
:1077100031493248324F334EC2F8CC55C2F8F845A1
:10772000C2F8FC35C2F80016C2F80406C2F8287682
:10773000C2F82C662C4D2D4C2D4B2E492E482F4F28
:107740002F4EC2F810564FF00A0CC2F81446C2F879
:107750001836C2F81C16C2F820062A4D2A4C2B48AF
:107760002B492C4B88F830C7C2F84876C2F86C66B3
:10777000294F2A4EC2F8705652E000BF0010014057
:10778000002001400100000F3811012000000240DC
:10779000BF0601200000002035190008E41A01206E
:1077A000F81A0120F0100120ED1C0008F51C00085B
:1077B000351B0008391B0008A1430008CD1C000838
:1077C000D51C0008A1420008E1420008191D00086C
:1077D0007D1D0008BD1D00081D430008251E000872
:1077E000E11F000861200008D51E00084D1F000899
:1077F000851F0008C91F0008813A0008C920000839
:10780000A93C0008DD3D000895420008C53F00087E
:107810000D210008612100081121000869210008DC
:10782000C2F87446C2F87806C2F88816C2F88C7698
:10783000C2F8A836C2F8B066784D794C79487A49D2
:107840007A4B7B4F7B4EC2F8A857C2F8B447C2F8B8
:10785000B807C2F8BC17C2F8C037C2F8C477C2F87C
:10786000C867754D754C76487649774B774F784E9B
:10787000C2F8CC57C2F8F847C2F8FC07C2F80018A3
:10788000C2F80438C2F80878C2F80C68DFF828E2B9
:10789000DFF82892DFF828A2DFF828B26D4D6E4C91
:1078A0006E486F496F4B704F704EC2F8ACE6C2F82D
:1078B000B496C2F8B8A6C2F8BCB6C2F81058C2F85E
:1078C0001448C2F81808C2F81C18C2F82038C2F8C8
:1078D0002878674DC2F82C68664C67486749684B42
:1078E000684F694EC2F84858C2F86C48C2F8700830
:1078F000C2F87418C2F87838C2F88878C2F88C6870
:10790000624D634C63486449644B654F654EC2F8F1
:10791000A858C2F8AC48C2F8B008C2F8B418C2F807
:10792000B838C2F8BC78C2F8A8695F4AC8F8F8212C
:1079300062B65E4D5E4EDFF890B18024AC610020EF
:10794000012788F8540288F86374FCF7B7F8FCF74D
:10795000F9F888F8AA70574991F8D459002D01F028
:107960002380012D00F03385022D01F0648198F809
:107970008626002A00F00783D8F88816D8F87836CB
:10798000B8F88C565C1AA7B2AF42C0F0FC82781BE4
:107990002944B8F88E562A18B2F5004FA1EB050419
:1079A00088BF24184FF000014FF098022CA888BF20
:1079B000A8F88C764FF0A00A02F076FA98F88516AF
:1079C000B8F88C96D8F80070ADF8B75005238DF84C
:1079D000B610ADF8B9908DF8B2A08DF8B53005E0CD
:1079E000D8F80020D11B642900F2B1820B212CA809
:1079F000F9F7EAF80028F3D0C4F30E04002D00F0E4
:107A0000B4824FF000094D4570D84B46DAB28DF87C
:107A1000B5200632D8F800A0D7B25EE07543000862
:107A2000ED4500083D1B0008BD1C0008D11C0008E6
:107A3000E91C0008051D0008091D0008551D000867
:107A4000AD1D0008DD1D0008FD1D00087D1E00089D
:107A50008D1E0008C11E0008F51E0008D94600084A
:107A6000A51F0008CD1F00085D2000088920000820
:107A7000A1200008FD2000080121000805210008C0
:107A800009210008F1230008094700081521000812
:107A9000652100086D210008452200084D220008DC
:107AA000B9220008914A00083D2800080000024061
:107AB0003022012038110120D9490008FD49000871
:107AC00049220008114A000800ED00E0D8F8002023
:107AD000A2EB0A01642900F2998639462CA8F9F72D
:107AE00073F80028F2D04D4540F23F822CAA0023C3
:107AF0009F4F023337F81400D071013414F4004F53
:107B00009BB209F10107A4B24FEA102118BF00246B
:107B1000802B1FFA87F9917103F102073FF476AFCA
:107B2000601C4D4509F1010E1FFA80FC02F10201B3
:107B30003FF46CAF8E4B10F4004F33F81400C87153
:107B40004FEA10231FFA8EF98B7108BF6446BBB24F
:107B500018BF00244D4503F1020001F1020709F1AD
:107B6000010A3FF453AF824931F81410F97101341E
:107B700014F4004F1FFA8AF9A4B24FEA112118BF7A
:107B80000024B97183B2671C4D4503F1020009F16D
:107B900001011FFA87FE3FF439AF754B17F4004F10
:107BA00033F8147057731FFA81F90CBF7446002420
:107BB000390A83B24D4504F10100117303F1020744
:107BC00009F101011FFA80FC3FF420AF684B10F46B
:107BD000004F33F81400D0731FFA81F90CBF6446CC
:107BE0000024010ABBB2601C4D45917303F10207EA
:107BF00009F101011FFA80FA3FF408AF5C4B10F461
:107C0000004F33F8140050741FFA81F90CBF54462A
:107C10000024010ABBB2601C4D45117402F10C0A2C
:107C200003F1020709F1010E1FFA80FC02F10E02B6
:107C30003FF4ECAE4E4B33F814108AF8071010F4F2
:107C4000004F1FFA8EF94FEA11200CBF6446002442
:107C50004D458AF80600BBB27FF44AAFD6E605F080
:107C6000FF07109788F86C77206C30432064236CF2
:107C700033403A46314610931C20109BF8F7D2FA55
:107C800032463C4E4FF0805535600F97216C41EAEB
:107C90000A072764246C04EA0A000F9009211D20BA
:107CA0000F9BF8F7BFFA4FF00052D8F83407326054
:107CB000FFF706BBFBF730F88346FBF72DF84FF0D4
:107CC000190909FB00F2B2FBF5F6FBF725F882462D
:107CD000FBF722F809FB00F1B1FBF5F7FBF71CF805
:107CE000FFF7D2BB2449189688F8E4600A6B024378
:107CF0000A630C6B04401894189A17960D6B054391
:107D00000D630B6B03401793179A16964F6C47F051
:107D100010024A64496C01F01004CDE92E601694FB
:107D20001648169B2CA907254FF480674FF400795D
:107D30004FF0120B3095CDE92C9AF8F795FBCDE971
:107D40002C7BF8F791FB324625200321F8F76AFADD
:107D50000848D8F8AC4020264660E368D8F8B470EC
:107D6000D8F8B05043F02002E260FFF743BB00BFF9
:107D70004000002000E100E0003802400000024026
:107D800003F5003C159488F8A040DCF830302B4314
:107D9000CCF83030DCF830202A4015921599149434
:107DA000DCF830102943CCF83010DCF830302B40B0
:107DB000149314991394DCF830202A43CCF8302023
:107DC000DCF830102940139113991294DCF830300C
:107DD0002B43CCF83030DCF830202A401292129934
:107DE0001194DCF8401041F48043CCF84030DCF8CA
:107DF00040202C9600F1804E0EF5013002F48041B7
:107E000011912CA9119B2D97CDE92E47F8F72CFB4A
:107E10004FF4806786612C974FF48056F8F724FB67
:107E200087612C96F8F720FB052386612D954FF48A
:107E3000005530932C954FF48047F8F715FB4FF41D
:107E400000422C92F8F710FB2C97F8F70DFB224616
:107E500021462420F8F7E6F95D48D8F85030102480
:107E60004460FFF767BA02F1804C0CF5104E744580
:107E70004FEA450600F0F7850EF58062944200F067
:107E8000F285FAF72FFF8346FAF72CFF4FF0190916
:107E900009FB00F7FAF726FFB7FBF6F78246FAF779
:107EA00021FF09FB00F5B5FBF6F5FAF71BFF00F023
:107EB000F0BDD8F8007098F83942202C7FF472ABEE
:107EC000594644483B461922F9F78EFE01460028E0
:107ED0007FF468AB98F83832012B3FF463ABD8F8E5
:107EE000FC5188F838B22A683B4822F400642C60C0
:107EF000D8F8FC514FF0220C88F839C288F83A6261
:107F0000C8F83C12C8F828022E6846F480632B603B
:107F1000D8F8FC01026842F4807404603B465A467B
:107F20004FF00110F9F760FE002841F08985D8F87C
:107F3000FC112A48A0250D613A465946FAF7F2FC91
:107F4000002801F05F85D8F83C3201F079BD244E5D
:107F500008234FF40064402080254FF48057B3611C
:107F6000B461B061B561B761FEE71E4D1E4F2C696B
:107F7000E11B00234810C8F8780688F88636C8F850
:107F8000883688F8853698F8CD29002A4CD098F89C
:107F9000CF4998F8CC09D8F8C879631CDDB2511ED6
:107FA000A84298BF002588F8CF5988F8CD1957F80E
:107FB000244094F805E0D4F886C0A644CEF806C064
:107FC000B4F88A20D8F80050AEF80A2014E000BFB8
:107FD00000E100E0020010000000FFFF02000100CD
:107FE000000002400000002040000020D8F80020DF
:107FF000511B642900F2DD8161790C312046C9B240
:10800000F8F7E2FD0028F1D098F83007092806D8E3
:1080100008EB80090130C9F8084788F8300798F85C
:10802000CD49002C00F05F8598F8D079002F40F002
:108030009B8498F80527002A40F06B8598F88016F5
:1080400000293FF488ACBE4F4FF480224FF48030BB
:108050004FF40035BD610024BA61B86188F862440C
:10806000FAF7ECFC72B6B74BB749596062B64FF4F9
:108070000005BD6198F8637488F8634498F8E520BA
:10808000212AFBD0AE48B14C4FF480124FF40023AC
:108090004FF480014FF08055836181618561826179
:1080A0004FF400002CA920604FF0000AA8480423D8
:1080B0004FF0030940248025CDE92C493093CDE9C8
:1080C0002EAAF8F7D1F92C95A24DF8F7CDF92A6C24
:1080D00022F400132B644FF40074CDE92D9ACDF8EF
:1080E000BCA02C94F8F7C0F94FF480622C92F8F7FA
:1080F000BBF94FF480532C934FF00509F8F7B4F90E
:108100004FF400522C92CDF8C090F8F7ADF94FF42F
:1081100000432C93F8F7A8F94FF480422C92F8F71B
:10812000A3F9696C4FF0E02221F480506864136970
:1081300023F00201116194FAA4F0B0FA80F303F184
:10814000845101F5603083008349012018600B6879
:1081500023F00303034381480B60016941F00403EA
:10816000036130BF016921F00403036194FAA4F4B0
:10817000B4FA84F000F1845101F560339C00C4F836
:1081800000A0106940F002011161CDF874A02A6CC2
:1081900042F080532B642C6C0F2104F080501D9012
:1081A0002C911D9B2A686B4C530356BF2B684B4682
:1081B000C3F300432D93206800F001012F91236841
:1081C000F82595FAA5FABAFA8AF203F0F805D5402F
:1081D0003095206F450758BF206F5E4C54BF00F0AC
:1081E000010005202E90636F03F001023192256893
:1081F00015F0807F0CBF012502253295606800F4E0
:1082000080033393626802F03F053495606847F657
:10821000C07191FAA1F30840B3FA83F1C8403590D8
:1082200065684FF4403999FAA9FA05F4403202F52D
:108230008030BAFA8AF14300CB40369365684FF03C
:10824000706999FAA9FABAFA8AF205F07060D0401A
:10825000379061684FF0E04393FAA3F5B5FA85F2E1
:1082600001F0E040D04001254FF0020938902CA8E1
:10827000CDE92C55CDF8C890FAF78AFE0F21209150
:10828000A36803F003022192A06800F0F00122919C
:10829000A36803F4E0522392A068314AC10801F4B4
:1082A000E05324931068209500F00F0120A8CDF82A
:1082B0008490FAF74BFD254925484FF40003C1F897
:1082C0008030402212214FF0000ACDE925210423FD
:1082D00025A92993CDE927AAF8F7C6F88022259287
:1082E0002895F8F7C1F8CDF87CA0206C40F4001177
:1082F0002164236C03F400121F921F9BFAF7AEFF58
:10830000CDF878A0606C40F480516164646C1048D2
:10831000269504F4805325A91E934FF400741E9BE8
:108320002594CDE927AAF8F79FF884614FF480647B
:108330002594F8F799F884614FF4805412E000BF57
:1083400000000240000000203519000800E100E0B4
:1083500000040240003802400070004000ED00E0E0
:10836000003C02402594F8F77FF8846105234FF420
:1083700000524FF4004425922993CDF89890F8F7D5
:1083800073F82594F8F770F8D64C4FF48042259294
:10839000F8F76AF81020A06172B6FBF7D3FB8021D2
:1083A000002F40F0B083002788F8807662B6FFF790
:1083B000D2BACC4E08234FF40067402080244FF4FB
:1083C0008055B361B761B061B461B561FEE7C64D78
:1083D00069692F8E95F81FA004970029BCBF01F58D
:1083E0007F513F318C1303944FF00009D8F870246B
:1083F000D8F8740482423FF4BAAA2CA8F9F74CFBCF
:1084000000283FF4B4AA98F8403FD8F86C54B6F866
:10841000E440019563B103F1FF3E0EEB8E0108EBE2
:10842000810CDCF8A47CEA1BB2F5806F00F2D082EC
:10843000D8F8487FAD483D46BA1CC8F8482F35F8F3
:1084400004EBC8F8485F7F88BDF9B02000EB041149
:1084500017FB02F51EFB02FC45F38F3EB1F90250FB
:10846000A1F802E02701AEEB050EA04D4CF38F30D2
:1084700035F907C0E853A0EB0C05D8F8580FD8F829
:108480004C7FB1F904C02844D8F85C5FC8F8580F95
:108490000EEB0500C8F85C0FBD1C3846C8F84C5FF1
:1084A00030F804EBC8F84C0F7F881EFB02F017FB76
:1084B00002F540F38F37B1F906008F8045F38F3511
:1084C000CD802D1AD8F8600FA7EB0C0E7044C8F8B9
:1084D000600FD8F8640FD8F8507F0544C8F8645F7F
:1084E0003846BD1CC8F8505F30F804CBC8F8500FB0
:1084F0007F881CFB02F017FB02FEB1F908C006934F
:1085000040F38F37B1F90A000F814EF38F354D815B
:108510002D1AD8F8680FA7EB0C0E7044C8F8680F36
:10852000D8F86C0FD8F8547F0544C8F86C5F38460B
:10853000BD1CC8F8545F30F804CBC8F8540F7F88CE
:108540001CFB02FE17FB02F04EF38F35684F40F321
:108550008F3E82FB0220920B42EA804207EB8407A7
:10856000B1F90C008D812D1AB1F90E00A1F80EE0C1
:10857000D7F8D819C7F8D829571AD8F8702F154442
:10858000C8F8705FD8F8745FAEEB00002844C8F8F4
:10859000740FD6F8E000074407F58071C6F8E07064
:1085A0005F1C05919C46029719460CE0D7F8A01C69
:1085B0000131C7F8A01C029F0CF101051FFA85FCD0
:1085C0006745614651DB0CF0010308EB031E01EB2C
:1085D0008102DEF85C5FDEF8583FDEF8600F08EBE2
:1085E0008207DEF8642F85FB055EAD0B45EA8E45FC
:1085F00083FB033E9B0B43EA8E4E754482FB022EA7
:10860000930B43EA8E4380FB000E820B42EA8E40BE
:1086100003441D44059B95FBF3F0D7F8985CA842F2
:108620005FFA8CF34FEA8102C0DD15B9019DC7F8EE
:10863000A85C0A4408EB82070299C7F8980C01333A
:10864000DBB20198C7F8A40C994287F89C9CC7F844
:10865000A09CB0DB03EB830E013308EB8E02DBB290
:108660009942C2F8989CF5DAA5E7069B039D03EBB7
:10867000830008EB800EDEF8982C954240F3D480FE
:108680000134C4F30804A6F8E440002C7FF4AEAE35
:10869000184F98F8445F98F845CF17483D44BC44BC
:1086A00095F8103795F812279CF814779CF816C7A0
:1086B00000EB830100EB820E00EB8C0300EB8702E2
:1086C000D1F80048DEF80058D2F80008D3F80018B6
:1086D000C8F8484FC8F84C5FC8F8500FC8F8541F86
:1086E00084E600BF00000240000000205424012066
:1086F0003811012090090108A0E70008D8F844606B
:10870000B64926F4885424F0020040F00202C8F86A
:1087100044204D6825F440374F604E68D8F8084033
:1087200026434E60596821F4807058605A68D8F822
:10873000145042EA05275F605E6826F040745C6072
:108740005868D8F80C10A64C084358609A6822F470
:1087500000659D609F68D8F8106037439F609968F6
:10876000D8F82C0021F070629A60A0429D6800F059
:108770005E82D8F82C6035439D609C6824F04050A0
:1087800098609A68D8F830100A439A609D6825F07E
:1087900002079F609E68D8F81C4046EA4400986033
:1087A000D8F82420002A40F02C82596821F4006572
:1087B0005D60DC6AD8F8200024F47002DA62DD6AB9
:1087C00000F1FF3A45EA0A51D9629F6827F4007622
:1087D0009E609C68D8F8340044EA40229A609D6804
:1087E00025F4806199609F68D8F81860002047EAF6
:1087F00086249C60C8F84800D8F8442022F003057D
:1088000045F00101C8F84410FEF79DBE754E0825DD
:108810004FF40064402080234FF48057B561B46169
:10882000B061B361B761FEE7DEF8A02C04986E4931
:108830006E4FC8F8C0188242C8F8B8780BD2002B27
:108840003FF41EAFD8F8A42C019D5902AA1A80311A
:108850008A427FF615AF13F0010C654F654914BFCE
:1088600004224FF4802208EB0C0EBA619EF8445F9C
:108870000135EAB201EB8C00022AD0F8F87708BF84
:1088800000228EF8442FB85C01EB800E0134DEF834
:10889000001808EBCC00C4F308053A4401EB850747
:1088A000C0F8487F9278534901EB820E524ADEF8B5
:1088B0000078524907EB8505C0F84C5F02EBCC0706
:1088C0000FFA8CF001EBCC05C7E90099C7E90499D0
:1088D000C7E90899C7E90C99C7E91099C7E914993C
:1088E000C7E91899C7E91C998037BD42ECD1444FBC
:1088F00007EB001C00011F2B47F80090CCE9019901
:10890000CCF80C9006D808EB4303B3F8B02601323C
:10891000A3F8B0269DF8083088F8403F142101FBE9
:10892000038E5345CEF8A09CFFF4ABAE0020D8F8E0
:10893000A42C3449864602E0CC68A51AAE44013026
:108940005FFA80F94B4501F11401F5D8BEFBF3FA4B
:1089500001332D4F02EB032454440225C6F8E840AE
:1089600087F8D459FFF703B8D8F89436002788F869
:10897000D0798BB1D8F85042D8F85022101B9842C9
:108980000AD222490D6925F004070F6130BFD8F8DB
:108990005022101B8342F5D81D48FDF799F8144B5F
:1089A00080249C61FFF74ABB4FF4006201F6D810A7
:1089B000294601F079FA2846C6F8E050FDF706F896
:1089C0001148012780F8D479FBF7BCF8FEF7CFBF38
:1089D0002046FCF7FBFF98F8403F29E500230140C3
:1089E0000100000F00000240DB1B0400B9A20100DF
:1089F00000080240A0E7000854240120544401204C
:108A0000980F0120D80C01203811012000ED00E062
:108A1000140A012003F58C3BC8F8487088F84070B0
:108A20001A97DBF8443043F48076CBF84460DBF8E7
:108A300044102C9501F480740320CDE92D071A947D
:108A4000AB481A9A2F952CA9F7F70EFD3A46092143
:108A50001220F7F7E7FBA74AD8F804304FF4802537
:108A60001560FEF76BBDFAF757F98346FAF754F92C
:108A70004FF0190909FB00F1B1FBF6F7FAF74CF9D1
:108A80008246FAF749F909FB00F3B3FBF6F5FAF76A
:108A900043F9642109FB0AFC09FB00F0BCFBF6F278
:108AA00009FB0BFEB2FBF1F3B0FBF6FB01FB137706
:108AB000BBFBF1F901FB1955E800FA003230323204
:108AC000B0FBF1F5B2FBF1F705F0070A7B0003F408
:108AD000F87CBEFBF6F6B6FBF1F60AEB0611614434
:108AE000A160FEF7F8BC98F88136012B7FF49CAAB0
:108AF00004F1804A0AF502354FF0006788F8824693
:108B0000AF61FFF791BAA16188F86354FAF7D6FF15
:108B100049E498F8070798F80447431CDDB2511E52
:108B2000AC4298BF0025D8F8002788F8051788F8C8
:108B3000075752F8204094F90210A07800292EDB44
:108B4000394695220DF1B30001F0AEF9FF2798F8F0
:108B50007F068DF8B2708DF8B00094F801908DF812
:108B6000B19094F804A0D8F800708DF8B4A005E096
:108B7000D8F80010C81B642800F2EB8706212CA847
:108B8000F8F722F80028F3D098F87F365A4D237072
:108B90002046FCF79DFF8022AA6100F0BEBF574B24
:108BA00080F0800103EB8109D9F8A855002D00F071
:108BB000B2872046A847002800F0D9873946982276
:108BC0002CA801F071F9A0788DF8B200D9F8A87737
:108BD0000DF1B600B847D8F800508DF8B50005E0A3
:108BE000D8F800305F1B642F00F2A5879DF8B520F0
:108BF00006322CA8D1B2F7F7E7FF0028F0D000F03A
:108C00008CBF5F6847F400645C60586820F4604281
:108C10004FF460465A6096FAA6F9D8F828705D6855
:108C2000B9FA89F17E1E8E402E435E60C1E525F0C3
:108C300040579F60AAE5D8F87024D8F874349A4257
:108C400002D02CA8F8F728FFD6F8E840D8F86C74C2
:108C5000BC427EF48CAEB8F89A0698F8855627493F
:108C6000254B01304FF0000E4FF40002022DA8F802
:108C70009A0681F8D4E99A6100F0FE82204D1E4BDD
:108C8000EA7F1F4895F81E900221996145690132DB
:108C9000B9EB020448BF0334002DB8BF05F57F557A
:108CA0004FEAA407B8BF3F35FCB2164A2092A91379
:108CB000FF2C059100F0D482134B144F4FF00009A4
:108CC000A64601254FF0000A20A80395CDF818907C
:108CD00004905546F146CDE925730023CDE92C33A8
:108CE000CDE92E33C6F8E0304FF4007417E000BF32
:108CF0000004024000E100E00008024038110120B9
:108D0000000000200100000198D7000898B7000873
:108D1000DBF8100020F00403CBF8103030BFD8F897
:108D20007074D8F8742497420DF12A00F0D0F8F747
:108D3000B3FE0028ECD02598BDF92A302C9ADDF836
:108D400098C00746013C37F804EB25971EFB03F15A
:108D500041F38F318A182C924088019210FB03FE58
:108D60002D9A4EF38F3160468A182D9230F804EB1D
:108D70002E9902921EFB03F242F38F320A442E9286
:108D8000BCF802E0269083FB031C2F981EFB03F324
:108D90008F0BD6F8E01047EA8C4E43F38F337144C3
:108DA0000344A4B2C6F8E0102F93002CB7D18C4630
:108DB0000CF5807E82FB022CDDE90110970B47EA5F
:108DC0008C4783FB033C9A0B42EA8C4381FB0121D5
:108DD0001F44930B80FB002043EA814C910B41EA36
:108DE0008043039A05989C44674497FBFEF7B8427A
:108DF000C8BF00220392BAF1000F1BD14FF0010A45
:108E000004990DF183048C421FD00C46734814F86A
:108E1000012F049400EB820EDEF8F83759195F5DDC
:108E20008C7800EB870C00EB8402DCF80078D2F839
:108E3000003850E70135EDB2012D22D904992546BD
:108E4000A2460DF183048C42DFD1039DDDF818A00A
:108E5000CE46C5B9F2450AF1010900F001825F4F23
:108E60009DF880C007EB8C03D3F8F807027884786C
:108E700007EB820107EB840AD1F80078DAF80038B2
:108E80001FE7A246BCE7B8F89C565FFA8AF00135A6
:108E90000628A8F89C5606D808EB4A0EBEF8F0261D
:108EA0000132AEF8F026D8F85042D8F87014D8F84D
:108EB00074744B4827444B4C7B1A4FF40035C6F86A
:108EC000EC30A561824698220021806B00F0ECFF17
:108ED0004FF489720021444800F0E6FF4FF48017F8
:108EE000414ACAF83C204FF400214FF400134FF4DC
:108EF00080054FF40000A161A761A361A561A06195
:108F00003A49D8F86C249AF81870C6F8F020032370
:108F1000002488F8833F002200234FF0FF0A4FF01F
:108F20000409022521F8604CC8F8844FC8F8884F1E
:108F3000C8F87C4F88F8814F41E91A2388F87B7F75
:108F400088F880AF88F88C9F88F8825FFDF714FC62
:108F50001B24FDF711FC601E84B2FDF70DFC611EA1
:108F60008FB2FDF709FC7A1E1FFA82FAFDF704FCA6
:108F70000AF1FF331FFA83F909F1FF35ACB2FDF7AF
:108F8000FBFBFDF7F9FB601E87B2FDF7F5FB791ED1
:108F90001FFA81FAFDF7F0FB0AF1FF321FFA82F99E
:108FA000FDF7EAFB09F1FF339CB2002CD1D10D4D46
:108FB0000D4920200822A861A646CDE90144CDE94B
:108FC0000444A44627462546204603940794099462
:108FD00008924FF0800A069496E000BFA0E70008D0
:108FE0000000002000080240B00A012038110120D2
:108FF000079A4B784FEA420A039AC3F3801949EA69
:1090000042039AB291F9013003924AEAD37293B2C1
:10901000079301312022059B91F800A05B0012EA22
:109020000A0F18BF43F001039BB25208059340F0AA
:109030009B80049A4B784FEA4209029AC3F3801A44
:109040004AEA42039AB291F90130029249EAD37294
:1090500093B2049301312022019B91F800905B00B0
:1090600012EA090F18BF43F001039BB25FEA520AEC
:10907000019340F09D8091F8019091F9012040000A
:10908000C9F3801A40EAD2734AEA440498B2A4B2FF
:10909000013120230A786D00134218BF45F0010505
:1090A0005B08ADB240F09F804B7891F901A07F0042
:1090B000C3F3801949EA4C0C47EADA721FFA8CFCB8
:1090C00097B2013120234FEA4E0291F800E013EAF3
:1090D0000E0F18BF42F001025FEA530A1FFA82FE28
:1090E00040F09E80069B91F901905B0043EAD972A3
:1090F00093B2069301314FF0400A089A531E13F0C1
:10910000FF02089200F04A81099B91F800905B00F1
:1091100019EA0A0F18BF43F001039BB209935FEAF3
:109120005A033FF465AF13EA090F079B4FEA430365
:1091300018BF43F001039BB207935FEA9A0340F024
:10914000A880039A4B784FEA420A059AC3F3801924
:1091500049EA42039AB291F9013005924AEAD37280
:1091600093B2039301312022049B91F800905B009D
:1091700012EA090F18BF43F001039BB2520804938F
:1091800040F0AA80029B91F801A04FEA4309019B9D
:10919000CAF3801242EA430A91F901301FFA8AF2B7
:1091A000019249EAD37293B2029301314FF0200A3F
:1091B0000A7840001AEA020F18BF40F001005FEA87
:1091C0005A0380B240F0A78091F8019091F90120F4
:1091D0006400C9F3801A44EAD2734AEA45059CB296
:1091E000ADB2013120230A787F00134218BF47F047
:1091F00001075B08BFB240F0A7804FEA4C0391F82B
:1092000001C091F901A0CCF3801943EADA7249EA6E
:109210004E0E1FFA8EFE1FFA82FC01314FF0200A1B
:10922000069B5A000B781AEA030F18BF42F001029E
:1092300092B25FEA5A0A069204BF01314FF0800AE7
:109240005BE7B8F8A40652490130A8F8A4064B69B8
:1092500083F0800747F400048C614D4D0222AA611F
:109260004B4F4C494C48C8F8B8184FF40033C8F875
:10927000C008BB61FEF77BBB98F88646002C7FF4E4
:10928000FDACD8F87876C8F88876012088F886068C
:10929000F4E413EA090F039B4FEA430318BF43F0BA
:1092A00001039BB25FEADA0203937FF4B4AE059B3D
:1092B00091F801904FEA430A049BC9F3801242EAF5
:1092C000430991F901301FFA89F204924AEAD372F4
:1092D00093B2059301312022029B91F800A05B001C
:1092E00012EA0A0F18BF43F001039BB2520802931F
:1092F0007FF4B2AE019B91F9012091F801905B00DF
:1093000043EAD273C9F3801A9AB24AEA400080B2A3
:109310000192013120230A786400134218BF44F0FF
:1093200001045B08A4B27FF4B5AE91F8019091F905
:1093300001206D00C9F3801A45EAD2734AEA470753
:109340009DB2BFB2013120234FEA4C0291F800C018
:1093500013EA0C0F18BF42F001025B081FFA82FCEF
:109360007FF4B1AE91F80190069AC9F3801A4AEAE7
:1093700042039AB291F9013006924FEA4E0E4EEA3C
:10938000D3721FFA82FE01314FF0200AB5E600BF0A
:1093900000080240B9A20100DB1B04000699079AED
:1093A000ADF8A2000198039BADF8AE10ADF8A8701F
:1093B000ADF8A650059F049DADF8A440ADF8A000FF
:1093C000029C0998ADF896202CA90DF12A02ADF85F
:1093D0009E40ADF89A70BB4CADF8ACE0ADF8AAC0B9
:1093E000ADF89C50ADF89830ADF894000DF19607AB
:1093F000F9F7E8F800283FF424AFBDF82A5095B1FA
:10940000B149B8F8A2C68A6B92F888A05CFA85FECA
:10941000AA44A8F8A2E682F888A0636983F0400015
:1094200040F48005A5610DF1B205BDF896000DF17F
:109430002A0229460237F9F7C5F800283FF401AFA0
:10944000BDF82A2092B1A049B8F8A296886B90F88E
:1094500088E059FA82FC9644A8F8A2C680F888E011
:10946000636983F0400242F48001A161023537F85C
:10947000020B0DF12A022946F9F7A4F800283FF45F
:10948000E0AEBDF82A0090B18F4BB8F8A2169A6BE7
:1094900092F8889051FA80FA8144A8F8A2A682F83E
:1094A0008890606980F0400C4CF48003A361023521
:1094B00038880DF12A022946F9F784F800283FF48C
:1094C000C0AEBDF82A2092B17F49B8F8A2E6886BF9
:1094D00090F888905EFA82FA9144A8F8A2A680F8E3
:1094E0008890636983F0400242F48001A16178882A
:1094F0000DF12A02A91CF9F765F800283FF4A1AE86
:10950000BDF82A0090B1704BB8F8A2169A6B92F889
:1095100088E051FA80FC8644A8F8A2C682F888E068
:10952000606980F0400A4AF48003A361B8880DF1B5
:109530002A02291D0637F9F745F800283FF481AEC5
:10954000BDF82A2092B16049B8F8A296886B90F8CD
:1095500088E059FA82FC9644A8F8A2C680F888E010
:10956000636983F0400242F48001A1612CA8B842F3
:1095700005F106057FF47BAF002220920DF1AE04C9
:10958000CDF8832010460DF1800A05E01FFA89F21C
:109590000435A8B238283CD06588A71CC5F3C004A0
:1095A00044EA4202C5F3800949EA420CC5F340038C
:1095B00043EA4C0105F00105420745EA4104B2F1D6
:1095C000004F0FFA84FE20D01FFA8EF1B7F80290F8
:1095D000BC1CC9F3C00747EA4103C9F3800C04303F
:1095E0004CEA4302C9F3400109F0010785B241EAA0
:1095F000420E400747EA4E03B0F1004F0FFA83F9DD
:10960000C4D10AF8019B0022C2E70AF801EB00214D
:10961000DCE7089D0DF17F0A05E00DF18600610091
:109620008245CDB245D01AF8014F6C4061B2002995
:10963000BABF4C0084F097046400E7B27BB2002B01
:10964000BABF5F0087F097077F00FAB255B2002DCE
:10965000BABF6A0082F097025200D0B244B2002C26
:10966000BABF600080F097004000C7B279B200290D
:10967000BABF4F0087F097077F00FBB25AB2002AAB
:10968000BABF530083F097035B00DDB268B20028D5
:10969000BABF450085F097056D00ECB267B2002FA8
:1096A000BBDA7B000DF1860083F097028245D5B2CC
:1096B000B9D1089555B1B8F8A0260132A8F8A0266E
:1096C000CBE500BF0008024000000020C94CCA4A98
:1096D000A76B209BBDF88450BD804FF400103B6009
:1096E00090617979002900F07D810C298CBF0222DC
:1096F00001221144CC00BF4F7A6B92F800C092F85F
:1097000001E06444631E93FBFCF51EFB05F0703022
:1097100081B2B1F5096F3FF6A0AD98F88C7FCC19F6
:10972000621E92FBF7F9A9F11C039CB2002C41D0F8
:10973000651E05F007070125FDF71EF8A54239D281
:1097400038B21FB301281BD0022816D0032811D02D
:1097500004280CD0052807D0062802D0FDF70CF805
:109760000225FDF709F80135FDF706F80135FDF78B
:1097700003F80135FDF700F80135FCF7FDFF013571
:109780000135FCF7F9FFA9B2A14213D20835FCF765
:10979000F3FFFCF7F1FFFCF7EFFFFCF7EDFFFCF741
:1097A000EBFFFCF7E9FFFCF7E7FFFCF7E5FFAAB2E8
:1097B000A242EBD3FBF75EFA00283FF44EADD8F897
:1097C0006C44D6F8F03098F88C5FD8F8881FD8F839
:1097D000840F884FE21A2B46F8F770FDBC6B84F8B3
:1097E0008600864830F860AC0023524650E91A01E2
:1097F000FDF7E6FA002903460A46C0F2F780B0F109
:10980000004F71F100014FF0010E0DDB990841EAA4
:109810008273B3F1004F4FEAA2024FEA4E0772F192
:1098200000015FFA87FEF1DA900340EA93404FEAC5
:1098300083394FF0804100239B0843EA81739945A7
:109840004FEAA10170EB0102F6DB53EA010226D0D8
:10985000CDE902541A4600231F46D5184FEA920458
:1098600041EB070CA945019470EB0C0409DBB9EB43
:10987000050960EB0C00921841EB0105D31845EB8C
:109880000707019A42EA817289105C0852EA0105D1
:1098900044EAC7734FEA6707DFD1DDE902548EFB64
:1098A00003ECA5FB0E20C821A2FB013705FB0C0928
:1098B0006FF4FF7001FB0972834272F1FF31C0F255
:1098C0009380002A04DA40F2FF115B1842F1000293
:1098D0005F0A47EAC25E1EF500504FEA622141F17D
:1098E000000C830B43EA8C42424F98F87B9FB87F71
:1098F000D8F87C3FFF2A28BFFF2284F88720D6F8BB
:10990000EC20C4F88C200430A2EB402109FB0AF7BC
:1099100005FB03F3B3FBF7F0637998F881AFC4F864
:10992000901098F8801F84F8890084F88A1084F8D1
:109930008BA03BB10C2B8CBF4FF0020A4FF0010AF9
:109940005344DB002B4FD7F834E09EF800109EF80C
:1099500001700B4403F1FF3C9CFBF1FA274907FB24
:109960000AF3681E7033D1F8A87909FB0300B0FB35
:10997000F5F502EB4522C4F8942057B12046204C5F
:10998000636983F0080545F40022A261B8471949CC
:109990008863B8F89E0698F88546174F01304FF453
:1099A0000023A8F89E064FF48015BB614FF4001207
:1099B0004FF480014FF400000223032CBD61BA6113
:1099C000B961B861BB617FF44BAC98F88676002F23
:1099D0007FF446ACD8F87846C8F88846012588F860
:1099E00086563DE4089C86E600227DE74FF0FF3E68
:1099F000F44656E70000002000080240381101201C
:109A000000000240D8F8FC611C9073691C93B26995
:109A10001C9238461C9BF8F71DF938B9D8F8FC4160
:109A200020613846F8F716F9014688B1D8F83C129B
:109A3000042905D1D8F8FC01036843F400750560DA
:109A40000026D8F83C22634C88F83862FDF7ABBD9D
:109A5000D8F8FC01056845F4807606603B465A4616
:109A60004FF00110F8F7C0F80028E9D1D8F8FC3120
:109A70005948A1221A6159463A46F8F753FF00287F
:109A80007EF461AAD8F8FC4100211B9165691B9501
:109A9000A6691B9638461B9BF8F70EFF0146002867
:109AA00040F09180D8F8FC010369426988F87C365F
:109AB00012F0040E62D00469484888F87D463B469F
:109AC0000122474CF8F790F8002854D1D8F8FC71DF
:109AD000396841F400703860D8F8FC311D69257090
:109AE0001E69667098F87C2600242027FF2A88F8D3
:109AF000397288F8384288F83A42364C7DF453ADD2
:109B000001212046F8F722F8B8F87D9681457DF4CA
:109B10004AADFDF754BDFAF789FF98F830170929C7
:109B20003EF68CAA08EB810E0131CEF8084788F882
:109B30003017FEF783BA2B4E08244FF40062402002
:109B400080214FF48055B461B261B061B161B561FB
:109B5000FEE7244E08234FF40065402480274FF48D
:109B60008052B361B561B461B761B261FEE7A078BC
:109B7000FAF75CFFD1E70134FDF715BD17481A4C21
:109B800071463B460122F8F72FF800BB3B46D8F858
:109B9000FC7112483D6825F480663E60D8F8FC21CF
:109BA000176927700122F8F71FF880B9D8F8FC115F
:109BB000086840F400730B60D8F8FC512E69667099
:109BC0002A69A2708EE7D8F83C32FDF7EBBC02346C
:109BD000FDF7E9BCBF0601200200010004000100FE
:109BE000BE06012000000240BD0601202DE9F0471D
:109BF000089D0E4604460F46002B4AD194468C45DC
:109C0000B2FA82F260D942B1C2F12003974020FA41
:109C100003F30CFA02FC1F4394404FEA1C4E1FFA58
:109C20008CF6B7FBFEF1230C0EFB117743EA0743DA
:109C300001FB06F098420AD91CEB030301F1FF3740
:109C400080F01581984240F21281023963441B1A58
:109C5000A4B2B3FBFEF00EFB103344EA034400FB56
:109C600006F6A6420AD91CEB040400F1FF3380F08B
:109C70000081A64240F2FD806444023840EA01407F
:109C8000A41B00211DB1D4400023C5E90043BDE859
:109C9000F0878B4205D90DB1C5E9000100210846C6
:109CA000F5E7B3FA83F1002946D1B34202D38242E9
:109CB00000F2F580841A66EB030201201746002D9E
:109CC000E5D0C5E90047E2E7002A40F09380A1EB28
:109CD0000C034FEA1C471FFA8CFE0121B3FBF7F679
:109CE00007FB1630230C43EA00430EFB06F09842B4
:109CF00008D91CEB030306F1FF3802D2984200F2A8
:109D0000D08046461B1AA4B2B3FBF7F007FB103312
:109D100044EA03440EFB00FEA64508D91CEB0404EC
:109D200000F1FF3302D2A64500F2B6801846A4EB3C
:109D30000E0440EA0640A5E7C1F120078B4022FA55
:109D400007FC4CEA030C06FA01FE20FA07F426FA97
:109D500007F344EA0E0400FA01F84FEA1C404FEA08
:109D60001449B3FBF0FE1FFA8CF600FB1E3349EAE0
:109D700003430EFB06F9994502FA01F20BD91CEBDD
:109D800003030EF1FF3A80F08580994540F282800E
:109D9000AEF1020E6344A3EB0909A4B2B9FBF0F3E0
:109DA00000FB139944EA094403FB06F6A64208D9CE
:109DB0001CEB040403F1FF3068D2A64266D9023BD3
:109DC000644443EA0E40A41BA0FB02E6B44273467F
:109DD000B14652D34FD05DB1B8EB030264EB090436
:109DE00004FA07F722FA01F31F43CC40C5E90074D7
:109DF00000214CE7C2F1200120FA01F30CFA02FC29
:109E000026FA01F1964033434FEA1C471FFA8CFEB5
:109E1000B1FBF7F007FB1016190C41EA064100FBF5
:109E20000EF68E4204FA02F408D91CEB010100F18F
:109E3000FF382DD28E422BD902386144891B9BB248
:109E4000B1FBF7F607FB161143EA014306FB0EF1DF
:109E5000994208D91CEB030306F1FF3814D299424A
:109E600012D9023E63445B1A46EA004136E739469E
:109E7000EDE6184602E7F045ADD2BEEB020366EB15
:109E80000C060138B146A6E74646ECE7034698E7DC
:109E90004046D3E7D6467EE76444023847E70846A3
:109EA0000DE7023E63442DE7830730B547D0541ECB
:109EB000002A3ED0CAB2034601E0013C39D303F880
:109EC000012B9D07F9D1032C2CD9CDB205EB05252B
:109ED0000F2C05EB054535D9A4F1100222F00F0C2B
:109EE00003F1100EE6444FEA121C1A46C2E900556F
:109EF000C2E9025510327245F8D10CF1010214F09A
:109F00000C0F03EB021204F00F0C13D0ACF104039E
:109F100023F003030433134442F8045B9342FBD160
:109F20000CF003042CB1C9B21C4403F8011BA3427A
:109F3000FBD130BD64461346002CF4D1F9E703464B
:109F40001446C0E71A46A446E0E700BF40EA010312
:109F50009B0710B501D1032A17D8844601F1FF3EB3
:109F600007E01EF8011F03F8011B541E29B19C468F
:109F700022466346002AF4D110BD9444002CFBD045
:109F800003F8011B6345FBD110BD8E468446DEF805
:109F90000040A4F1013323EA040313F0803F71462B
:109FA0000EF1040EDAD1043A032A4CF8044BEED831
:049FB0007146D3E73C
:109FB40008B5F6F723F900BF024A136801331360AA
:109FC400704700BF4000012080B5094B094A98B092
:109FD4001968914200AF13D1074D084E1D6086F3F6
:109FE4000888A3F5303CDCF80440A047FEE700BF36
:109FF40000C00120AD700DB0EFBEADDEF82A002028
:10A00400A54EA64BD6F8884044F47005C6F888508F
:10A014001A68A34C002042F00101196098601D6881
:10A0240025F0847222F4803119605C601D689D4CB7
:10A0340025F480224FF000611A60D860B160B460EA
:10A04400D6F888509848994B45F470049842C6F85D
:10A05400884007D25E1E321A22F003029449043269
:10A06400FCF716FF93489449884207D24D1E2B1AD9
:10A0740023F0030204320021FFF714FF8F4E8648B9
:10A0840034688F4A44F400713160356845F4806364
:10A094003360316841F480753560C668894D4FF688
:10A0A400FF0426403243C2602C684FF47A78B4FB34
:10A0B400F8FC0CF1FF33B3F1807F0CD24FF0E02EAB
:10A0C400F022CEF81430072180F823200020CEF8A7
:10A0D4001800CEF81010704EF468C4F30223C3F1D4
:10A0E4000700042803F1040228BF04204FF0FF31C5
:10A0F400062A01FA00F18CBFDA1E0022CE439640F4
:10A1040033016548654C0026DAB280F823203E61AD
:10A11400216C6D4841F080532364226C02F080511D
:10A1240039613A69FE60036843F4404202600068A2
:10A13400664B00F44041F9600122F968DA640122B7
:10A144000123C7E90A234FF4B47310214FF48000AC
:10A15400FB6402220723C7E91423C7E91101022281
:10A1640007F128003A64F8F711FF0F200221C7E92C
:10A17400061678614FF4A0584FF48056052107F174
:10A184001400C7E90886F8F7DFFDA36803F00C02A2
:10A19400082A00F0EF804E4E404B4E4C98684E4AD1
:10A1A400C0F3031E744494F818174C4CCE402E6030
:10A1B400151BAE10002D7E604BDD701E54F8043B61
:10A1C40000F0070698477A680125AA4241DD3EB3AC
:10A1D400012E1ED0022E18D0032E12D0042E0CD025
:10A1E400052E06D0062E40F0DA8054F8040B804782
:10A1F400013554F8043B9847013554F8046BB047D3
:10A20400013554F8042B9047013554F8041B884752
:10A21400013554F8040B80477B680135AB4218DDE7
:10A22400A046083558F8046BB04762689047D8F8E0
:10A2340004108847E0688047236998476669B047F7
:10A24400A2699047E16988477868A84204F120042C
:10A25400E6DC234C234D631B002B4FEAA30640F39B
:10A264008780721E55F8041B02F0070488470120FA
:10A27400864280467CDD002C5CD0012C52D0022C1E
:10A284004AD0032C42D0042C3AD0052C32D0062CD0
:10A2940040F08A8028E000BF00ED00E00038024072
:10A2A40010300024000000080000002040000120BD
:10A2B4002CFA02084000012054440120003C0240D2
:10A2C4000003FA050000002000700040000047422F
:10A2D4000024F400900901082CFA02082CFA020860
:10A2E4002CFA02082CFA020855F8042B9047414630
:10A2F4000131884655F8044BA0474046013080465A
:10A3040055F8043B984742460132904655F8041BE1
:10A31400444688470134A04655F8040B8047434619
:10A324000133984655F8042B9047414601318E423B
:10A3340088461DDD2C46203554F8040B804755F81B
:10A344001C3C98476268904755F8141C884755F898
:10A35400104CA04755F80C0C804755F8083C98471A
:10A3640055F8042C9047414608318E428846E1DC7A
:10A37400FCF7B0FE63680F4E606864680E4900F035
:10A384003F0C7068B1FBFCF2C4F38813C0F30144C2
:10A39400013402FB03F36100B3FBF1F6FCE654F86D
:10A3A400041B8847022520E755F8043B98474FF0E3
:0CA3B400020899E7003802400024F40081
:10A3C0000100010101020103010401050106010769
:10A3D00001080109010A010B010C010D010E010F19
:10A3E00001100111011200800000000004080000AB
:10A3F00051240008C52500080B1000003525000871
:10A40000992600080D000B00080007000400020058
:10A4100001000E00D506B30500048F030002000101
:10A4200080007F00400020001000080004000200AF
:10A4300001006907AA0066001E00FF00AAAA66665E
:10A440001E1EFE01FFFF000000061016000610167B
:10A4500000000000010203040102030406070809CA
:10A46000AAAA0000055085ABC5D8E5EEF5FAFD00B7
:10A4700000402C37D72F7428A622981ED41A9F1874
:10A480003F168A1435133C12C0116811FC10CA1013
:10A490005710F70FBC0FA80F920F670F740F200F04
:10A4A000CC0E470EDD0D590DAD0C2D0C800BC90ADD
:10A4B000140A5509B2083D08EE07D107B907C307CA
:10A4C000B907C007AE0789076907B6079F070B08DA
:10A4D00009080040CB377F30CB2ADB26CF22412032
:10A4E000E21D231C001B901A631B9B1C6B1D291E65
:10A4F000C61D1C1BD117CC145A129610720FEB0EEE
:10A50000E20E8D0FDB10741255138814BE159416CD
:10A5100047150011FE0DD50B1D0AF2081A086A072F
:10A520000507DD06DB06FB06F8064D07B0074C08FD
:10A530000709A0090040DA3C403AB3391237263601
:10A5400041359730812AB52681244A24BB24A2258F
:10A550002324E820F21D6A1BFC18641600141F1245
:10A560001010200E4C0C9B0A48096908AE070E0714
:10A57000890621067505A3042204F203CA03910388
:10A5800066033E031503EF02D102B7029F028D025C
:10A590007B02620256020040BC3B15380735583238
:10A5A000CC2F772D4C2B4C296A27A425F623632228
:10A5B000F3209C1F4F1E0B1DCB1B921A60194318D2
:10A5C00033172F1636154E147513A212DB112211F4
:10A5D0008110FB0F800F780EDA0D630DEA0C5F0C13
:10A5E000D50B4B0BC80A4F0AE10979091609BA08BD
:10A5F00062081208CB078907C83E603A233C953FA2
:10A6000000409536012C2924F71D6518D3141C131E
:10A610004413CF14BE158A17C617B3161115441369
:10A62000A6110A10790E130D860B380A11091B08A2
:10A63000E9079C074507E80686068206AB06E7069B
:10A64000250757077C073A07BC064606A50584057B
:10A650009505CC056D069E063607E90C9C0BE60AAF
:10A660003C0A9109BC08FB0744079606E405470528
:10A67000C3045204F703A603640333030D03EA0281
:10A68000CD02B402A00294028F029602A802C70271
:10A69000F0022E037503CE033704B1044005EE0526
:10A6A000C806CE070209510ADF0BB30DFC0F1013C9
:10A6B0003017851C3B23B42B1735004080AB0008B6
:10A6C00064F40008B8F40208B8F00208B8EC020814
:10A6D000B8E80208B8E40208B8E00208B8DC0208EA
:10A6E000B8D80208B8D40208B8D00208B8CC02081A
:10A6F000B8C8020864F80008B8C40208B8C0020864
:10A70000B8BC0208B8B8020864FC0008B8B4020873
:10A71000B8B00208B8AC0208B8A80208B8A4020889
:10A72000B8A00208B89C0208B8980208B8940208B9
:10A73000B8900208B88C0208B888020864F00008D3
:10A74000B8840208B8800208B87C0208B878020809
:10A75000B8740208B8700208B86C0208B868020839
:10A76000B8640208B8600208B85C0208B858020869
:10A77000B8540208B8500208B84C0208B848020899
:10A780000000640994125D1B8E23FA2A7931E536A4
:10A79000203B143EB13FEC3FC53E423C713867332D
:10A7A000412D1F262B1E8F157C0C2303BBF974F043
:10A7B00083E719DF67D795D0CACA26C6C2C2B2C01E
:10A7C00000C0B2C0C2C226C6CACA95D067D719DFB8
:10A7D00083E774F0BBF923037C0C8F152B1E1F2617
:10A7E000412D67337138423CC53EEC3FB13F143ECA
:10A7F000203BE5367931FA2A8E235D1B94126409D9
:10A8000000009CF66CEDA3E472DC06D587CE1BC974
:10A81000E0C4ECC14FC014C03BC1BEC38FC799CCCC
:10A82000BFD2E1D9D5E171EA84F3DDFC45068C0F96
:10A830007D18E72099286B2F3635DA393E3D4E3F9B
:10A8400000404E3F3E3DDA3936356B2F9928E720E0
:10A850007D188C0F4506DDFC84F371EAD5E1E1D962
:10A86000BFD299CC8FC7BEC33BC114C04FC0ECC18F
:10A87000E0C41BC987CE06D572DCA3E46CED9CF660
:10A880000000640994125D1B8E23FA2A7931E536A3
:10A89000203B143EB13FEC3FC53E423C713867332C
:10A8A000412D1F262B1E8F157C0C2303BBF974F042
:10A8B00083E719DF67D795D0CACA26C6C2C2B2C01D
:10A8C00000C0B2C0C2C226C6CACA95D067D719DFB7
:10A8D00083E774F0BBF923037C0C8F152B1E1F2616
:10A8E000412D67337138423CC53EEC3FB13F143EC9
:10A8F000203BE5367931FA2A8E235D1B94126409D8
:10A9000000009CF66CEDA3E472DC06D587CE1BC973
:10A91000E0C4ECC14FC014C03BC1BEC38FC799CCCB
:10A92000BFD2E1D9D5E171EA84F3DDFC45068C0F95
:10A930007D18E72099286B2F3635DA393E3D4E3F9A
:10A9400000404E3F3E3DDA3936356B2F9928E720DF
:10A950007D188C0F4506DDFC84F371EAD5E1E1D961
:10A96000BFD299CC8FC7BEC33BC114C04FC0ECC18E
:10A97000E0C41BC987CE06D572DCA3E46CED9CF65F
:10A980000000640994125D1B8E23FA2A7931E536A2
:10A99000203B143EB13FEC3FC53E423C713867332B
:10A9A000412D1F262B1E8F157C0C2303BBF974F041
:10A9B00083E719DF67D795D0CACA26C6C2C2B2C01C
:10A9C00000C0B2C0C2C226C6CACA95D067D719DFB6
:10A9D00083E774F0BBF923037C0C8F152B1E1F2615
:10A9E000412D67337138423CC53EEC3FB13F143EC8
:10A9F000203BE5367931FA2A8E235D1B94126409D7
:10AA000000009CF66CEDA3E472DC06D587CE1BC972
:10AA1000E0C4ECC14FC014C03BC1BEC38FC799CCCA
:10AA2000BFD2E1D9D5E171EA84F3DDFC45068C0F94
:10AA30007D18E72099286B2F3635DA393E3D4E3F99
:10AA400000404E3F3E3DDA3936356B2F9928E720DE
:10AA50007D188C0F4506DDFC84F371EAD5E1E1D960
:10AA6000BFD299CC8FC7BEC33BC114C04FC0ECC18D
:10AA7000E0C41BC987CE06D572DCA3E46CED9CF65E
:10AA80000000640994125D1B8E23FA2A7931E536A1
:10AA9000203B143EB13FEC3FC53E423C713867332A
:10AAA000412D1F262B1E8F157C0C2303BBF974F040
:10AAB00083E719DF67D795D0CACA26C6C2C2B2C01B
:10AAC00000C0B2C0C2C226C6CACA95D067D719DFB5
:10AAD00083E774F0BBF923037C0C8F152B1E1F2614
:10AAE000412D67337138423CC53EEC3FB13F143EC7
:10AAF000203BE5367931FA2A8E235D1B94126409D6
:10AB000000009CF66CEDA3E472DC06D587CE1BC971
:10AB1000E0C4ECC14FC014C03BC1BEC38FC799CCC9
:10AB2000BFD2E1D9D5E171EA84F3DDFC45068C0F93
:10AB30007D18E72099286B2F3635DA393E3D4E3F98
:10AB400000404E3F3E3DDA3936356B2F9928E720DD
:10AB50007D188C0F4506DDFC84F371EAD5E1E1D95F
:10AB6000BFD299CC8FC7BEC33BC114C04FC0ECC18C
:10AB7000E0C41BC987CE06D572DCA3E46CED9CF65D
:10AB80000000412D0040412D0000BFD200C0BFD2C7
:10AB90000000412D0040412D0000BFD200C0BFD2B7
:10ABA0000000412D0040412D0000BFD200C0BFD2A7
:10ABB0000000412D0040412D0000BFD200C0BFD297
:10ABC0000000412D0040412D0000BFD200C0BFD287
:10ABD0000000412D0040412D0000BFD200C0BFD277
:10ABE0000000412D0040412D0000BFD200C0BFD267
:10ABF0000000412D0040412D0000BFD200C0BFD257
:10AC00000000412D0040412D0000BFD200C0BFD246
:10AC10000000412D0040412D0000BFD200C0BFD236
:10AC20000000412D0040412D0000BFD200C0BFD226
:10AC30000000412D0040412D0000BFD200C0BFD216
:10AC40000000412D0040412D0000BFD200C0BFD206
:10AC50000000412D0040412D0000BFD200C0BFD2F6
:10AC60000000412D0040412D0000BFD200C0BFD2E6
:10AC70000000412D0040412D0000BFD200C0BFD2D6
:10AC80000000412D0040412D0000BFD200C0BFD2C6
:10AC90000000412D0040412D0000BFD200C0BFD2B6
:10ACA0000000412D0040412D0000BFD200C0BFD2A6
:10ACB0000000412D0040412D0000BFD200C0BFD296
:10ACC0000000412D0040412D0000BFD200C0BFD286
:10ACD0000000412D0040412D0000BFD200C0BFD276
:10ACE0000000412D0040412D0000BFD200C0BFD266
:10ACF0000000412D0040412D0000BFD200C0BFD256
:10AD00000000412D0040412D0000BFD200C0BFD245
:10AD10000000412D0040412D0000BFD200C0BFD235
:10AD20000000412D0040412D0000BFD200C0BFD225
:10AD30000000412D0040412D0000BFD200C0BFD215
:10AD40000000412D0040412D0000BFD200C0BFD205
:10AD50000000412D0040412D0000BFD200C0BFD2F5
:10AD60000000412D0040412D0000BFD200C0BFD2E5
:10AD70000000412D0040412D0000BFD200C0BFD2D5
:10AD80000000412D0040412D0000BFD200C0BFD2C5
:10AD90000000412D0040412D0000BFD200C0BFD2B5
:10ADA0000000412D0040412D0000BFD200C0BFD2A5
:10ADB0000000412D0040412D0000BFD200C0BFD295
:10ADC0000000412D0040412D0000BFD200C0BFD285
:10ADD0000000412D0040412D0000BFD200C0BFD275
:10ADE0000000412D0040412D0000BFD200C0BFD265
:10ADF0000000412D0040412D0000BFD200C0BFD255
:10AE00000000412D0040412D0000BFD200C0BFD244
:10AE10000000412D0040412D0000BFD200C0BFD234
:10AE20000000412D0040412D0000BFD200C0BFD224
:10AE30000000412D0040412D0000BFD200C0BFD214
:10AE40000000412D0040412D0000BFD200C0BFD204
:10AE50000000412D0040412D0000BFD200C0BFD2F4
:10AE60000000412D0040412D0000BFD200C0BFD2E4
:10AE70000000412D0040412D0000BFD200C0BFD2D4
:10AE80000000412D0040412D0000BFD200C0BFD2C4
:10AE90000000412D0040412D0000BFD200C0BFD2B4
:10AEA0000000412D0040412D0000BFD200C0BFD2A4
:10AEB0000000412D0040412D0000BFD200C0BFD294
:10AEC0000000412D0040412D0000BFD200C0BFD284
:10AED0000000412D0040412D0000BFD200C0BFD274
:10AEE0000000412D0040412D0000BFD200C0BFD264
:10AEF0000000412D0040412D0000BFD200C0BFD254
:10AF00000000412D0040412D0000BFD200C0BFD243
:10AF10000000412D0040412D0000BFD200C0BFD233
:10AF20000000412D0040412D0000BFD200C0BFD223
:10AF30000000412D0040412D0000BFD200C0BFD213
:10AF40000000412D0040412D0000BFD200C0BFD203
:10AF50000000412D0040412D0000BFD200C0BFD2F3
:10AF60000000412D0040412D0000BFD200C0BFD2E3
:10AF70000000412D0040412D0000BFD200C0BFD2D3
:10AF8000E0F90208E4F90208F0F90208F8F9020809
:10AF900004FA020814FA0208000000405A2E212C7C
:10AFA000EC3FDDFCCD298ACFBBF94FC08CCDA1D8B9
:10AFB000B2C0640926DB53347C0CC53E12363D22F8
:10AFC000143E74F08B1F51C86CEDC2C2D6C63AE372
:10AFD000BEC38F1511E6823A7D18203BB63B081799
:10AFE000DA39A3E413143BC3D5E18FC752C2EFEEA5
:10AFF0001BC9E720FBF1713E8E2336350E3FF10A67
:10B000006733E1D9D5077CC067D787CE2DC04BFB0E
:10B0100095D0FA2A6EFEFB3F412D412DFB3F6EFE7F
:10B02000FA2A95D04BFB2DC087CE67D77CC0D507B9
:10B03000E1D96733F10A0E3F36358E23713EFBF1BD
:10B04000E7201BC9EFEE52C28FC7D5E13BC31314F3
:10B05000A3E4DA390817B63B203B7D18823A11E6A3
:10B060008F15BEC33AE3D6C6C2C26CED51C88B1F62
:10B0700074F0143E3D221236C53E7C0C533426DB60
:10B080006409B2C0A1D88CCD4FC0BBF98ACFCD29FD
:10B09000DDFCEC3F212C5A2E00400000212CA6D1D3
:10B0A000DDFC14C08ACF33D64FC04506A1D8743218
:10B0B00064094E3F5334DA24C53E84F33D22EEC981
:10B0C00074F0ECC151C875E0C2C294123AE32A3957
:10B0D0008F15423C823AEF19203B83E708174AC498
:10B0E000A3E426C63BC3EDEB8FC72B1EEFEEAE3DB0
:10B0F000E720E536713E050E363572DCF10AF2C006
:10B10000E1D999CC7CC02BF887CE99284BFBD33F53
:10B11000FA2A6B2FFB3F9201412DBFD26EFE05C074
:10B1200095D006D52DC0B50467D77931D507843FB2
:10B1300067331F260E3F0FF58E23CACAFBF18FC15E
:10B140001BC919DF52C21111D5E171381314C53C66
:10B15000DA395D1BB63BF8E87D18E0C411E67EC520
:10B16000BEC371EAD6C6C61C6CED3E3D8B1FAF3721
:10B17000143E8C0F1236C3DD7C0C3BC126DBADCBFD
:10B18000B2C09CF68CCD5F27BBF9B13FCD2976309C
:10B19000EC3F23035A2EDFD3000000C0A6D1DFD33B
:10B1A00014C0230333D676304506B13F74325F278F
:10B1B0004E3F9CF6DA24ADCB84F33BC1EEC9C3DD30
:10B1C000ECC18C0F75E0AF3794123E3D2A39C61C96
:10B1D000423C71EAEF197EC583E7E0C44AC4F8E84F
:10B1E00026C65D1BEDEBC53C2B1E7138AE3D111123
:10B1F000E53619DF050E8FC172DCCACAF2C00FF541
:10B2000099CC1F262BF8843F99287931D33FB50478
:10B210006B2F06D5920105C0BFD2BFD205C09201E7
:10B2200006D56B2FB504D33F79319928843F2BF88D
:10B230001F2699CC0FF5F2C0CACA72DC8FC1050E69
:10B2400019DFE5361111AE3D71382B1EC53CEDEB13
:10B250005D1B26C6F8E84AC4E0C483E77EC5EF1943
:10B2600071EA423CC61C2A393E3D9412AF3775E064
:10B270008C0FECC1C3DDEEC93BC184F3ADCBDA2446
:10B280009CF64E3F5F277432B13F4506763033D689
:10B29000230314C0DFD3A6D100C00000DFD35A2E91
:10B2A0002303EC3F7630CD29B13FBBF95F278CCD2E
:10B2B0009CF6B2C0ADCB26DB3BC17C0CC3DD1236A5
:10B2C0008C0F143EAF378B1F3E3D6CEDC61CD6C6AF
:10B2D00071EABEC37EC511E6E0C47D18F8E8B63B4E
:10B2E0005D1BDA39C53C13147138D5E1111152C216
:10B2F00019DF1BC98FC1FBF1CACA8E230FF50E3FA0
:10B300001F266733843FD507793167D7B5042DC031
:10B3100006D595D005C06EFEBFD2412D9201FB3FF0
:10B320006B2FFA2AD33F4BFB992887CE2BF87CC092
:10B3300099CCE1D9F2C0F10A72DC3635050E713EC6
:10B34000E536E720AE3DEFEE2B1E8FC7EDEB3BC39E
:10B3500026C6A3E44AC4081783E7203BEF19823AC4
:10B36000423C8F152A393AE39412C2C275E051C8A3
:10B37000ECC174F0EEC93D2284F3C53EDA245334A7
:10B380004E3F64097432A1D845064FC033D68ACFE8
:10B3900014C0DDFCA6D1212C000000405A2E212C27
:10B3A000EC3FDDFCCD298ACFBBF94FC08CCDA1D8B5
:10B3B000B2C0640926DB53347C0CC53E12363D22F4
:10B3C000143E74F08B1F51C86CEDC2C2D6C63AE36E
:10B3D000BEC38F1511E6823A7D18203BB63B081795
:10B3E000DA39A3E413143BC3D5E18FC752C2EFEEA1
:10B3F0001BC9E720FBF1713E8E2336350E3FF10A63
:10B400006733E1D9D5077CC067D787CE2DC04BFB0A
:10B4100095D0FA2A6EFEFB3F412D412DFB3F6EFE7B
:10B42000FA2A95D04BFB2DC087CE67D77CC0D507B5
:10B43000E1D96733F10A0E3F36358E23713EFBF1B9
:10B44000E7201BC9EFEE52C28FC7D5E13BC31314EF
:10B45000A3E4DA390817B63B203B7D18823A11E69F
:10B460008F15BEC33AE3D6C6C2C26CED51C88B1F5E
:10B4700074F0143E3D221236C53E7C0C533426DB5C
:10B480006409B2C0A1D88CCD4FC0BBF98ACFCD29F9
:10B49000DDFCEC3F212C5A2E00400000212CA6D1CF
:10B4A000DDFC14C08ACF33D64FC04506A1D8743214
:10B4B00064094E3F5334DA24C53E84F33D22EEC97D
:10B4C00074F0ECC151C875E0C2C294123AE32A3953
:10B4D0008F15423C823AEF19203B83E708174AC494
:10B4E000A3E426C63BC3EDEB8FC72B1EEFEEAE3DAC
:10B4F000E720E536713E050E363572DCF10AF2C002
:10B50000E1D999CC7CC02BF887CE99284BFBD33F4F
:10B51000FA2A6B2FFB3F9201412DBFD26EFE05C070
:10B5200095D006D52DC0B50467D77931D507843FAE
:10B5300067331F260E3F0FF58E23CACAFBF18FC15A
:10B540001BC919DF52C21111D5E171381314C53C62
:10B55000DA395D1BB63BF8E87D18E0C411E67EC51C
:10B56000BEC371EAD6C6C61C6CED3E3D8B1FAF371D
:10B57000143E8C0F1236C3DD7C0C3BC126DBADCBF9
:10B58000B2C09CF68CCD5F27BBF9B13FCD29763098
:10B59000EC3F23035A2EDFD3000000C0A6D1DFD337
:10B5A00014C0230333D676304506B13F74325F278B
:10B5B0004E3F9CF6DA24ADCB84F33BC1EEC9C3DD2C
:10B5C000ECC18C0F75E0AF3794123E3D2A39C61C92
:10B5D000423C71EAEF197EC583E7E0C44AC4F8E84B
:10B5E00026C65D1BEDEBC53C2B1E7138AE3D11111F
:10B5F000E53619DF050E8FC172DCCACAF2C00FF53D
:10B6000099CC1F262BF8843F99287931D33FB50474
:10B610006B2F06D5920105C0BFD2BFD205C09201E3
:10B6200006D56B2FB504D33F79319928843F2BF889
:10B630001F2699CC0FF5F2C0CACA72DC8FC1050E65
:10B6400019DFE5361111AE3D71382B1EC53CEDEB0F
:10B650005D1B26C6F8E84AC4E0C483E77EC5EF193F
:10B6600071EA423CC61C2A393E3D9412AF3775E060
:10B670008C0FECC1C3DDEEC93BC184F3ADCBDA2442
:10B680009CF64E3F5F277432B13F4506763033D685
:10B69000230314C0DFD3A6D100C00000DFD35A2E8D
:10B6A0002303EC3F7630CD29B13FBBF95F278CCD2A
:10B6B0009CF6B2C0ADCB26DB3BC17C0CC3DD1236A1
:10B6C0008C0F143EAF378B1F3E3D6CEDC61CD6C6AB
:10B6D00071EABEC37EC511E6E0C47D18F8E8B63B4A
:10B6E0005D1BDA39C53C13147138D5E1111152C212
:10B6F00019DF1BC98FC1FBF1CACA8E230FF50E3F9C
:10B700001F266733843FD507793167D7B5042DC02D
:10B7100006D595D005C06EFEBFD2412D9201FB3FEC
:10B720006B2FFA2AD33F4BFB992887CE2BF87CC08E
:10B7300099CCE1D9F2C0F10A72DC3635050E713EC2
:10B74000E536E720AE3DEFEE2B1E8FC7EDEB3BC39A
:10B7500026C6A3E44AC4081783E7203BEF19823AC0
:10B76000423C8F152A393AE39412C2C275E051C89F
:10B77000ECC174F0EEC93D2284F3C53EDA245334A3
:10B780004E3F64097432A1D845064FC033D68ACFE4
:10B7900014C0DDFCA6D1212C00000040DA395D1B6D
:10B7A000793167D774F0ECC13BC184F3E1D96733D9
:10B7B0002B1E7138EC3FDDFC7D18E0C406D595D01A
:10B7C000C2C294129CF64E3F36358E23E53619DF01
:10B7D000BBF94FC0BEC371EABFD2412D8F15423CA9
:10B7E000B13F4506E7201BC972DCCACAB2C0640972
:10B7F0006CED3E3D6B2FFA2A203B83E7230314C0F8
:10B800008FC7D5E199CC1F267C0CC53E143E8C0F0A
:10B81000992887CEA3E426C600C00000A3E4DA3945
:10B8200099287931143E74F07C0C3BC199CCE1D954
:10B830008FC72B1E2303EC3F203B7D186B2F06D5B3
:10B840006CEDC2C2B2C09CF672DC3635E720E5363C
:10B85000B13FBBF98F15BEC3BFD2BFD2BEC38F15D8
:10B86000BBF9B13FE536E720363572DC9CF6B2C055
:10B87000C2C26CED06D56B2F7D18203BEC3F230335
:10B880002B1E8FC7E1D999CC3BC17C0C74F0143EC0
:10B8900079319928DA39A3E4000000C026C6A3E470
:10B8A00087CE99288C0F143EC53E7C0C1F2699CC60
:10B8B000D5E18FC714C0230383E7203BFA2A6B2FFF
:10B8C0003E3D6CED6409B2C0CACA72DC1BC9E720F8
:10B8D0004506B13F423C8F15412DBFD271EABEC330
:10B8E0004FC0BBF919DFE5368E2336354E3F9CF647
:10B8F0009412C2C295D006D5E0C47D18DDFCEC3FA1
:10B9000071382B1E6733E1D984F33BC1ECC174F06D
:10B9100067D779315D1BDA39004000005D1B26C610
:10B9200067D787CEECC18C0F84F3C53E67331F26E3
:10B930007138D5E1DDFC14C0E0C483E795D0FA2A64
:10B9400094123E3D4E3F64098E23CACA19DF1BC9BB
:10B950004FC0450671EA423C412D412D423C71EAFF
:10B9600045064FC01BC919DFCACA8E2364094E3F62
:10B970003E3D9412FA2A95D083E7E0C414C0DDFC62
:10B98000D5E171381F266733C53E84F38C0FECC1B7
:10B9900087CE67D726C65D1B00000040DA395D1BE5
:10B9A000793167D774F0ECC13BC184F3E1D96733D7
:10B9B0002B1E7138EC3FDDFC7D18E0C406D595D018
:10B9C000C2C294129CF64E3F36358E23E53619DFFF
:10B9D000BBF94FC0BEC371EABFD2412D8F15423CA7
:10B9E000B13F4506E7201BC972DCCACAB2C0640970
:10B9F0006CED3E3D6B2FFA2A203B83E7230314C0F6
:10BA00008FC7D5E199CC1F267C0CC53E143E8C0F08
:10BA1000992887CEA3E426C600C00000A3E4DA3943
:10BA200099287931143E74F07C0C3BC199CCE1D952
:10BA30008FC72B1E2303EC3F203B7D186B2F06D5B1
:10BA40006CEDC2C2B2C09CF672DC3635E720E5363A
:10BA5000B13FBBF98F15BEC3BFD2BFD2BEC38F15D6
:10BA6000BBF9B13FE536E720363572DC9CF6B2C053
:10BA7000C2C26CED06D56B2F7D18203BEC3F230333
:10BA80002B1E8FC7E1D999CC3BC17C0C74F0143EBE
:10BA900079319928DA39A3E4000000C026C6A3E46E
:10BAA00087CE99288C0F143EC53E7C0C1F2699CC5E
:10BAB000D5E18FC714C0230383E7203BFA2A6B2FFD
:10BAC0003E3D6CED6409B2C0CACA72DC1BC9E720F6
:10BAD0004506B13F423C8F15412DBFD271EABEC32E
:10BAE0004FC0BBF919DFE5368E2336354E3F9CF645
:10BAF0009412C2C295D006D5E0C47D18DDFCEC3F9F
:10BB000071382B1E6733E1D984F33BC1ECC174F06B
:10BB100067D779315D1BDA39004000005D1B26C60E
:10BB200067D787CEECC18C0F84F3C53E67331F26E1
:10BB30007138D5E1DDFC14C0E0C483E795D0FA2A62
:10BB400094123E3D4E3F64098E23CACA19DF1BC9B9
:10BB50004FC0450671EA423C412D412D423C71EAFD
:10BB600045064FC01BC919DFCACA8E2364094E3F60
:10BB70003E3D9412FA2A95D083E7E0C414C0DDFC60
:10BB8000D5E171381F266733C53E84F38C0FECC1B5
:10BB900087CE67D726C65D1B00000040DA395D1BE3
:10BBA000793167D774F0ECC13BC184F3E1D96733D5
:10BBB0002B1E7138EC3FDDFC7D18E0C406D595D016
:10BBC000C2C294129CF64E3F36358E23E53619DFFD
:10BBD000BBF94FC0BEC371EABFD2412D8F15423CA5
:10BBE000B13F4506E7201BC972DCCACAB2C064096E
:10BBF0006CED3E3D6B2FFA2A203B83E7230314C0F4
:10BC00008FC7D5E199CC1F267C0CC53E143E8C0F06
:10BC1000992887CEA3E426C600C00000A3E4DA3941
:10BC200099287931143E74F07C0C3BC199CCE1D950
:10BC30008FC72B1E2303EC3F203B7D186B2F06D5AF
:10BC40006CEDC2C2B2C09CF672DC3635E720E53638
:10BC5000B13FBBF98F15BEC3BFD2BFD2BEC38F15D4
:10BC6000BBF9B13FE536E720363572DC9CF6B2C051
:10BC7000C2C26CED06D56B2F7D18203BEC3F230331
:10BC80002B1E8FC7E1D999CC3BC17C0C74F0143EBC
:10BC900079319928DA39A3E4000000C026C6A3E46C
:10BCA00087CE99288C0F143EC53E7C0C1F2699CC5C
:10BCB000D5E18FC714C0230383E7203BFA2A6B2FFB
:10BCC0003E3D6CED6409B2C0CACA72DC1BC9E720F4
:10BCD0004506B13F423C8F15412DBFD271EABEC32C
:10BCE0004FC0BBF919DFE5368E2336354E3F9CF643
:10BCF0009412C2C295D006D5E0C47D18DDFCEC3F9D
:10BD000071382B1E6733E1D984F33BC1ECC174F069
:10BD100067D779315D1BDA39004000005D1B26C60C
:10BD200067D787CEECC18C0F84F3C53E67331F26DF
:10BD30007138D5E1DDFC14C0E0C483E795D0FA2A60
:10BD400094123E3D4E3F64098E23CACA19DF1BC9B7
:10BD50004FC0450671EA423C412D412D423C71EAFB
:10BD600045064FC01BC919DFCACA8E2364094E3F5E
:10BD70003E3D9412FA2A95D083E7E0C414C0DDFC5E
:10BD8000D5E171381F266733C53E84F38C0FECC1B3
:10BD900087CE67D726C65D1B00000040DA395D1BE1
:10BDA000793167D774F0ECC13BC184F3E1D96733D3
:10BDB0002B1E7138EC3FDDFC7D18E0C406D595D014
:10BDC000C2C294129CF64E3F36358E23E53619DFFB
:10BDD000BBF94FC0BEC371EABFD2412D8F15423CA3
:10BDE000B13F4506E7201BC972DCCACAB2C064096C
:10BDF0006CED3E3D6B2FFA2A203B83E7230314C0F2
:10BE00008FC7D5E199CC1F267C0CC53E143E8C0F04
:10BE1000992887CEA3E426C600C00000A3E4DA393F
:10BE200099287931143E74F07C0C3BC199CCE1D94E
:10BE30008FC72B1E2303EC3F203B7D186B2F06D5AD
:10BE40006CEDC2C2B2C09CF672DC3635E720E53636
:10BE5000B13FBBF98F15BEC3BFD2BFD2BEC38F15D2
:10BE6000BBF9B13FE536E720363572DC9CF6B2C04F
:10BE7000C2C26CED06D56B2F7D18203BEC3F23032F
:10BE80002B1E8FC7E1D999CC3BC17C0C74F0143EBA
:10BE900079319928DA39A3E4000000C026C6A3E46A
:10BEA00087CE99288C0F143EC53E7C0C1F2699CC5A
:10BEB000D5E18FC714C0230383E7203BFA2A6B2FF9
:10BEC0003E3D6CED6409B2C0CACA72DC1BC9E720F2
:10BED0004506B13F423C8F15412DBFD271EABEC32A
:10BEE0004FC0BBF919DFE5368E2336354E3F9CF641
:10BEF0009412C2C295D006D5E0C47D18DDFCEC3F9B
:10BF000071382B1E6733E1D984F33BC1ECC174F067
:10BF100067D779315D1BDA39004000005D1B26C60A
:10BF200067D787CEECC18C0F84F3C53E67331F26DD
:10BF30007138D5E1DDFC14C0E0C483E795D0FA2A5E
:10BF400094123E3D4E3F64098E23CACA19DF1BC9B5
:10BF50004FC0450671EA423C412D412D423C71EAF9
:10BF600045064FC01BC919DFCACA8E2364094E3F5C
:10BF70003E3D9412FA2A95D083E7E0C414C0DDFC5C
:10BF8000D5E171381F266733C53E84F38C0FECC1B1
:10BF900087CE67D726C65D1B0000004079319928FF
:10BFA000C53E84F32B1E8FC783E7E0C4C2C26CED8D
:10BFB000CACA8E23BBF9B13F412D412DB13FBBF918
:10BFC0008E23CACA6CEDC2C2E0C483E78FC72B1EA2
:10BFD00084F3C53E9928793100400000992887CE26
:10BFE00084F33BC18FC7D5E1E0C47D186CED3E3DC5
:10BFF0008E233635B13F4506412DBFD2BBF94FC028
:10C00000CACA72DCC2C2941283E7203B2B1E71386D
:10C01000C53E7C0C793167D7000000C087CE67D75A
:10C020003BC17C0CD5E171387D18203B3E3D94121C
:10C03000363572DC45064FC0BFD2BFD24FC0450671
:10C0400072DC363594123E3D203B7D187138D5E1C7
:10C050007C0C3BC167D787CE00C0000067D7793121
:10C060007C0CC53E71382B1E203B83E79412C2C264
:10C0700072DCCACA4FC0BBF9BFD2412D4506B13FE1
:10C0800036358E233E3D6CED7D18E0C4D5E18FC77B
:10C090003BC184F387CE992800000040793199286C
:10C0A000C53E84F32B1E8FC783E7E0C4C2C26CED8C
:10C0B000CACA8E23BBF9B13F412D412DB13FBBF917
:10C0C0008E23CACA6CEDC2C2E0C483E78FC72B1EA1
:10C0D00084F3C53E9928793100400000992887CE25
:10C0E00084F33BC18FC7D5E1E0C47D186CED3E3DC4
:10C0F0008E233635B13F4506412DBFD2BBF94FC027
:10C10000CACA72DCC2C2941283E7203B2B1E71386C
:10C11000C53E7C0C793167D7000000C087CE67D759
:10C120003BC17C0CD5E171387D18203B3E3D94121B
:10C13000363572DC45064FC0BFD2BFD24FC0450670
:10C1400072DC363594123E3D203B7D187138D5E1C6
:10C150007C0C3BC167D787CE00C0000067D7793120
:10C160007C0CC53E71382B1E203B83E79412C2C263
:10C1700072DCCACA4FC0BBF9BFD2412D4506B13FE0
:10C1800036358E233E3D6CED7D18E0C4D5E18FC77A
:10C190003BC184F387CE992800000040793199286B
:10C1A000C53E84F32B1E8FC783E7E0C4C2C26CED8B
:10C1B000CACA8E23BBF9B13F412D412DB13FBBF916
:10C1C0008E23CACA6CEDC2C2E0C483E78FC72B1EA0
:10C1D00084F3C53E9928793100400000992887CE24
:10C1E00084F33BC18FC7D5E1E0C47D186CED3E3DC3
:10C1F0008E233635B13F4506412DBFD2BBF94FC026
:10C20000CACA72DCC2C2941283E7203B2B1E71386B
:10C21000C53E7C0C793167D7000000C087CE67D758
:10C220003BC17C0CD5E171387D18203B3E3D94121A
:10C23000363572DC45064FC0BFD2BFD24FC045066F
:10C2400072DC363594123E3D203B7D187138D5E1C5
:10C250007C0C3BC167D787CE00C0000067D779311F
:10C260007C0CC53E71382B1E203B83E79412C2C262
:10C2700072DCCACA4FC0BBF9BFD2412D4506B13FDF
:10C2800036358E233E3D6CED7D18E0C4D5E18FC779
:10C290003BC184F387CE992800000040793199286A
:10C2A000C53E84F32B1E8FC783E7E0C4C2C26CED8A
:10C2B000CACA8E23BBF9B13F412D412DB13FBBF915
:10C2C0008E23CACA6CEDC2C2E0C483E78FC72B1E9F
:10C2D00084F3C53E9928793100400000992887CE23
:10C2E00084F33BC18FC7D5E1E0C47D186CED3E3DC2
:10C2F0008E233635B13F4506412DBFD2BBF94FC025
:10C30000CACA72DCC2C2941283E7203B2B1E71386A
:10C31000C53E7C0C793167D7000000C087CE67D757
:10C320003BC17C0CD5E171387D18203B3E3D941219
:10C33000363572DC45064FC0BFD2BFD24FC045066E
:10C3400072DC363594123E3D203B7D187138D5E1C4
:10C350007C0C3BC167D787CE00C0000067D779311E
:10C360007C0CC53E71382B1E203B83E79412C2C261
:10C3700072DCCACA4FC0BBF9BFD2412D4506B13FDE
:10C3800036358E233E3D6CED7D18E0C4D5E18FC778
:10C390003BC184F387CE9928000000407931992869
:10C3A000C53E84F32B1E8FC783E7E0C4C2C26CED89
:10C3B000CACA8E23BBF9B13F412D412DB13FBBF914
:10C3C0008E23CACA6CEDC2C2E0C483E78FC72B1E9E
:10C3D00084F3C53E9928793100400000992887CE22
:10C3E00084F33BC18FC7D5E1E0C47D186CED3E3DC1
:10C3F0008E233635B13F4506412DBFD2BBF94FC024
:10C40000CACA72DCC2C2941283E7203B2B1E713869
:10C41000C53E7C0C793167D7000000C087CE67D756
:10C420003BC17C0CD5E171387D18203B3E3D941218
:10C43000363572DC45064FC0BFD2BFD24FC045066D
:10C4400072DC363594123E3D203B7D187138D5E1C3
:10C450007C0C3BC167D787CE00C0000067D779311D
:10C460007C0CC53E71382B1E203B83E79412C2C260
:10C4700072DCCACA4FC0BBF9BFD2412D4506B13FDD
:10C4800036358E233E3D6CED7D18E0C4D5E18FC777
:10C490003BC184F387CE9928000000407931992868
:10C4A000C53E84F32B1E8FC783E7E0C4C2C26CED88
:10C4B000CACA8E23BBF9B13F412D412DB13FBBF913
:10C4C0008E23CACA6CEDC2C2E0C483E78FC72B1E9D
:10C4D00084F3C53E9928793100400000992887CE21
:10C4E00084F33BC18FC7D5E1E0C47D186CED3E3DC0
:10C4F0008E233635B13F4506412DBFD2BBF94FC023
:10C50000CACA72DCC2C2941283E7203B2B1E713868
:10C51000C53E7C0C793167D7000000C087CE67D755
:10C520003BC17C0CD5E171387D18203B3E3D941217
:10C53000363572DC45064FC0BFD2BFD24FC045066C
:10C5400072DC363594123E3D203B7D187138D5E1C2
:10C550007C0C3BC167D787CE00C0000067D779311C
:10C560007C0CC53E71382B1E203B83E79412C2C25F
:10C5700072DCCACA4FC0BBF9BFD2412D4506B13FDC
:10C5800036358E233E3D6CED7D18E0C4D5E18FC776
:10C590003BC184F387CE9928000000407931992867
:10C5A000C53E84F32B1E8FC783E7E0C4C2C26CED87
:10C5B000CACA8E23BBF9B13F412D412DB13FBBF912
:10C5C0008E23CACA6CEDC2C2E0C483E78FC72B1E9C
:10C5D00084F3C53E9928793100400000992887CE20
:10C5E00084F33BC18FC7D5E1E0C47D186CED3E3DBF
:10C5F0008E233635B13F4506412DBFD2BBF94FC022
:10C60000CACA72DCC2C2941283E7203B2B1E713867
:10C61000C53E7C0C793167D7000000C087CE67D754
:10C620003BC17C0CD5E171387D18203B3E3D941216
:10C63000363572DC45064FC0BFD2BFD24FC045066B
:10C6400072DC363594123E3D203B7D187138D5E1C1
:10C650007C0C3BC167D787CE00C0000067D779311B
:10C660007C0CC53E71382B1E203B83E79412C2C25E
:10C6700072DCCACA4FC0BBF9BFD2412D4506B13FDB
:10C6800036358E233E3D6CED7D18E0C4D5E18FC775
:10C690003BC184F387CE9928000000407931992866
:10C6A000C53E84F32B1E8FC783E7E0C4C2C26CED86
:10C6B000CACA8E23BBF9B13F412D412DB13FBBF911
:10C6C0008E23CACA6CEDC2C2E0C483E78FC72B1E9B
:10C6D00084F3C53E9928793100400000992887CE1F
:10C6E00084F33BC18FC7D5E1E0C47D186CED3E3DBE
:10C6F0008E233635B13F4506412DBFD2BBF94FC021
:10C70000CACA72DCC2C2941283E7203B2B1E713866
:10C71000C53E7C0C793167D7000000C087CE67D753
:10C720003BC17C0CD5E171387D18203B3E3D941215
:10C73000363572DC45064FC0BFD2BFD24FC045066A
:10C7400072DC363594123E3D203B7D187138D5E1C0
:10C750007C0C3BC167D787CE00C0000067D779311A
:10C760007C0CC53E71382B1E203B83E79412C2C25D
:10C7700072DCCACA4FC0BBF9BFD2412D4506B13FDA
:10C7800036358E233E3D6CED7D18E0C4D5E18FC774
:10C790003BC184F387CE99280000004012363D2229
:10C7A000DA39A3E4D5077CC087CE67D73BC313141F
:10C7B00074F0143E212C5A2EC53E84F308174AC447
:10C7C000E1D999CC2DC0B504D5E171388B1FAF37B5
:10C7D000EC3F2303DA24ADCB83E7E0C4F2C00FF5CE
:10C7E00006D56B2F1111AE3D3E3D9412763033D6F7
:10C7F0009CF6B2C07EC511E6CACA8E239201FB3FE9
:10C80000E536E7202A393AE345064FC08CCDA1D85A
:10C81000BEC38F15FBF1713E412D412D713EFBF1E1
:10C820008F15BEC3A1D88CCD4FC045063AE32A3937
:10C83000E720E536FB3F92018E23CACA11E67EC58A
:10C84000B2C09CF633D6763094123E3DAE3D111107
:10C850006B2F06D50FF5F2C0E0C483E7ADCBDA2429
:10C860002303EC3FAF378B1F7138D5E1B5042DC0E2
:10C8700099CCE1D94AC4081784F3C53E5A2E212C1D
:10C88000143E74F013143BC367D787CE7CC0D50722
:10C89000A3E4DA393D221236004000003D22EEC901
:10C8A000A3E426C67CC02BF867D779311314C53CA6
:10C8B000143E8C0F5A2EDFD384F33BC14AC4F8E8F0
:10C8C00099CC1F26B504D33F71382B1EAF3775E0C6
:10C8D000230314C0ADCB26DBE0C47D180FF50E3F5B
:10C8E0006B2FFA2AAE3DEFEE9412C2C233D68ACF36
:10C8F000B2C0640911E6823A8E233635FB3F6EFEE4
:10C90000E7201BC93AE3D6C64FC0BBF9A1D87432A1
:10C910008F15423C713E050E412DBFD2FBF18FC1F8
:10C92000BEC371EA8CCD5F274506B13F2A39C61CCC
:10C93000E53619DF920105C0CACA72DC7EC5EF195F
:10C940009CF64E3F7630CD293E3D6CED111152C222
:10C9500006D595D0F2C0F10A83E7203BDA245334A0
:10C96000EC3FDDFC8B1F51C8D5E18FC72DC04BFBC1
:10C97000E1D967330817B63BC53E7C0C212CA6D104
:10C9800074F0ECC13BC3EDEB87CE9928D507843F0B
:10C99000DA395D1B1236C3DD000000C0EEC9C3DD0D
:10C9A00026C65D1B2BF8843F79319928C53CEDEBF9
:10C9B0008C0FECC1DFD3A6D13BC17C0CF8E8B63BB1
:10C9C0001F266733D33F4BFB2B1E8FC775E051C823
:10C9D00014C0DDFC26DB53347D18203B0E3FF10AEA
:10C9E000FA2A95D0EFEE52C2C2C26CED8ACFCD29A1
:10C9F00064094E3F823AEF19363572DC6EFE05C08F
:10CA00001BC919DFD6C6C61CBBF9B13F74325F27FC
:10CA1000423C71EA050E8FC1BFD2BFD28FC1050E55
:10CA200071EA423C5F277432B13FBBF9C61CD6C6DF
:10CA300019DF1BC905C06EFE72DC3635EF19823A6C
:10CA40004E3F6409CD298ACF6CEDC2C252C2EFEECF
:10CA500095D0FA2AF10A0E3F203B7D18533426DB8D
:10CA6000DDFC14C051C875E08FC72B1E4BFBD33FB4
:10CA700067331F26B63BF8E87C0C3BC1A6D1DFD359
:10CA8000ECC18C0FEDEBC53C99287931843F2BF834
:10CA90005D1B26C6C3DDEEC900C00000C3DD123633
:10CAA0005D1BDA39843FD507992887CEEDEB3BC370
:10CAB000ECC174F0A6D1212C7C0CC53EB63B081706
:10CAC0006733E1D94BFB2DC08FC7D5E151C88B1F10
:10CAD000DDFCEC3F5334DA24203B83E7F10AF2C05B
:10CAE00095D006D552C211116CED3E3DCD29763060
:10CAF0004E3F9CF6EF197EC572DCCACA05C0920192
:10CB000019DFE536C61C2A39B13F45065F278CCDB3
:10CB100071EABEC38FC1FBF1BFD2412D050E713E3C
:10CB2000423C8F157432A1D8BBF94FC0D6C63AE348
:10CB30001BC9E7206EFEFB3F36358E23823A11E695
:10CB40006409B2C08ACF33D6C2C29412EFEEAE3DB2
:10CB5000FA2A6B2F0E3F0FF57D18E0C426DBADCB14
:10CB600014C0230375E0AF372B1E7138D33FB504D3
:10CB70001F2699CCF8E84AC43BC184F3DFD35A2E70
:10CB80008C0F143EC53C1314793167D72BF87CC049
:10CB900026C6A3E4EEC93D220000004012363D2225
:10CBA000DA39A3E4D5077CC087CE67D73BC313141B
:10CBB00074F0143E212C5A2EC53E84F308174AC443
:10CBC000E1D999CC2DC0B504D5E171388B1FAF37B1
:10CBD000EC3F2303DA24ADCB83E7E0C4F2C00FF5CA
:10CBE00006D56B2F1111AE3D3E3D9412763033D6F3
:10CBF0009CF6B2C07EC511E6CACA8E239201FB3FE5
:10CC0000E536E7202A393AE345064FC08CCDA1D856
:10CC1000BEC38F15FBF1713E412D412D713EFBF1DD
:10CC20008F15BEC3A1D88CCD4FC045063AE32A3933
:10CC3000E720E536FB3F92018E23CACA11E67EC586
:10CC4000B2C09CF633D6763094123E3DAE3D111103
:10CC50006B2F06D50FF5F2C0E0C483E7ADCBDA2425
:10CC60002303EC3FAF378B1F7138D5E1B5042DC0DE
:10CC700099CCE1D94AC4081784F3C53E5A2E212C19
:10CC8000143E74F013143BC367D787CE7CC0D5071E
:10CC9000A3E4DA393D221236004000003D22EEC9FD
:10CCA000A3E426C67CC02BF867D779311314C53CA2
:10CCB000143E8C0F5A2EDFD384F33BC14AC4F8E8EC
:10CCC00099CC1F26B504D33F71382B1EAF3775E0C2
:10CCD000230314C0ADCB26DBE0C47D180FF50E3F57
:10CCE0006B2FFA2AAE3DEFEE9412C2C233D68ACF32
:10CCF000B2C0640911E6823A8E233635FB3F6EFEE0
:10CD0000E7201BC93AE3D6C64FC0BBF9A1D874329D
:10CD10008F15423C713E050E412DBFD2FBF18FC1F4
:10CD2000BEC371EA8CCD5F274506B13F2A39C61CC8
:10CD3000E53619DF920105C0CACA72DC7EC5EF195B
:10CD40009CF64E3F7630CD293E3D6CED111152C21E
:10CD500006D595D0F2C0F10A83E7203BDA2453349C
:10CD6000EC3FDDFC8B1F51C8D5E18FC72DC04BFBBD
:10CD7000E1D967330817B63BC53E7C0C212CA6D100
:10CD800074F0ECC13BC3EDEB87CE9928D507843F07
:10CD9000DA395D1B1236C3DD000000C0EEC9C3DD09
:10CDA00026C65D1B2BF8843F79319928C53CEDEBF5
:10CDB0008C0FECC1DFD3A6D13BC17C0CF8E8B63BAD
:10CDC0001F266733D33F4BFB2B1E8FC775E051C81F
:10CDD00014C0DDFC26DB53347D18203B0E3FF10AE6
:10CDE000FA2A95D0EFEE52C2C2C26CED8ACFCD299D
:10CDF00064094E3F823AEF19363572DC6EFE05C08B
:10CE00001BC919DFD6C6C61CBBF9B13F74325F27F8
:10CE1000423C71EA050E8FC1BFD2BFD28FC1050E51
:10CE200071EA423C5F277432B13FBBF9C61CD6C6DB
:10CE300019DF1BC905C06EFE72DC3635EF19823A68
:10CE40004E3F6409CD298ACF6CEDC2C252C2EFEECB
:10CE500095D0FA2AF10A0E3F203B7D18533426DB89
:10CE6000DDFC14C051C875E08FC72B1E4BFBD33FB0
:10CE700067331F26B63BF8E87C0C3BC1A6D1DFD355
:10CE8000ECC18C0FEDEBC53C99287931843F2BF830
:10CE90005D1B26C6C3DDEEC900C00000C3DD12362F
:10CEA0005D1BDA39843FD507992887CEEDEB3BC36C
:10CEB000ECC174F0A6D1212C7C0CC53EB63B081702
:10CEC0006733E1D94BFB2DC08FC7D5E151C88B1F0C
:10CED000DDFCEC3F5334DA24203B83E7F10AF2C057
:10CEE00095D006D552C211116CED3E3DCD2976305C
:10CEF0004E3F9CF6EF197EC572DCCACA05C092018E
:10CF000019DFE536C61C2A39B13F45065F278CCDAF
:10CF100071EABEC38FC1FBF1BFD2412D050E713E38
:10CF2000423C8F157432A1D8BBF94FC0D6C63AE344
:10CF30001BC9E7206EFEFB3F36358E23823A11E691
:10CF40006409B2C08ACF33D6C2C29412EFEEAE3DAE
:10CF5000FA2A6B2F0E3F0FF57D18E0C426DBADCB10
:10CF600014C0230375E0AF372B1E7138D33FB504CF
:10CF70001F2699CCF8E84AC43BC184F3DFD35A2E6C
:10CF80008C0F143EC53C1314793167D72BF87CC045
:10CF900026C6A3E4EEC93D22000000400040000088
:10CFA000000000C000C00000000000400040000081
:10CFB000000000C000C00000000000400040000071
:10CFC000000000C000C00000000000400040000061
:10CFD000000000C000C00000000000400040000051
:10CFE000000000C000C00000000000400040000041
:10CFF000000000C000C00000000000400040000031
:10D00000000000C000C00000000000400040000020
:10D01000000000C000C00000000000400040000010
:10D02000000000C000C00000000000400040000000
:10D03000000000C000C000000000004000400000F0
:10D04000000000C000C000000000004000400000E0
:10D05000000000C000C000000000004000400000D0
:10D06000000000C000C000000000004000400000C0
:10D07000000000C000C000000000004000400000B0
:10D08000000000C000C000000000004000400000A0
:10D09000000000C000C00000000000400040000090
:10D0A000000000C000C00000000000400040000080
:10D0B000000000C000C00000000000400040000070
:10D0C000000000C000C00000000000400040000060
:10D0D000000000C000C00000000000400040000050
:10D0E000000000C000C00000000000400040000040
:10D0F000000000C000C00000000000400040000030
:10D10000000000C000C0000000000040004000001F
:10D11000000000C000C0000000000040004000000F
:10D12000000000C000C000000000004000400000FF
:10D13000000000C000C000000000004000400000EF
:10D14000000000C000C000000000004000400000DF
:10D15000000000C000C000000000004000400000CF
:10D16000000000C000C000000000004000400000BF
:10D17000000000C000C000000000004000400000AF
:10D18000000000C000C0000000000040004000009F
:10D19000000000C000C0000000000040004000008F
:10D1A000000000C000C0000000000040004000007F
:10D1B000000000C000C0000000000040004000006F
:10D1C000000000C000C0000000000040004000005F
:10D1D000000000C000C0000000000040004000004F
:10D1E000000000C000C0000000000040004000003F
:10D1F000000000C000C0000000000040004000002F
:10D20000000000C000C0000000000040004000001E
:10D21000000000C000C0000000000040004000000E
:10D22000000000C000C000000000004000400000FE
:10D23000000000C000C000000000004000400000EE
:10D24000000000C000C000000000004000400000DE
:10D25000000000C000C000000000004000400000CE
:10D26000000000C000C000000000004000400000BE
:10D27000000000C000C000000000004000400000AE
:10D28000000000C000C0000000000040004000009E
:10D29000000000C000C0000000000040004000008E
:10D2A000000000C000C0000000000040004000007E
:10D2B000000000C000C0000000000040004000006E
:10D2C000000000C000C0000000000040004000005E
:10D2D000000000C000C0000000000040004000004E
:10D2E000000000C000C0000000000040004000003E
:10D2F000000000C000C0000000000040004000002E
:10D30000000000C000C0000000000040004000001D
:10D31000000000C000C0000000000040004000000D
:10D32000000000C000C000000000004000400000FD
:10D33000000000C000C000000000004000400000ED
:10D34000000000C000C000000000004000400000DD
:10D35000000000C000C000000000004000400000CD
:10D36000000000C000C000000000004000400000BD
:10D37000000000C000C000000000004000400000AD
:10D38000000000C000C0000000000040004000009D
:10D39000000000C000C0000000000040004000008D
:10D3A000000000C000C0000000000040004000007D
:10D3B000000000C000C0000000000040004000006D
:10D3C000000000C000C0000000000040004000005D
:10D3D000000000C000C0000000000040004000004D
:10D3E000000000C000C0000000000040004000003D
:10D3F000000000C000C0000000000040004000002D
:10D40000000000C000C0000000000040004000001C
:10D41000000000C000C0000000000040004000000C
:10D42000000000C000C000000000004000400000FC
:10D43000000000C000C000000000004000400000EC
:10D44000000000C000C000000000004000400000DC
:10D45000000000C000C000000000004000400000CC
:10D46000000000C000C000000000004000400000BC
:10D47000000000C000C000000000004000400000AC
:10D48000000000C000C0000000000040004000009C
:10D49000000000C000C0000000000040004000008C
:10D4A000000000C000C0000000000040004000007C
:10D4B000000000C000C0000000000040004000006C
:10D4C000000000C000C0000000000040004000005C
:10D4D000000000C000C0000000000040004000004C
:10D4E000000000C000C0000000000040004000003C
:10D4F000000000C000C0000000000040004000002C
:10D50000000000C000C0000000000040004000001B
:10D51000000000C000C0000000000040004000000B
:10D52000000000C000C000000000004000400000FB
:10D53000000000C000C000000000004000400000EB
:10D54000000000C000C000000000004000400000DB
:10D55000000000C000C000000000004000400000CB
:10D56000000000C000C000000000004000400000BB
:10D57000000000C000C000000000004000400000AB
:10D58000000000C000C0000000000040004000009B
:10D59000000000C000C0000000000040004000008B
:10D5A000000000C000C0000000000040004000007B
:10D5B000000000C000C0000000000040004000006B
:10D5C000000000C000C0000000000040004000005B
:10D5D000000000C000C0000000000040004000004B
:10D5E000000000C000C0000000000040004000003B
:10D5F000000000C000C0000000000040004000002B
:10D60000000000C000C0000000000040004000001A
:10D61000000000C000C0000000000040004000000A
:10D62000000000C000C000000000004000400000FA
:10D63000000000C000C000000000004000400000EA
:10D64000000000C000C000000000004000400000DA
:10D65000000000C000C000000000004000400000CA
:10D66000000000C000C000000000004000400000BA
:10D67000000000C000C000000000004000400000AA
:10D68000000000C000C0000000000040004000009A
:10D69000000000C000C0000000000040004000008A
:10D6A000000000C000C0000000000040004000007A
:10D6B000000000C000C0000000000040004000006A
:10D6C000000000C000C0000000000040004000005A
:10D6D000000000C000C0000000000040004000004A
:10D6E000000000C000C0000000000040004000003A
:10D6F000000000C000C0000000000040004000002A
:10D70000000000C000C00000000000400040000019
:10D71000000000C000C00000000000400040000009
:10D72000000000C000C000000000004000400000F9
:10D73000000000C000C000000000004000400000E9
:10D74000000000C000C000000000004000400000D9
:10D75000000000C000C000000000004000400000C9
:10D76000000000C000C000000000004000400000B9
:10D77000000000C000C000000000004000400000A9
:10D78000000000C000C00000000000400040000099
:10D79000000000C000C0000000000040C53C1314A1
:10D7A0001F2699CC26DBADCBC2C294126EFEFB3F86
:10D7B000423C8F155F278CCD72DCCACA52C2111150
:10D7C000DDFCEC3FB63B0817992887CEC3DDEEC9D8
:10D7D000ECC18C0F4BFBD33F203B7D18CD298ACF6A
:10D7E00019DF1BC98FC1050EBBF9B13F823AEF1992
:10D7F000FA2A95D075E051C83BC17C0C2BF8843FC8
:10D80000DA395D1B212CA6D1D5E18FC7F2C0F10A10
:10D810009CF64E3F2A39C61C412DBFD23AE3D6C6EC
:10D82000B2C064090FF50E3F71382B1E5A2EDFD39C
:10D83000A3E426C67CC0D50784F3C53EAF378B1F53
:10D840006B2F06D511E67EC54FC04506FBF1713E34
:10D85000E536E720763033D683E7E0C42DC0B50443
:10D8600074F0143E12363D22793167D7F8E84AC485
:10D8700014C02303EFEEAE3D36358E237432A1D8AB
:10D8800071EABEC305C092016CED3E3D5334DA240B
:10D890006733E1D9EDEB3BC300C00000EDEBC53CC5
:10D8A00067331F26533426DB6CEDC2C205C06EFE03
:10D8B00071EA423C74325F27363572DCEFEE52C2B9
:10D8C00014C0DDFCF8E8B63B793199281236C3DD87
:10D8D00074F0ECC12DC04BFB83E7203B7630CD29A3
:10D8E000E53619DFFBF18FC14FC0BBF911E6823A73
:10D8F0006B2FFA2AAF3775E084F33BC17CC02BF85D
:10D90000A3E4DA395A2E212C7138D5E10FF5F2C093
:10D91000B2C09CF63AE32A39412D412D2A393AE327
:10D920009CF6B2C0F2C00FF5D5E17138212C5A2E09
:10D93000DA39A3E42BF87CC03BC184F375E0AF3740
:10D94000FA2A6B2F823A11E6BBF94FC08FC1FBF167
:10D9500019DFE536CD297630203B83E74BFB2DC020
:10D96000ECC174F0C3DD123699287931B63BF8E882
:10D97000DDFC14C052C2EFEE72DC36355F27743224
:10D98000423C71EA6EFE05C0C2C26CED26DB533428
:10D990001F266733C53CEDEB000000C03BC3EDEB39
:10D9A000E1D96733DA2453343E3D6CED920105C072
:10D9B000BEC371EAA1D874328E233635AE3DEFEE88
:10D9C000230314C04AC4F8E867D779313D221236E0
:10D9D000143E74F0B5042DC0E0C483E733D676302E
:10D9E000E720E536713EFBF145064FC07EC511E6E6
:10D9F00006D56B2F8B1FAF37C53E84F3D5077CC090
:10DA000026C6A3E4DFD35A2E2B1E71380E3F0FF526
:10DA10006409B2C0D6C63AE3BFD2412DC61C2A392A
:10DA20004E3F9CF6F10AF2C08FC7D5E1A6D1212C5A
:10DA30005D1BDA39843F2BF87C0C3BC151C875E083
:10DA400095D0FA2AEF19823AB13FBBF9050E8FC182
:10DA50001BC919DF8ACFCD297D18203BD33F4BFB53
:10DA60008C0FECC1EEC9C3DD87CE99280817B63BF1
:10DA7000EC3FDDFC111152C2CACA72DC8CCD5F27AB
:10DA80008F15423CFB3F6EFE9412C2C2ADCB26DB2B
:10DA900099CC1F261314C53C0040000013143BC34F
:10DAA00099CCE1D9ADCBDA2494123E3DFB3F9201F3
:10DAB0008F15BEC38CCDA1D8CACA8E231111AE3D1D
:10DAC000EC3F230308174AC487CE67D7EEC93D222F
:10DAD0008C0F143ED33FB5047D18E0C48ACF33D6F3
:10DAE0001BC9E720050E713EB13F4506EF197EC503
:10DAF00095D006D551C88B1F7C0CC53E843FD507F9
:10DB00005D1B26C6A6D1DFD38FC72B1EF10A0E3FA1
:10DB10004E3F6409C61CD6C6BFD2BFD2D6C6C61CED
:10DB200064094E3F0E3FF10A2B1E8FC7DFD3A6D1EB
:10DB300026C65D1BD507843FC53E7C0C8B1F51C894
:10DB400006D595D07EC5EF194506B13F713E050E4D
:10DB5000E7201BC933D68ACFE0C47D18B504D33F74
:10DB6000143E8C0F3D22EEC967D787CE4AC40817F2
:10DB70002303EC3FAE3D11118E23CACAA1D88CCD30
:10DB8000BEC38F159201FB3F3E3D9412DA24ADCB0C
:10DB9000E1D999CC3BC3131400000040C53C1314D9
:10DBA0001F2699CC26DBADCBC2C294126EFEFB3F82
:10DBB000423C8F155F278CCD72DCCACA52C211114C
:10DBC000DDFCEC3FB63B0817992887CEC3DDEEC9D4
:10DBD000ECC18C0F4BFBD33F203B7D18CD298ACF66
:10DBE00019DF1BC98FC1050EBBF9B13F823AEF198E
:10DBF000FA2A95D075E051C83BC17C0C2BF8843FC4
:10DC0000DA395D1B212CA6D1D5E18FC7F2C0F10A0C
:10DC10009CF64E3F2A39C61C412DBFD23AE3D6C6E8
:10DC2000B2C064090FF50E3F71382B1E5A2EDFD398
:10DC3000A3E426C67CC0D50784F3C53EAF378B1F4F
:10DC40006B2F06D511E67EC54FC04506FBF1713E30
:10DC5000E536E720763033D683E7E0C42DC0B5043F
:10DC600074F0143E12363D22793167D7F8E84AC481
:10DC700014C02303EFEEAE3D36358E237432A1D8A7
:10DC800071EABEC305C092016CED3E3D5334DA2407
:10DC90006733E1D9EDEB3BC300C00000EDEBC53CC1
:10DCA00067331F26533426DB6CEDC2C205C06EFEFF
:10DCB00071EA423C74325F27363572DCEFEE52C2B5
:10DCC00014C0DDFCF8E8B63B793199281236C3DD83
:10DCD00074F0ECC12DC04BFB83E7203B7630CD299F
:10DCE000E53619DFFBF18FC14FC0BBF911E6823A6F
:10DCF0006B2FFA2AAF3775E084F33BC17CC02BF859
:10DD0000A3E4DA395A2E212C7138D5E10FF5F2C08F
:10DD1000B2C09CF63AE32A39412D412D2A393AE323
:10DD20009CF6B2C0F2C00FF5D5E17138212C5A2E05
:10DD3000DA39A3E42BF87CC03BC184F375E0AF373C
:10DD4000FA2A6B2F823A11E6BBF94FC08FC1FBF163
:10DD500019DFE536CD297630203B83E74BFB2DC01C
:10DD6000ECC174F0C3DD123699287931B63BF8E87E
:10DD7000DDFC14C052C2EFEE72DC36355F27743220
:10DD8000423C71EA6EFE05C0C2C26CED26DB533424
:10DD90001F266733C53CEDEB000000C03BC3EDEB35
:10DDA000E1D96733DA2453343E3D6CED920105C06E
:10DDB000BEC371EAA1D874328E233635AE3DEFEE84
:10DDC000230314C04AC4F8E867D779313D221236DC
:10DDD000143E74F0B5042DC0E0C483E733D676302A
:10DDE000E720E536713EFBF145064FC07EC511E6E2
:10DDF00006D56B2F8B1FAF37C53E84F3D5077CC08C
:10DE000026C6A3E4DFD35A2E2B1E71380E3F0FF522
:10DE10006409B2C0D6C63AE3BFD2412DC61C2A3926
:10DE20004E3F9CF6F10AF2C08FC7D5E1A6D1212C56
:10DE30005D1BDA39843F2BF87C0C3BC151C875E07F
:10DE400095D0FA2AEF19823AB13FBBF9050E8FC17E
:10DE50001BC919DF8ACFCD297D18203BD33F4BFB4F
:10DE60008C0FECC1EEC9C3DD87CE99280817B63BED
:10DE7000EC3FDDFC111152C2CACA72DC8CCD5F27A7
:10DE80008F15423CFB3F6EFE9412C2C2ADCB26DB27
:10DE900099CC1F261314C53C0040000013143BC34B
:10DEA00099CCE1D9ADCBDA2494123E3DFB3F9201EF
:10DEB0008F15BEC38CCDA1D8CACA8E231111AE3D19
:10DEC000EC3F230308174AC487CE67D7EEC93D222B
:10DED0008C0F143ED33FB5047D18E0C48ACF33D6EF
:10DEE0001BC9E720050E713EB13F4506EF197EC5FF
:10DEF00095D006D551C88B1F7C0CC53E843FD507F5
:10DF00005D1B26C6A6D1DFD38FC72B1EF10A0E3F9D
:10DF10004E3F6409C61CD6C6BFD2BFD2D6C6C61CE9
:10DF200064094E3F0E3FF10A2B1E8FC7DFD3A6D1E7
:10DF300026C65D1BD507843FC53E7C0C8B1F51C890
:10DF400006D595D07EC5EF194506B13F713E050E49
:10DF5000E7201BC933D68ACFE0C47D18B504D33F70
:10DF6000143E8C0F3D22EEC967D787CE4AC40817EE
:10DF70002303EC3FAE3D11118E23CACAA1D88CCD2C
:10DF8000BEC38F159201FB3F3E3D9412DA24ADCB08
:10DF9000E1D999CC3BC3131400000040D33FB50432
:10DFA0006409B2C08FC1FBF16CED3E3DB63B081772
:10DFB0005D1B26C651C875E072DC363574325F27AA
:10DFC000FA2A95D0DFD3A6D187CE9928DA24533404
:10DFD000E53619DF3AE3D6C6E0C47D181314C53C14
:10DFE000143E74F00FF5F2C04FC045069201FB3F9E
:10DFF000EC3F2303D5077CC03BC184F3EFEEAE3D7D
:10E00000423C8F15EF197EC58FC7D5E1C3DD1236AF
:10E0100067331F26CD298ACFBFD2BFD28ACFCD2961
:10E020001F2667331236C3DDD5E18FC77EC5EF19D2
:10E030008F15423CAE3DEFEE84F33BC17CC0D5076B
:10E040002303EC3FFB3F920145064FC0F2C00FF5A2
:10E0500074F0143EC53C13147D18E0C4D6C63AE3F0
:10E0600019DFE5365334DA24992887CEA6D1DFD3D9
:10E0700095D0FA2A5F277432363572DC75E051C8C4
:10E0800026C65D1B0817B63B3E3D6CEDFBF18FC10C
:10E09000B2C06409B504D33F00400000B5042DC0F0
:10E0A000B2C09CF6FBF1713E3E3D941208174AC483
:10E0B00026C6A3E475E0AF3736358E235F278CCDB7
:10E0C00095D006D5A6D1212C99287931533426DB59
:10E0D00019DF1BC9D6C6C61C7D18203BC53CEDEB1D
:10E0E00074F0ECC1F2C0F10A4506B13FFB3F6EFE91
:10E0F000230314C07CC02BF884F3C53EAE3D111140
:10E100008F15BEC37EC511E6D5E1713812363D22AA
:10E110001F2699CC8ACF33D6BFD2412DCD29763058
:10E120006733E1D9C3DDEEC98FC72B1EEF19823AE1
:10E13000423C71EAEFEE52C23BC17C0CD507843FF2
:10E14000EC3FDDFC920105C04FC0BBF90FF50E3F5F
:10E15000143E8C0F13143BC3E0C483E73AE32A391F
:10E16000E536E720DA24ADCB87CE67D7DFD35A2E4A
:10E17000FA2A6B2F7432A1D872DCCACA51C88B1F1D
:10E180005D1BDA39B63BF8E86CEDC2C28FC1050EF3
:10E1900064094E3FD33F4BFB000000C02DC04BFB3A
:10E1A0009CF64E3F713E050E9412C2C24AC4F8E876
:10E1B000A3E4DA39AF378B1F8E23CACA8CCDA1D81E
:10E1C00006D56B2F212C5A2E793167D726DBADCBA4
:10E1D0001BC9E720C61C2A39203B83E7EDEB3BC374
:10E1E000ECC18C0FF10A0E3FB13FBBF96EFE05C0CA
:10E1F00014C0DDFC2BF8843FC53E7C0C111152C2CB
:10E20000BEC371EA11E6823A71382B1E3D22EEC977
:10E2100099CCE1D933D67630412D412D763033D6A5
:10E22000E1D999CCEEC93D222B1E7138823A11E614
:10E2300071EABEC352C211117C0CC53E843F2BF85B
:10E24000DDFC14C005C06EFEBBF9B13F0E3FF10A04
:10E250008C0FECC13BC3EDEB83E7203B2A39C61C96
:10E26000E7201BC9ADCB26DB67D779315A2E212C8D
:10E270006B2F06D5A1D88CCDCACA8E238B1FAF3782
:10E28000DA39A3E4F8E84AC4C2C29412050E713E1A
:10E290004E3F9CF64BFB2DC000C000004BFBD33F14
:10E2A0004E3F6409050E8FC1C2C26CEDF8E8B63B63
:10E2B000DA395D1B8B1F51C8CACA72DCA1D874320F
:10E2C0006B2FFA2A5A2EDFD367D787CEADCBDA244D
:10E2D000E720E5362A393AE383E7E0C43BC3131469
:10E2E0008C0F143E0E3F0FF5BBF94FC005C09201D5
:10E2F000DDFCEC3F843FD5077C0C3BC152C2EFEE06
:10E3000071EA423C823AEF192B1E8FC7EEC9C3DD7A
:10E31000E1D967337630CD29412DBFD233D68ACFAC
:10E3200099CC1F263D2212367138D5E111E67EC503
:10E33000BEC38F151111AE3DC53E84F32BF87CC0D2
:10E3400014C023036EFEFB3FB13F4506F10AF2C045
:10E35000ECC174F0EDEBC53C203B7D18C61CD6C665
:10E360001BC919DF26DB533479319928212CA6D11A
:10E3700006D595D08CCD5F278E233635AF3775E027
:10E38000A3E426C64AC4081794123E3D713EFBF131
:10E390009CF6B2C02DC0B50400000040D33FB504C8
:10E3A0006409B2C08FC1FBF16CED3E3DB63B08176E
:10E3B0005D1B26C651C875E072DC363574325F27A6
:10E3C000FA2A95D0DFD3A6D187CE9928DA24533400
:10E3D000E53619DF3AE3D6C6E0C47D181314C53C10
:10E3E000143E74F00FF5F2C04FC045069201FB3F9A
:10E3F000EC3F2303D5077CC03BC184F3EFEEAE3D79
:10E40000423C8F15EF197EC58FC7D5E1C3DD1236AB
:10E4100067331F26CD298ACFBFD2BFD28ACFCD295D
:10E420001F2667331236C3DDD5E18FC77EC5EF19CE
:10E430008F15423CAE3DEFEE84F33BC17CC0D50767
:10E440002303EC3FFB3F920145064FC0F2C00FF59E
:10E4500074F0143EC53C13147D18E0C4D6C63AE3EC
:10E4600019DFE5365334DA24992887CEA6D1DFD3D5
:10E4700095D0FA2A5F277432363572DC75E051C8C0
:10E4800026C65D1B0817B63B3E3D6CEDFBF18FC108
:10E49000B2C06409B504D33F00400000B5042DC0EC
:10E4A000B2C09CF6FBF1713E3E3D941208174AC47F
:10E4B00026C6A3E475E0AF3736358E235F278CCDB3
:10E4C00095D006D5A6D1212C99287931533426DB55
:10E4D00019DF1BC9D6C6C61C7D18203BC53CEDEB19
:10E4E00074F0ECC1F2C0F10A4506B13FFB3F6EFE8D
:10E4F000230314C07CC02BF884F3C53EAE3D11113C
:10E500008F15BEC37EC511E6D5E1713812363D22A6
:10E510001F2699CC8ACF33D6BFD2412DCD29763054
:10E520006733E1D9C3DDEEC98FC72B1EEF19823ADD
:10E53000423C71EAEFEE52C23BC17C0CD507843FEE
:10E54000EC3FDDFC920105C04FC0BBF90FF50E3F5B
:10E55000143E8C0F13143BC3E0C483E73AE32A391B
:10E56000E536E720DA24ADCB87CE67D7DFD35A2E46
:10E57000FA2A6B2F7432A1D872DCCACA51C88B1F19
:10E580005D1BDA39B63BF8E86CEDC2C28FC1050EEF
:10E5900064094E3FD33F4BFB000000C02DC04BFB36
:10E5A0009CF64E3F713E050E9412C2C24AC4F8E872
:10E5B000A3E4DA39AF378B1F8E23CACA8CCDA1D81A
:10E5C00006D56B2F212C5A2E793167D726DBADCBA0
:10E5D0001BC9E720C61C2A39203B83E7EDEB3BC370
:10E5E000ECC18C0FF10A0E3FB13FBBF96EFE05C0C6
:10E5F00014C0DDFC2BF8843FC53E7C0C111152C2C7
:10E60000BEC371EA11E6823A71382B1E3D22EEC973
:10E6100099CCE1D933D67630412D412D763033D6A1
:10E62000E1D999CCEEC93D222B1E7138823A11E610
:10E6300071EABEC352C211117C0CC53E843F2BF857
:10E64000DDFC14C005C06EFEBBF9B13F0E3FF10A00
:10E650008C0FECC13BC3EDEB83E7203B2A39C61C92
:10E66000E7201BC9ADCB26DB67D779315A2E212C89
:10E670006B2F06D5A1D88CCDCACA8E238B1FAF377E
:10E68000DA39A3E4F8E84AC4C2C29412050E713E16
:10E690004E3F9CF64BFB2DC000C000004BFBD33F10
:10E6A0004E3F6409050E8FC1C2C26CEDF8E8B63B5F
:10E6B000DA395D1B8B1F51C8CACA72DCA1D874320B
:10E6C0006B2FFA2A5A2EDFD367D787CEADCBDA2449
:10E6D000E720E5362A393AE383E7E0C43BC3131465
:10E6E0008C0F143E0E3F0FF5BBF94FC005C09201D1
:10E6F000DDFCEC3F843FD5077C0C3BC152C2EFEE02
:10E7000071EA423C823AEF192B1E8FC7EEC9C3DD76
:10E71000E1D967337630CD29412DBFD233D68ACFA8
:10E7200099CC1F263D2212367138D5E111E67EC5FF
:10E73000BEC38F151111AE3DC53E84F32BF87CC0CE
:10E7400014C023036EFEFB3FB13F4506F10AF2C041
:10E75000ECC174F0EDEBC53C203B7D18C61CD6C661
:10E760001BC919DF26DB533479319928212CA6D116
:10E7700006D595D08CCD5F278E233635AF3775E023
:10E78000A3E426C64AC4081794123E3D713EFBF12D
:10E790009CF6B2C02DC0B50400000040C53E7C0C04
:10E7A0007D18E0C4CACA72DCBFD2412D8E23363533
:10E7B000203B83E784F33BC100C0000084F3C53EE7
:10E7C000203B7D188E23CACABFD2BFD2CACA8E23AD
:10E7D0007D18203BC53E84F3000000C03BC184F39C
:10E7E00083E7203B36358E23412DBFD272DCCACA67
:10E7F000E0C47D187C0CC53E004000007C0C3BC191
:10E80000E0C483E772DC3635412D412D363572DCAC
:10E8100083E7E0C43BC17C0C00000040C53E7C0C9B
:10E820007D18E0C4CACA72DCBFD2412D8E233635B2
:10E83000203B83E784F33BC100C0000084F3C53E66
:10E84000203B7D188E23CACABFD2BFD2CACA8E232C
:10E850007D18203BC53E84F3000000C03BC184F31B
:10E8600083E7203B36358E23412DBFD272DCCACAE6
:10E87000E0C47D187C0CC53E004000007C0C3BC110
:10E88000E0C483E772DC3635412D412D363572DC2C
:10E8900083E7E0C43BC17C0C00000040C53E7C0C1B
:10E8A0007D18E0C4CACA72DCBFD2412D8E23363532
:10E8B000203B83E784F33BC100C0000084F3C53EE6
:10E8C000203B7D188E23CACABFD2BFD2CACA8E23AC
:10E8D0007D18203BC53E84F3000000C03BC184F39B
:10E8E00083E7203B36358E23412DBFD272DCCACA66
:10E8F000E0C47D187C0CC53E004000007C0C3BC190
:10E90000E0C483E772DC3635412D412D363572DCAB
:10E9100083E7E0C43BC17C0C00000040C53E7C0C9A
:10E920007D18E0C4CACA72DCBFD2412D8E233635B1
:10E93000203B83E784F33BC100C0000084F3C53E65
:10E94000203B7D188E23CACABFD2BFD2CACA8E232B
:10E950007D18203BC53E84F3000000C03BC184F31A
:10E9600083E7203B36358E23412DBFD272DCCACAE5
:10E97000E0C47D187C0CC53E004000007C0C3BC10F
:10E98000E0C483E772DC3635412D412D363572DC2B
:10E9900083E7E0C43BC17C0C00000040C53E7C0C1A
:10E9A0007D18E0C4CACA72DCBFD2412D8E23363531
:10E9B000203B83E784F33BC100C0000084F3C53EE5
:10E9C000203B7D188E23CACABFD2BFD2CACA8E23AB
:10E9D0007D18203BC53E84F3000000C03BC184F39A
:10E9E00083E7203B36358E23412DBFD272DCCACA65
:10E9F000E0C47D187C0CC53E004000007C0C3BC18F
:10EA0000E0C483E772DC3635412D412D363572DCAA
:10EA100083E7E0C43BC17C0C00000040C53E7C0C99
:10EA20007D18E0C4CACA72DCBFD2412D8E233635B0
:10EA3000203B83E784F33BC100C0000084F3C53E64
:10EA4000203B7D188E23CACABFD2BFD2CACA8E232A
:10EA50007D18203BC53E84F3000000C03BC184F319
:10EA600083E7203B36358E23412DBFD272DCCACAE4
:10EA7000E0C47D187C0CC53E004000007C0C3BC10E
:10EA8000E0C483E772DC3635412D412D363572DC2A
:10EA900083E7E0C43BC17C0C00000040C53E7C0C19
:10EAA0007D18E0C4CACA72DCBFD2412D8E23363530
:10EAB000203B83E784F33BC100C0000084F3C53EE4
:10EAC000203B7D188E23CACABFD2BFD2CACA8E23AA
:10EAD0007D18203BC53E84F3000000C03BC184F399
:10EAE00083E7203B36358E23412DBFD272DCCACA64
:10EAF000E0C47D187C0CC53E004000007C0C3BC18E
:10EB0000E0C483E772DC3635412D412D363572DCA9
:10EB100083E7E0C43BC17C0C00000040C53E7C0C98
:10EB20007D18E0C4CACA72DCBFD2412D8E233635AF
:10EB3000203B83E784F33BC100C0000084F3C53E63
:10EB4000203B7D188E23CACABFD2BFD2CACA8E2329
:10EB50007D18203BC53E84F3000000C03BC184F318
:10EB600083E7203B36358E23412DBFD272DCCACAE3
:10EB7000E0C47D187C0CC53E004000007C0C3BC10D
:10EB8000E0C483E772DC3635412D412D363572DC29
:10EB900083E7E0C43BC17C0C00000040C53E7C0C18
:10EBA0007D18E0C4CACA72DCBFD2412D8E2336352F
:10EBB000203B83E784F33BC100C0000084F3C53EE3
:10EBC000203B7D188E23CACABFD2BFD2CACA8E23A9
:10EBD0007D18203BC53E84F3000000C03BC184F398
:10EBE00083E7203B36358E23412DBFD272DCCACA63
:10EBF000E0C47D187C0CC53E004000007C0C3BC18D
:10EC0000E0C483E772DC3635412D412D363572DCA8
:10EC100083E7E0C43BC17C0C00000040C53E7C0C97
:10EC20007D18E0C4CACA72DCBFD2412D8E233635AE
:10EC3000203B83E784F33BC100C0000084F3C53E62
:10EC4000203B7D188E23CACABFD2BFD2CACA8E2328
:10EC50007D18203BC53E84F3000000C03BC184F317
:10EC600083E7203B36358E23412DBFD272DCCACAE2
:10EC7000E0C47D187C0CC53E004000007C0C3BC10C
:10EC8000E0C483E772DC3635412D412D363572DC28
:10EC900083E7E0C43BC17C0C00000040C53E7C0C17
:10ECA0007D18E0C4CACA72DCBFD2412D8E2336352E
:10ECB000203B83E784F33BC100C0000084F3C53EE2
:10ECC000203B7D188E23CACABFD2BFD2CACA8E23A8
:10ECD0007D18203BC53E84F3000000C03BC184F397
:10ECE00083E7203B36358E23412DBFD272DCCACA62
:10ECF000E0C47D187C0CC53E004000007C0C3BC18C
:10ED0000E0C483E772DC3635412D412D363572DCA7
:10ED100083E7E0C43BC17C0C00000040C53E7C0C96
:10ED20007D18E0C4CACA72DCBFD2412D8E233635AD
:10ED3000203B83E784F33BC100C0000084F3C53E61
:10ED4000203B7D188E23CACABFD2BFD2CACA8E2327
:10ED50007D18203BC53E84F3000000C03BC184F316
:10ED600083E7203B36358E23412DBFD272DCCACAE1
:10ED7000E0C47D187C0CC53E004000007C0C3BC10B
:10ED8000E0C483E772DC3635412D412D363572DC27
:10ED900083E7E0C43BC17C0C00000040C53E7C0C16
:10EDA0007D18E0C4CACA72DCBFD2412D8E2336352D
:10EDB000203B83E784F33BC100C0000084F3C53EE1
:10EDC000203B7D188E23CACABFD2BFD2CACA8E23A7
:10EDD0007D18203BC53E84F3000000C03BC184F396
:10EDE00083E7203B36358E23412DBFD272DCCACA61
:10EDF000E0C47D187C0CC53E004000007C0C3BC18B
:10EE0000E0C483E772DC3635412D412D363572DCA6
:10EE100083E7E0C43BC17C0C00000040C53E7C0C95
:10EE20007D18E0C4CACA72DCBFD2412D8E233635AC
:10EE3000203B83E784F33BC100C0000084F3C53E60
:10EE4000203B7D188E23CACABFD2BFD2CACA8E2326
:10EE50007D18203BC53E84F3000000C03BC184F315
:10EE600083E7203B36358E23412DBFD272DCCACAE0
:10EE7000E0C47D187C0CC53E004000007C0C3BC10A
:10EE8000E0C483E772DC3635412D412D363572DC26
:10EE900083E7E0C43BC17C0C00000040C53E7C0C15
:10EEA0007D18E0C4CACA72DCBFD2412D8E2336352C
:10EEB000203B83E784F33BC100C0000084F3C53EE0
:10EEC000203B7D188E23CACABFD2BFD2CACA8E23A6
:10EED0007D18203BC53E84F3000000C03BC184F395
:10EEE00083E7203B36358E23412DBFD272DCCACA60
:10EEF000E0C47D187C0CC53E004000007C0C3BC18A
:10EF0000E0C483E772DC3635412D412D363572DCA5
:10EF100083E7E0C43BC17C0C00000040C53E7C0C94
:10EF20007D18E0C4CACA72DCBFD2412D8E233635AB
:10EF3000203B83E784F33BC100C0000084F3C53E5F
:10EF4000203B7D188E23CACABFD2BFD2CACA8E2325
:10EF50007D18203BC53E84F3000000C03BC184F314
:10EF600083E7203B36358E23412DBFD272DCCACADF
:10EF7000E0C47D187C0CC53E004000007C0C3BC109
:10EF8000E0C483E772DC3635412D412D363572DC25
:10EF900083E7E0C43BC17C0CA0100108A410010869
:10EFA000B840020898AF0008B8380208B830020824
:10EFB00098BF00088808010888000108B8280208DE
:10EFC000B820020898C70008B8180208B81002084C
:10EFD000B8080208B800020898B70008B8F8010895
:10EFE000B8F00108B8E80108B8E0010898D70008AF
:10EFF000B8D80108B8D00108B8C80108B8C00108DD
:10F0000098E70008B8B80108B8B00108B8A8010826
:10F01000B8A0010898DF0008B8980108B890010866
:10F0200098CF0008B8880108B8800108B8780108AE
:10F03000B8700108B8680108B8600108B85801083C
:10F04000B8500108B8480108B8400108B8380108AC
:10F05000B8300108B8280108B8200108B81801081C
:10F06000B810010800000040000000C0000000408F
:10F07000000000C000000040000000C00000004090
:10F08000000000C000000040000000C00000004080
:10F09000000000C000000040000000C00000004070
:10F0A000000000C000000040000000C00000004060
:10F0B000000000C000000040000000C00000004050
:10F0C000000000C000000040000000C00000004040
:10F0D000000000C000000040000000C00000004030
:10F0E000000000C000000040000000C00000004020
:10F0F000000000C000000040000000C00000004010
:10F10000000000C000000040000000C000000040FF
:10F11000000000C000000040000000C000000040EF
:10F12000000000C000000040000000C000000040DF
:10F13000000000C000000040000000C000000040CF
:10F14000000000C000000040000000C000000040BF
:10F15000000000C000000040000000C000000040AF
:10F16000000000C000000040000000C0000000409F
:10F17000000000C000000040000000C0000000408F
:10F18000000000C000000040000000C0000000407F
:10F19000000000C000000040000000C0000000406F
:10F1A000000000C000000040000000C0000000405F
:10F1B000000000C000000040000000C0000000404F
:10F1C000000000C000000040000000C0000000403F
:10F1D000000000C000000040000000C0000000402F
:10F1E000000000C000000040000000C0000000401F
:10F1F000000000C000000040000000C0000000400F
:10F20000000000C000000040000000C000000040FE
:10F21000000000C000000040000000C000000040EE
:10F22000000000C000000040000000C000000040DE
:10F23000000000C000000040000000C000000040CE
:10F24000000000C000000040000000C000000040BE
:10F25000000000C000000040000000C000000040AE
:10F26000000000C000000040000000C0000000409E
:10F27000000000C000000040000000C0000000408E
:10F28000000000C000000040000000C0000000407E
:10F29000000000C000000040000000C0000000406E
:10F2A000000000C000000040000000C0000000405E
:10F2B000000000C000000040000000C0000000404E
:10F2C000000000C000000040000000C0000000403E
:10F2D000000000C000000040000000C0000000402E
:10F2E000000000C000000040000000C0000000401E
:10F2F000000000C000000040000000C0000000400E
:10F30000000000C000000040000000C000000040FD
:10F31000000000C000000040000000C000000040ED
:10F32000000000C000000040000000C000000040DD
:10F33000000000C000000040000000C000000040CD
:10F34000000000C000000040000000C000000040BD
:10F35000000000C000000040000000C000000040AD
:10F36000000000C000000040000000C0000000409D
:10F37000000000C000000040000000C0000000408D
:10F38000000000C000000040000000C0000000407D
:10F39000000000C000000040000000C0000000406D
:10F3A000000000C000000040000000C0000000405D
:10F3B000000000C000000040000000C0000000404D
:10F3C000000000C000000040000000C0000000403D
:10F3D000000000C000000040000000C0000000402D
:10F3E000000000C000000040000000C0000000401D
:10F3F000000000C000000040000000C0000000400D
:10F40000000000C000000040000000C000000040FC
:10F41000000000C000000040000000C000000040EC
:10F42000000000C000000040000000C000000040DC
:10F43000000000C000000040000000C000000040CC
:10F44000000000C000000040000000C000000040BC
:10F45000000000C000000040000000C000000040AC
:10F46000000000C000005A2EEC3FCD29BBF98CCD26
:10F47000B2C026DB7C0C1236143E8B1F6CEDD6C658
:10F48000BEC311E67D18B63BDA391314D5E152C27A
:10F490001BC9FBF18E230E3F6733D50767D72DC0FD
:10F4A00095D06EFE412DFB3FFA2A4BFB87CE7CC0E8
:10F4B000E1D9F10A3635713EE720EFEE8FC73BC345
:10F4C000A3E40817203B823A8F153AE3C2C251C821
:10F4D00074F03D22C53E53346409A1D84FC08ACF91
:10F4E000DDFC212C0040212CDDFC8ACF4FC0A1D8AF
:10F4F00064095334C53E3D2274F051C8C2C23AE398
:10F500008F15823A203B0817A3E43BC38FC7EFEE69
:10F51000E720713E3635F10AE1D97CC087CE4BFB3E
:10F52000FA2AFB3F412D6EFE95D02DC067D7D50737
:10F5300067330E3F8E23FBF11BC952C2D5E1131472
:10F54000DA39B63B7D1811E6BEC3D6C66CED8B1F0B
:10F55000143E12367C0C26DBB2C08CCDBBF9CD2913
:10F56000EC3F5A2E0000A6D114C033D645067432A3
:10F570004E3FDA2484F3EEC9ECC175E094122A39C7
:10F58000423CEF1983E74AC426C6EDEB2B1EAE3D85
:10F59000E536050E72DCF2C099CC2BF89928D33FE2
:10F5A0006B2F9201BFD205C006D5B5047931843FD7
:10F5B0001F260FF5CACA8FC119DF11117138C53C5A
:10F5C0005D1BF8E8E0C47EC571EAC61C3E3DAF375E
:10F5D0008C0FC3DD3BC1ADCB9CF65F27B13F7630CE
:10F5E0002303DFD300C0DFD323037630B13F5F278F
:10F5F0009CF6ADCB3BC1C3DD8C0FAF373E3DC61C87
:10F6000071EA7EC5E0C4F8E85D1BC53C7138111194
:10F6100019DF8FC1CACA0FF51F26843F7931B5049F
:10F6200006D505C0BFD292016B2FD33F99282BF886
:10F6300099CCF2C072DC050EE536AE3D2B1EEDEB2B
:10F6400026C64AC483E7EF19423C2A39941275E072
:10F65000ECC1EEC984F3DA244E3F7432450633D64A
:10F6600014C0A6D100005A2EEC3FCD29BBF98CCD99
:10F67000B2C026DB7C0C1236143E8B1F6CEDD6C656
:10F68000BEC311E67D18B63BDA391314D5E152C278
:10F690001BC9FBF18E230E3F6733D50767D72DC0FB
:10F6A00095D06EFE412DFB3FFA2A4BFB87CE7CC0E6
:10F6B000E1D9F10A3635713EE720EFEE8FC73BC343
:10F6C000A3E40817203B823A8F153AE3C2C251C81F
:10F6D00074F03D22C53E53346409A1D84FC08ACF8F
:10F6E000DDFC212C0040212CDDFC8ACF4FC0A1D8AD
:10F6F00064095334C53E3D2274F051C8C2C23AE396
:10F700008F15823A203B0817A3E43BC38FC7EFEE67
:10F71000E720713E3635F10AE1D97CC087CE4BFB3C
:10F72000FA2AFB3F412D6EFE95D02DC067D7D50735
:10F7300067330E3F8E23FBF11BC952C2D5E1131470
:10F74000DA39B63B7D1811E6BEC3D6C66CED8B1F09
:10F75000143E12367C0C26DBB2C08CCDBBF9CD2911
:10F76000EC3F5A2E0000A6D114C033D645067432A1
:10F770004E3FDA2484F3EEC9ECC175E094122A39C5
:10F78000423CEF1983E74AC426C6EDEB2B1EAE3D83
:10F79000E536050E72DCF2C099CC2BF89928D33FE0
:10F7A0006B2F9201BFD205C006D5B5047931843FD5
:10F7B0001F260FF5CACA8FC119DF11117138C53C58
:10F7C0005D1BF8E8E0C47EC571EAC61C3E3DAF375C
:10F7D0008C0FC3DD3BC1ADCB9CF65F27B13F7630CC
:10F7E0002303DFD300C0DFD323037630B13F5F278D
:10F7F0009CF6ADCB3BC1C3DD8C0FAF373E3DC61C85
:10F8000071EA7EC5E0C4F8E85D1BC53C7138111192
:10F8100019DF8FC1CACA0FF51F26843F7931B5049D
:10F8200006D505C0BFD292016B2FD33F99282BF884
:10F8300099CCF2C072DC050EE536AE3D2B1EEDEB29
:10F8400026C64AC483E7EF19423C2A39941275E070
:10F85000ECC1EEC984F3DA244E3F7432450633D648
:10F8600014C0A6D10000DA39793174F03BC1E1D976
:10F870002B1EEC3F7D1806D5C2C29CF63635E53608
:10F88000BBF9BEC3BFD28F15B13FE72072DCB2C057
:10F890006CED6B2F203B23038FC799CC7C0C143E5F
:10F8A0009928A3E400C0A3E49928143E7C0C99CCC9
:10F8B0008FC72303203B6B2F6CEDB2C072DCE720B7
:10F8C000B13F8F15BFD2BEC3BBF9E53636359CF6C6
:10F8D000C2C206D57D18EC3F2B1EE1D93BC174F0A6
:10F8E0007931DA39000026C687CE8C0FC53E1F2637
:10F8F000D5E114C083E7FA2A3E3D6409CACA1BC990
:10F900004506423C412D71EA4FC019DF8E234E3F20
:10F91000941295D0E0C4DDFC7138673384F3ECC1F8
:10F9200067D75D1B00405D1B67D7ECC184F367336D
:10F930007138DDFCE0C495D094124E3F8E2319DF60
:10F940004FC071EA412D423C45061BC9CACA640931
:10F950003E3DFA2A83E714C0D5E11F26C53E8C0F31
:10F9600087CE26C60000DA39793174F03BC1E1D97F
:10F970002B1EEC3F7D1806D5C2C29CF63635E53607
:10F98000BBF9BEC3BFD28F15B13FE72072DCB2C056
:10F990006CED6B2F203B23038FC799CC7C0C143E5E
:10F9A0009928A3E400C0A3E49928143E7C0C99CCC8
:10F9B0008FC72303203B6B2F6CEDB2C072DCE720B6
:10F9C000B13F8F15BFD2BEC3BBF9E53636359CF6C5
:10F9D000C2C206D57D18EC3F2B1EE1D93BC174F0A5
:10F9E0007931DA39000026C687CE8C0FC53E1F2636
:10F9F000D5E114C083E7FA2A3E3D6409CACA1BC98F
:10FA00004506423C412D71EA4FC019DF8E234E3F1F
:10FA1000941295D0E0C4DDFC7138673384F3ECC1F7
:10FA200067D75D1B00405D1B67D7ECC184F367336C
:10FA30007138DDFCE0C495D094124E3F8E2319DF5F
:10FA40004FC071EA412D423C45061BC9CACA640930
:10FA50003E3DFA2A83E714C0D5E11F26C53E8C0F30
:10FA600087CE26C60000DA39793174F03BC1E1D97E
:10FA70002B1EEC3F7D1806D5C2C29CF63635E53606
:10FA8000BBF9BEC3BFD28F15B13FE72072DCB2C055
:10FA90006CED6B2F203B23038FC799CC7C0C143E5D
:10FAA0009928A3E400C0A3E49928143E7C0C99CCC7
:10FAB0008FC72303203B6B2F6CEDB2C072DCE720B5
:10FAC000B13F8F15BFD2BEC3BBF9E53636359CF6C4
:10FAD000C2C206D57D18EC3F2B1EE1D93BC174F0A4
:10FAE0007931DA39000026C687CE8C0FC53E1F2635
:10FAF000D5E114C083E7FA2A3E3D6409CACA1BC98E
:10FB00004506423C412D71EA4FC019DF8E234E3F1E
:10FB1000941295D0E0C4DDFC7138673384F3ECC1F6
:10FB200067D75D1B00405D1B67D7ECC184F367336B
:10FB30007138DDFCE0C495D094124E3F8E2319DF5E
:10FB40004FC071EA412D423C45061BC9CACA64092F
:10FB50003E3DFA2A83E714C0D5E11F26C53E8C0F2F
:10FB600087CE26C60000DA39793174F03BC1E1D97D
:10FB70002B1EEC3F7D1806D5C2C29CF63635E53605
:10FB8000BBF9BEC3BFD28F15B13FE72072DCB2C054
:10FB90006CED6B2F203B23038FC799CC7C0C143E5C
:10FBA0009928A3E400C0A3E49928143E7C0C99CCC6
:10FBB0008FC72303203B6B2F6CEDB2C072DCE720B4
:10FBC000B13F8F15BFD2BEC3BBF9E53636359CF6C3
:10FBD000C2C206D57D18EC3F2B1EE1D93BC174F0A3
:10FBE0007931DA39000026C687CE8C0FC53E1F2634
:10FBF000D5E114C083E7FA2A3E3D6409CACA1BC98D
:10FC00004506423C412D71EA4FC019DF8E234E3F1D
:10FC1000941295D0E0C4DDFC7138673384F3ECC1F5
:10FC200067D75D1B00405D1B67D7ECC184F367336A
:10FC30007138DDFCE0C495D094124E3F8E2319DF5D
:10FC40004FC071EA412D423C45061BC9CACA64092E
:10FC50003E3DFA2A83E714C0D5E11F26C53E8C0F2E
:10FC600087CE26C60000C53C1F2626DBC2C26EFE1C
:10FC7000423C5F2772DC52C2DDFCB63B9928C3DDF3
:10FC8000ECC14BFB203BCD2919DF8FC1BBF9823A78
:10FC9000FA2A75E03BC12BF8DA39212CD5E1F2C004
:10FCA0009CF62A39412D3AE3B2C00FF571385A2E2D
:10FCB000A3E47CC084F3AF376B2F11E64FC0FBF198
:10FCC000E536763083E72DC074F012367931F8E8E6
:10FCD00014C0EFEE3635743271EA05C06CED533462
:10FCE0006733EDEB00C0EDEB673353346CED05C0CB
:10FCF00071EA74323635EFEE14C0F8E87931123615
:10FD000074F02DC083E77630E536FBF14FC011E685
:10FD10006B2FAF3784F37CC0A3E45A2E71380FF5F4
:10FD2000B2C03AE3412D2A399CF6F2C0D5E1212C2C
:10FD3000DA392BF83BC175E0FA2A823ABBF98FC158
:10FD400019DFCD29203B4BFBECC1C3DD9928B63B25
:10FD5000DDFC52C272DC5F27423C6EFEC2C226DB73
:10FD60001F26C53C00003BC3E1D9DA243E3D920189
:10FD7000BEC3A1D88E23AE3D23034AC467D73D221C
:10FD8000143EB504E0C433D6E720713E45067EC577
:10FD900006D58B1FC53ED50726C6DFD32B1E0E3FCB
:10FDA0006409D6C6BFD2C61C4E3FF10A8FC7A6D182
:10FDB0005D1B843F7C0C51C895D0EF19B13F050EF7
:10FDC0001BC98ACF7D18D33F8C0FEEC987CE081789
:10FDD000EC3F1111CACA8CCD8F15FB3F9412ADCBED
:10FDE00099CC13140040131499CCADCB9412FB3F63
:10FDF0008F158CCDCACA1111EC3F081787CEEEC9FA
:10FE00008C0FD33F7D188ACF1BC9050EB13FEF1968
:10FE100095D051C87C0C843F5D1BA6D18FC7F10AD9
:10FE20004E3FC61CBFD2D6C664090E3F2B1EDFD381
:10FE300026C6D507C53E8B1F06D57EC54506713E35
:10FE4000E72033D6E0C4B504143E3D2267D74AC448
:10FE50002303AE3D8E23A1D8BEC392013E3DDA24DA
:10FE6000E1D93BC30000C53C1F2626DBC2C26EFEA3
:10FE7000423C5F2772DC52C2DDFCB63B9928C3DDF1
:10FE8000ECC14BFB203BCD2919DF8FC1BBF9823A76
:10FE9000FA2A75E03BC12BF8DA39212CD5E1F2C002
:10FEA0009CF62A39412D3AE3B2C00FF571385A2E2B
:10FEB000A3E47CC084F3AF376B2F11E64FC0FBF196
:10FEC000E536763083E72DC074F012367931F8E8E4
:10FED00014C0EFEE3635743271EA05C06CED533460
:10FEE0006733EDEB00C0EDEB673353346CED05C0C9
:10FEF00071EA74323635EFEE14C0F8E87931123613
:10FF000074F02DC083E77630E536FBF14FC011E683
:10FF10006B2FAF3784F37CC0A3E45A2E71380FF5F2
:10FF2000B2C03AE3412D2A399CF6F2C0D5E1212C2A
:10FF3000DA392BF83BC175E0FA2A823ABBF98FC156
:10FF400019DFCD29203B4BFBECC1C3DD9928B63B23
:10FF5000DDFC52C272DC5F27423C6EFEC2C226DB71
:10FF60001F26C53C00003BC3E1D9DA243E3D920187
:10FF7000BEC3A1D88E23AE3D23034AC467D73D221A
:10FF8000143EB504E0C433D6E720713E45067EC575
:10FF900006D58B1FC53ED50726C6DFD32B1E0E3FC9
:10FFA0006409D6C6BFD2C61C4E3FF10A8FC7A6D180
:10FFB0005D1B843F7C0C51C895D0EF19B13F050EF5
:10FFC0001BC98ACF7D18D33F8C0FEEC987CE081787
:10FFD000EC3F1111CACA8CCD8F15FB3F9412ADCBEB
:10FFE00099CC13140040131499CCADCB9412FB3F61
:10FFF0008F158CCDCACA1111EC3F081787CEEEC9F8
:020000040801F1
:100000008C0FD33F7D188ACF1BC9050EB13FEF1966
:1000100095D051C87C0C843F5D1BA6D18FC7F10AD7
:100020004E3FC61CBFD2D6C664090E3F2B1EDFD37F
:1000300026C6D507C53E8B1F06D57EC54506713E33
:10004000E72033D6E0C4B504143E3D2267D74AC446
:100050002303AE3D8E23A1D8BEC392013E3DDA24D8
:10006000E1D93BC301000001881001089410010888
:10007000000301020103010002030200010002016A
:1000800000020100020100020000004067331F2649
:100090003E3D6CED8F15BEC372DCCACA14C0DDFCD8
:1000A00067D779318C0F143E203B7D18E53619DF78
:1000B00045064FC095D006D53BC17C0CA3E4DA3988
:1000C0002B1E71384E3F6409412DBFD29CF6B2C041
:1000D0008FC7D5E126C65D1B84F3C53EFA2A6B2F78
:1000E000B13FBBF9E7201BC983E7E0C4ECC174F062
:1000F00087CE99282303EC3F36358E23423C71EAA4
:100100009412C2C2E1D999CC00C00000E1D9673392
:1001100094123E3D423C8F15363572DC230314C0E9
:1001200087CE67D7ECC18C0F83E7203BE720E5360D
:10013000B13F4506FA2A95D084F33BC126C6A3E415
:100140008FC72B1E9CF64E3F412D412D4E3F9CF6F6
:100150002B1E8FC7A3E426C63BC184F395D0FA2A91
:100160004506B13FE536E720203B83E78C0FECC125
:1001700067D787CE14C0230372DC36358F15423C17
:100180003E3D94126733E1D9000000C099CCE1D91B
:10019000C2C2941271EA423C8E233635EC3F2303EF
:1001A000992887CE74F0ECC1E0C483E71BC9E7202F
:1001B000BBF9B13F6B2FFA2AC53E84F35D1B26C6FF
:1001C000D5E18FC7B2C09CF6BFD2412D64094E3F26
:1001D00071382B1EDA39A3E47C0C3BC106D595D0CF
:1001E0004FC0450619DFE5367D18203B143E8C0FC5
:1001F000793167D7DDFC14C0CACA72DCBEC38F1563
:100200006CED3E3D1F266733004000001F2699CC51
:100210006CEDC2C2BEC371EACACA8E23DDFCEC3FDC
:1002200079319928143E74F07D18E0C419DF1BC998
:100230004FC0BBF906D56B2F7C0CC53EDA395D1B70
:100240007138D5E16409B2C0BFD2BFD2B2C064096F
:10025000D5E171385D1BDA39C53E7C0C6B2F06D5B4
:10026000BBF94FC01BC919DFE0C47D1874F0143E00
:1002700099287931EC3FDDFC8E23CACA71EABEC3EE
:10028000C2C26CED99CC1F260000004067331F26C8
:100290003E3D6CED8F15BEC372DCCACA14C0DDFCD6
:1002A00067D779318C0F143E203B7D18E53619DF76
:1002B00045064FC095D006D53BC17C0CA3E4DA3986
:1002C0002B1E71384E3F6409412DBFD29CF6B2C03F
:1002D0008FC7D5E126C65D1B84F3C53EFA2A6B2F76
:1002E000B13FBBF9E7201BC983E7E0C4ECC174F060
:1002F00087CE99282303EC3F36358E23423C71EAA2
:100300009412C2C2E1D999CC00C00000E1D9673390
:1003100094123E3D423C8F15363572DC230314C0E7
:1003200087CE67D7ECC18C0F83E7203BE720E5360B
:10033000B13F4506FA2A95D084F33BC126C6A3E413
:100340008FC72B1E9CF64E3F412D412D4E3F9CF6F4
:100350002B1E8FC7A3E426C63BC184F395D0FA2A8F
:100360004506B13FE536E720203B83E78C0FECC123
:1003700067D787CE14C0230372DC36358F15423C15
:100380003E3D94126733E1D9000000C099CCE1D919
:10039000C2C2941271EA423C8E233635EC3F2303ED
:1003A000992887CE74F0ECC1E0C483E71BC9E7202D
:1003B000BBF9B13F6B2FFA2AC53E84F35D1B26C6FD
:1003C000D5E18FC7B2C09CF6BFD2412D64094E3F24
:1003D00071382B1EDA39A3E47C0C3BC106D595D0CD
:1003E0004FC0450619DFE5367D18203B143E8C0FC3
:1003F000793167D7DDFC14C0CACA72DCBEC38F1561
:100400006CED3E3D1F266733004000001F2699CC4F
:100410006CEDC2C2BEC371EACACA8E23DDFCEC3FDA
:1004200079319928143E74F07D18E0C419DF1BC996
:100430004FC0BBF906D56B2F7C0CC53EDA395D1B6E
:100440007138D5E16409B2C0BFD2BFD2B2C064096D
:10045000D5E171385D1BDA39C53E7C0C6B2F06D5B2
:10046000BBF94FC01BC919DFE0C47D1874F0143EFE
:1004700099287931EC3FDDFC8E23CACA71EABEC3EC
:10048000C2C26CED99CC1F260000004067331F26C6
:100490003E3D6CED8F15BEC372DCCACA14C0DDFCD4
:1004A00067D779318C0F143E203B7D18E53619DF74
:1004B00045064FC095D006D53BC17C0CA3E4DA3984
:1004C0002B1E71384E3F6409412DBFD29CF6B2C03D
:1004D0008FC7D5E126C65D1B84F3C53EFA2A6B2F74
:1004E000B13FBBF9E7201BC983E7E0C4ECC174F05E
:1004F00087CE99282303EC3F36358E23423C71EAA0
:100500009412C2C2E1D999CC00C00000E1D967338E
:1005100094123E3D423C8F15363572DC230314C0E5
:1005200087CE67D7ECC18C0F83E7203BE720E53609
:10053000B13F4506FA2A95D084F33BC126C6A3E411
:100540008FC72B1E9CF64E3F412D412D4E3F9CF6F2
:100550002B1E8FC7A3E426C63BC184F395D0FA2A8D
:100560004506B13FE536E720203B83E78C0FECC121
:1005700067D787CE14C0230372DC36358F15423C13
:100580003E3D94126733E1D9000000C099CCE1D917
:10059000C2C2941271EA423C8E233635EC3F2303EB
:1005A000992887CE74F0ECC1E0C483E71BC9E7202B
:1005B000BBF9B13F6B2FFA2AC53E84F35D1B26C6FB
:1005C000D5E18FC7B2C09CF6BFD2412D64094E3F22
:1005D00071382B1EDA39A3E47C0C3BC106D595D0CB
:1005E0004FC0450619DFE5367D18203B143E8C0FC1
:1005F000793167D7DDFC14C0CACA72DCBEC38F155F
:100600006CED3E3D1F266733004000001F2699CC4D
:100610006CEDC2C2BEC371EACACA8E23DDFCEC3FD8
:1006200079319928143E74F07D18E0C419DF1BC994
:100630004FC0BBF906D56B2F7C0CC53EDA395D1B6C
:100640007138D5E16409B2C0BFD2BFD2B2C064096B
:10065000D5E171385D1BDA39C53E7C0C6B2F06D5B0
:10066000BBF94FC01BC919DFE0C47D1874F0143EFC
:1006700099287931EC3FDDFC8E23CACA71EABEC3EA
:10068000C2C26CED99CC1F260000004067331F26C4
:100690003E3D6CED8F15BEC372DCCACA14C0DDFCD2
:1006A00067D779318C0F143E203B7D18E53619DF72
:1006B00045064FC095D006D53BC17C0CA3E4DA3982
:1006C0002B1E71384E3F6409412DBFD29CF6B2C03B
:1006D0008FC7D5E126C65D1B84F3C53EFA2A6B2F72
:1006E000B13FBBF9E7201BC983E7E0C4ECC174F05C
:1006F00087CE99282303EC3F36358E23423C71EA9E
:100700009412C2C2E1D999CC00C00000E1D967338C
:1007100094123E3D423C8F15363572DC230314C0E3
:1007200087CE67D7ECC18C0F83E7203BE720E53607
:10073000B13F4506FA2A95D084F33BC126C6A3E40F
:100740008FC72B1E9CF64E3F412D412D4E3F9CF6F0
:100750002B1E8FC7A3E426C63BC184F395D0FA2A8B
:100760004506B13FE536E720203B83E78C0FECC11F
:1007700067D787CE14C0230372DC36358F15423C11
:100780003E3D94126733E1D9000000C099CCE1D915
:10079000C2C2941271EA423C8E233635EC3F2303E9
:1007A000992887CE74F0ECC1E0C483E71BC9E72029
:1007B000BBF9B13F6B2FFA2AC53E84F35D1B26C6F9
:1007C000D5E18FC7B2C09CF6BFD2412D64094E3F20
:1007D00071382B1EDA39A3E47C0C3BC106D595D0C9
:1007E0004FC0450619DFE5367D18203B143E8C0FBF
:1007F000793167D7DDFC14C0CACA72DCBEC38F155D
:100800006CED3E3D1F266733004000001F2699CC4B
:100810006CEDC2C2BEC371EACACA8E23DDFCEC3FD6
:1008200079319928143E74F07D18E0C419DF1BC992
:100830004FC0BBF906D56B2F7C0CC53EDA395D1B6A
:100840007138D5E16409B2C0BFD2BFD2B2C0640969
:10085000D5E171385D1BDA39C53E7C0C6B2F06D5AE
:10086000BBF94FC01BC919DFE0C47D1874F0143EFA
:1008700099287931EC3FDDFC8E23CACA71EABEC3E8
:10088000C2C26CED99CC1F260000004074325F2775
:10089000143E74F0EF197EC5D5E18FC7F2C00FF595
:1008A00095D0FA2AB504D33F36358E23C53CEDEBFF
:1008B0008F15BEC3C3DDEEC94FC0BBF9DFD35A2EBF
:1008C00064094E3FAF378B1F203B83E7111152C2A3
:1008D000E1D999CC05C06EFE67D77931050E713E1E
:1008E000DA395D1B2A393AE37C0C3BC133D68ACF17
:1008F00014C0230326DB533494123E3DB63B081745
:10090000E53619DFD5077CC0BFD2BFD27CC0D50782
:1009100019DFE5360817B63B3E3D9412533426DB0B
:10092000230314C08ACF33D63BC17C0C3AE32A3967
:100930005D1BDA39713E050E793167D76EFE05C051
:1009400099CCE1D952C2111183E7203B8B1FAF37FD
:100950004E3F64095A2EDFD3BBF94FC0EEC9C3DD49
:10096000BEC38F15EDEBC53C8E233635D33FB504A2
:10097000FA2A95D00FF5F2C08FC7D5E17EC5EF19E1
:1009800074F0143E5F277432004000005F278CCD66
:1009900074F0ECC17EC511E68FC72B1E0FF50E3F1C
:1009A000FA2A6B2FD33F4BFB8E23CACAEDEB3BC316
:1009B000BEC371EAEEC93D22BBF9B13F5A2E212CCC
:1009C0004E3F9CF68B1F51C883E7E0C452C2EFEE46
:1009D00099CC1F266EFEFB3F79319928713EFBF1C1
:1009E0005D1B26C63AE3D6C63BC184F38ACFCD2928
:1009F0002303EC3F5334DA243E3D6CED08174AC420
:100A000019DF1BC97CC02BF8BFD2412DD507843F0D
:100A1000E536E720B63BF8E89412C2C226DBADCB40
:100A200014C0DDFC33D676307C0CC53E2A39C61C9A
:100A3000DA39A3E4050E8FC167D787CE05C09201CE
:100A4000E1D967331111AE3D203B7D18AF3775E01A
:100A50006409B2C0DFD3A6D14FC04506C3DD12364C
:100A60008F15423CC53C1314363572DCB5042DC0DD
:100A700095D006D5F2C0F10AD5E17138EF19823A66
:100A8000143E8C0F7432A1D8000000C08CCDA1D8C8
:100A9000ECC18C0F11E6823A2B1E71380E3FF10A21
:100AA0006B2F06D54BFB2DC0CACA72DC3BC3131497
:100AB00071EA423C3D221236B13F4506212CA6D1B7
:100AC0009CF6B2C051C875E0E0C47D18EFEEAE3DB3
:100AD0001F266733FB3F9201992887CEFBF18FC118
:100AE00026C6A3E4D6C6C61C84F3C53ECD297630FF
:100AF000EC3FDDFCDA24ADCB6CEDC2C24AC4F8E8B1
:100B00001BC9E7202BF8843F412D412D843F2BF852
:100B1000E7201BC9F8E84AC4C2C26CEDADCBDA24A9
:100B2000DDFCEC3F7630CD29C53E84F3C61CD6C62D
:100B3000A3E426C68FC1FBF187CE99289201FB3F23
:100B400067331F26AE3DEFEE7D18E0C475E051C857
:100B5000B2C09CF6A6D1212C4506B13F12363D22EB
:100B6000423C71EA13143BC372DCCACA2DC04BFB72
:100B700006D56B2FF10A0E3F71382B1E823A11E613
:100B80008C0FECC1A1D88CCD00C00000A1D874326C
:100B90008C0F143E823AEF197138D5E1F10AF2C098
:100BA00006D595D02DC0B50472DC36351314C53C7E
:100BB000423C8F151236C3DD45064FC0A6D1DFD3A8
:100BC000B2C0640975E0AF377D18203BAE3D11110E
:100BD0006733E1D9920105C087CE67D78FC1050E73
:100BE000A3E4DA39C61C2A39C53E7C0C763033D6EC
:100BF000DDFC14C0ADCB26DBC2C29412F8E8B63BD4
:100C0000E720E536843FD507412DBFD22BF87CC0C5
:100C10001BC919DF4AC408176CED3E3DDA24533472
:100C2000EC3F2303CD298ACF84F33BC1D6C63AE3F8
:100C300026C65D1BFBF1713E99287931FB3F6EFEA4
:100C40001F2699CCEFEE52C2E0C483E751C88B1F38
:100C50009CF64E3F212C5A2EB13FBBF93D22EEC9E6
:100C600071EABEC33BC3EDEBCACA8E234BFBD33F35
:100C70006B2FFA2A0E3F0FF52B1E8FC711E67EC58C
:100C8000ECC174F08CCD5F270000004074325F2708
:100C9000143E74F0EF197EC5D5E18FC7F2C00FF591
:100CA00095D0FA2AB504D33F36358E23C53CEDEBFB
:100CB0008F15BEC3C3DDEEC94FC0BBF9DFD35A2EBB
:100CC00064094E3FAF378B1F203B83E7111152C29F
:100CD000E1D999CC05C06EFE67D77931050E713E1A
:100CE000DA395D1B2A393AE37C0C3BC133D68ACF13
:100CF00014C0230326DB533494123E3DB63B081741
:100D0000E53619DFD5077CC0BFD2BFD27CC0D5077E
:100D100019DFE5360817B63B3E3D9412533426DB07
:100D2000230314C08ACF33D63BC17C0C3AE32A3963
:100D30005D1BDA39713E050E793167D76EFE05C04D
:100D400099CCE1D952C2111183E7203B8B1FAF37F9
:100D50004E3F64095A2EDFD3BBF94FC0EEC9C3DD45
:100D6000BEC38F15EDEBC53C8E233635D33FB5049E
:100D7000FA2A95D00FF5F2C08FC7D5E17EC5EF19DD
:100D800074F0143E5F277432004000005F278CCD62
:100D900074F0ECC17EC511E68FC72B1E0FF50E3F18
:100DA000FA2A6B2FD33F4BFB8E23CACAEDEB3BC312
:100DB000BEC371EAEEC93D22BBF9B13F5A2E212CC8
:100DC0004E3F9CF68B1F51C883E7E0C452C2EFEE42
:100DD00099CC1F266EFEFB3F79319928713EFBF1BD
:100DE0005D1B26C63AE3D6C63BC184F38ACFCD2924
:100DF0002303EC3F5334DA243E3D6CED08174AC41C
:100E000019DF1BC97CC02BF8BFD2412DD507843F09
:100E1000E536E720B63BF8E89412C2C226DBADCB3C
:100E200014C0DDFC33D676307C0CC53E2A39C61C96
:100E3000DA39A3E4050E8FC167D787CE05C09201CA
:100E4000E1D967331111AE3D203B7D18AF3775E016
:100E50006409B2C0DFD3A6D14FC04506C3DD123648
:100E60008F15423CC53C1314363572DCB5042DC0D9
:100E700095D006D5F2C0F10AD5E17138EF19823A62
:100E8000143E8C0F7432A1D8000000C08CCDA1D8C4
:100E9000ECC18C0F11E6823A2B1E71380E3FF10A1D
:100EA0006B2F06D54BFB2DC0CACA72DC3BC3131493
:100EB00071EA423C3D221236B13F4506212CA6D1B3
:100EC0009CF6B2C051C875E0E0C47D18EFEEAE3DAF
:100ED0001F266733FB3F9201992887CEFBF18FC114
:100EE00026C6A3E4D6C6C61C84F3C53ECD297630FB
:100EF000EC3FDDFCDA24ADCB6CEDC2C24AC4F8E8AD
:100F00001BC9E7202BF8843F412D412D843F2BF84E
:100F1000E7201BC9F8E84AC4C2C26CEDADCBDA24A5
:100F2000DDFCEC3F7630CD29C53E84F3C61CD6C629
:100F3000A3E426C68FC1FBF187CE99289201FB3F1F
:100F400067331F26AE3DEFEE7D18E0C475E051C853
:100F5000B2C09CF6A6D1212C4506B13F12363D22E7
:100F6000423C71EA13143BC372DCCACA2DC04BFB6E
:100F700006D56B2FF10A0E3F71382B1E823A11E60F
:100F80008C0FECC1A1D88CCD00C00000A1D8743268
:100F90008C0F143E823AEF197138D5E1F10AF2C094
:100FA00006D595D02DC0B50472DC36351314C53C7A
:100FB000423C8F151236C3DD45064FC0A6D1DFD3A4
:100FC000B2C0640975E0AF377D18203BAE3D11110A
:100FD0006733E1D9920105C087CE67D78FC1050E6F
:100FE000A3E4DA39C61C2A39C53E7C0C763033D6E8
:100FF000DDFC14C0ADCB26DBC2C29412F8E8B63BD0
:10100000E720E536843FD507412DBFD22BF87CC0C1
:101010001BC919DF4AC408176CED3E3DDA2453346E
:10102000EC3F2303CD298ACF84F33BC1D6C63AE3F4
:1010300026C65D1BFBF1713E99287931FB3F6EFEA0
:101040001F2699CCEFEE52C2E0C483E751C88B1F34
:101050009CF64E3F212C5A2EB13FBBF93D22EEC9E2
:1010600071EABEC33BC3EDEBCACA8E234BFBD33F31
:101070006B2FFA2A0E3F0FF52B1E8FC711E67EC588
:10108000ECC174F08CCD5F270205070A0C0F111418
:1010900016191B1E0306080B0D101215171A1C1F1C
:1010A0000104201D0E0913180000000000000000BC
:1010B000010203040607080900000040203B83E703
:1010C000BFD2BFD283E7203B0040000083E7E0C4EB
:1010D000BFD2412D203B7D18000000C0E0C47D1828
:1010E000412D412D7D18E0C400C000007D18203B3B
:1010F000412DBFD2E0C483E700000040203B83E7DE
:10110000BFD2BFD283E7203B0040000083E7E0C4AA
:10111000BFD2412D203B7D18000000C0E0C47D18E7
:10112000412D412D7D18E0C400C000007D18203BFA
:10113000412DBFD2E0C483E700000040203B83E79D
:10114000BFD2BFD283E7203B0040000083E7E0C46A
:10115000BFD2412D203B7D18000000C0E0C47D18A7
:10116000412D412D7D18E0C400C000007D18203BBA
:10117000412DBFD2E0C483E700000040203B83E75D
:10118000BFD2BFD283E7203B0040000083E7E0C42A
:10119000BFD2412D203B7D18000000C0E0C47D1867
:1011A000412D412D7D18E0C400C000007D18203B7A
:1011B000412DBFD2E0C483E700000040203B83E71D
:1011C000BFD2BFD283E7203B0040000083E7E0C4EA
:1011D000BFD2412D203B7D18000000C0E0C47D1827
:1011E000412D412D7D18E0C400C000007D18203B3A
:1011F000412DBFD2E0C483E700000040203B83E7DD
:10120000BFD2BFD283E7203B0040000083E7E0C4A9
:10121000BFD2412D203B7D18000000C0E0C47D18E6
:10122000412D412D7D18E0C400C000007D18203BF9
:10123000412DBFD2E0C483E700000040203B83E79C
:10124000BFD2BFD283E7203B0040000083E7E0C469
:10125000BFD2412D203B7D18000000C0E0C47D18A6
:10126000412D412D7D18E0C400C000007D18203BB9
:10127000412DBFD2E0C483E700000040203B83E75C
:10128000BFD2BFD283E7203B0040000083E7E0C429
:10129000BFD2412D203B7D18000000C0E0C47D1866
:1012A000412D412D7D18E0C400C000007D18203B79
:1012B000412DBFD2E0C483E700000040203B83E71C
:1012C000BFD2BFD283E7203B0040000083E7E0C4E9
:1012D000BFD2412D203B7D18000000C0E0C47D1826
:1012E000412D412D7D18E0C400C000007D18203B39
:1012F000412DBFD2E0C483E700000040203B83E7DC
:10130000BFD2BFD283E7203B0040000083E7E0C4A8
:10131000BFD2412D203B7D18000000C0E0C47D18E5
:10132000412D412D7D18E0C400C000007D18203BF8
:10133000412DBFD2E0C483E700000040203B83E79B
:10134000BFD2BFD283E7203B0040000083E7E0C468
:10135000BFD2412D203B7D18000000C0E0C47D18A5
:10136000412D412D7D18E0C400C000007D18203BB8
:10137000412DBFD2E0C483E700000040203B83E75B
:10138000BFD2BFD283E7203B0040000083E7E0C428
:10139000BFD2412D203B7D18000000C0E0C47D1865
:1013A000412D412D7D18E0C400C000007D18203B78
:1013B000412DBFD2E0C483E700000040203B83E71B
:1013C000BFD2BFD283E7203B0040000083E7E0C4E8
:1013D000BFD2412D203B7D18000000C0E0C47D1825
:1013E000412D412D7D18E0C400C000007D18203B38
:1013F000412DBFD2E0C483E700000040203B83E7DB
:10140000BFD2BFD283E7203B0040000083E7E0C4A7
:10141000BFD2412D203B7D18000000C0E0C47D18E4
:10142000412D412D7D18E0C400C000007D18203BF7
:10143000412DBFD2E0C483E700000040203B83E79A
:10144000BFD2BFD283E7203B0040000083E7E0C467
:10145000BFD2412D203B7D18000000C0E0C47D18A4
:10146000412D412D7D18E0C400C000007D18203BB7
:10147000412DBFD2E0C483E700000040203B83E75A
:10148000BFD2BFD283E7203B0040000083E7E0C427
:10149000BFD2412D203B7D18000000C0E0C47D1864
:1014A000412D412D7D18E0C400C000007D18203B77
:1014B000412DBFD2E0C483E700000040203B83E71A
:1014C000BFD2BFD283E7203B0040000083E7E0C4E7
:1014D000BFD2412D203B7D18000000C0E0C47D1824
:1014E000412D412D7D18E0C400C000007D18203B37
:1014F000412DBFD2E0C483E700000040203B83E7DA
:10150000BFD2BFD283E7203B0040000083E7E0C4A6
:10151000BFD2412D203B7D18000000C0E0C47D18E3
:10152000412D412D7D18E0C400C000007D18203BF6
:10153000412DBFD2E0C483E700000040203B83E799
:10154000BFD2BFD283E7203B0040000083E7E0C466
:10155000BFD2412D203B7D18000000C0E0C47D18A3
:10156000412D412D7D18E0C400C000007D18203BB6
:10157000412DBFD2E0C483E700000040203B83E759
:10158000BFD2BFD283E7203B0040000083E7E0C426
:10159000BFD2412D203B7D18000000C0E0C47D1863
:1015A000412D412D7D18E0C400C000007D18203B76
:1015B000412DBFD2E0C483E700000040203B83E719
:1015C000BFD2BFD283E7203B0040000083E7E0C4E6
:1015D000BFD2412D203B7D18000000C0E0C47D1823
:1015E000412D412D7D18E0C400C000007D18203B36
:1015F000412DBFD2E0C483E700000040203B83E7D9
:10160000BFD2BFD283E7203B0040000083E7E0C4A5
:10161000BFD2412D203B7D18000000C0E0C47D18E2
:10162000412D412D7D18E0C400C000007D18203BF5
:10163000412DBFD2E0C483E700000040203B83E798
:10164000BFD2BFD283E7203B0040000083E7E0C465
:10165000BFD2412D203B7D18000000C0E0C47D18A2
:10166000412D412D7D18E0C400C000007D18203BB5
:10167000412DBFD2E0C483E700000040203B83E758
:10168000BFD2BFD283E7203B0040000083E7E0C425
:10169000BFD2412D203B7D18000000C0E0C47D1862
:1016A000412D412D7D18E0C400C000007D18203B75
:1016B000412DBFD2E0C483E700000040203B83E718
:1016C000BFD2BFD283E7203B0040000083E7E0C4E5
:1016D000BFD2412D203B7D18000000C0E0C47D1822
:1016E000412D412D7D18E0C400C000007D18203B35
:1016F000412DBFD2E0C483E700000040203B83E7D8
:10170000BFD2BFD283E7203B0040000083E7E0C4A4
:10171000BFD2412D203B7D18000000C0E0C47D18E1
:10172000412D412D7D18E0C400C000007D18203BF4
:10173000412DBFD2E0C483E700000040203B83E797
:10174000BFD2BFD283E7203B0040000083E7E0C464
:10175000BFD2412D203B7D18000000C0E0C47D18A1
:10176000412D412D7D18E0C400C000007D18203BB4
:10177000412DBFD2E0C483E700000040203B83E757
:10178000BFD2BFD283E7203B0040000083E7E0C424
:10179000BFD2412D203B7D18000000C0E0C47D1861
:1017A000412D412D7D18E0C400C000007D18203B74
:1017B000412DBFD2E0C483E700000040203B83E717
:1017C000BFD2BFD283E7203B0040000083E7E0C4E4
:1017D000BFD2412D203B7D18000000C0E0C47D1821
:1017E000412D412D7D18E0C400C000007D18203B34
:1017F000412DBFD2E0C483E700000040203B83E7D7
:10180000BFD2BFD283E7203B0040000083E7E0C4A3
:10181000BFD2412D203B7D18000000C0E0C47D18E0
:10182000412D412D7D18E0C400C000007D18203BF3
:10183000412DBFD2E0C483E700000040203B83E796
:10184000BFD2BFD283E7203B0040000083E7E0C463
:10185000BFD2412D203B7D18000000C0E0C47D18A0
:10186000412D412D7D18E0C400C000007D18203BB3
:10187000412DBFD2E0C483E700000040203B83E756
:10188000BFD2BFD283E7203B0040000083E7E0C423
:10189000BFD2412D203B7D18000000C0E0C47D1860
:1018A000412D412D7D18E0C400C000007D18203B73
:1018B000412DBFD2E0C483E700000040B63BF8E80A
:1018C00006D595D03AE32A39B13F4506EFEE52C22C
:1018D00099CC1F2612363D227C0C3BC1F2C0F10A86
:1018E000E720E5365F278CCDC2C26CEDB504D33F4F
:1018F000DA39A3E4A6D1DFD383E7203BFB3F920193
:1019000071EABEC38ACFCD2971382B1ED5077CC0A2
:10191000ECC18C0FDA2453348E23CACA8FC1FBF179
:1019200064094E3FAF3775E087CE67D7EDEBC53C16
:10193000EC3FDDFC11E67EC5BFD2412D823AEF19A6
:10194000230314C03BC31314992879318B1F51C84A
:10195000B2C09CF6050E713E363572DCADCB26DB8F
:1019600074F0143E843F2BF8D5E18FC733D6763020
:10197000423C8F156EFE05C0E0C47D18212C5A2E06
:101980005D1B26C62DC04BFB94123E3D7432A1D880
:101990001BC919DF0FF50E3FC53E84F3C3DDEEC949
:1019A000E1D96733AE3D1111BBF94FC0D6C6C61C95
:1019B0006B2FFA2A08174AC400C000000817B63B6C
:1019C0006B2F06D5D6C63AE3BBF9B13FAE3DEFEE7D
:1019D000E1D999CCC3DD1236C53E7C0C0FF5F2C0BF
:1019E0001BC9E72074325F279412C2C22DC0B50410
:1019F0005D1BDA39212CA6D1E0C483E76EFEFB3FE4
:101A0000423C71EA33D68ACFD5E17138843FD5079D
:101A100074F0ECC1ADCBDA2436358E23050E8FC1C0
:101A2000B2C064098B1FAF37992887CE3BC3EDEB5B
:101A30002303EC3F823A11E6BFD2BFD211E6823ACD
:101A4000EC3F2303EDEB3BC387CE9928AF378B1FC9
:101A50006409B2C08FC1050E8E233635DA24ADCBB2
:101A6000ECC174F0D507843F7138D5E18ACF33D605
:101A700071EA423CFB3F6EFE83E7E0C4A6D1212C15
:101A8000DA395D1BB5042DC0C2C294125F277432CF
:101A9000E7201BC9F2C00FF57C0CC53E1236C3DD32
:101AA00099CCE1D9EFEEAE3DB13FBBF93AE3D6C6F2
:101AB00006D56B2FB63B0817000000C04AC40817B4
:101AC000FA2A6B2FC61CD6C64FC0BBF91111AE3D0A
:101AD0006733E1D9EEC9C3DD84F3C53E0E3F0FF590
:101AE00019DF1BC9A1D874323E3D94124BFB2DC0A7
:101AF00026C65D1B5A2E212C7D18E0C405C06EFE43
:101B00008F15423C763033D68FC7D5E12BF8843F12
:101B1000143E74F026DBADCB72DC3635713E050E1B
:101B20009CF6B2C051C88B1F7931992813143BC35E
:101B300014C02303EF19823A412DBFD27EC511E6AE
:101B4000DDFCEC3FC53CEDEB67D787CE75E0AF37EA
:101B50004E3F6409FBF18FC1CACA8E235334DA2485
:101B60008C0FECC17CC0D5072B1E7138CD298ACFD4
:101B7000BEC371EA9201FB3F203B83E7DFD3A6D1CE
:101B8000A3E4DA39D33FB5046CEDC2C28CCD5F2734
:101B9000E536E720F10AF2C03BC17C0C3D2212364B
:101BA0001F2699CC52C2EFEE4506B13F2A393AE3DF
:101BB00095D006D5F8E8B63B00400000F8E84AC4E6
:101BC00095D0FA2A2A39C61C45064FC052C21111B7
:101BD0001F2667333D22EEC93BC184F3F10A0E3F55
:101BE000E53619DF8CCDA1D86CED3E3DD33F4BFBE4
:101BF000A3E426C6DFD35A2E203B7D18920105C0F0
:101C0000BEC38F15CD2976302B1E8FC77CC02BF815
:101C10008C0F143E533426DBCACA72DCFBF1713ED2
:101C20004E3F9CF675E051C867D77931C53C131417
:101C3000DDFC14C07EC5EF19412D412DEF197EC585
